:10000000F4FB0220990100009D3B0100553B0100DB
:10001000553B0100553B0100553B0100553B01009C
:10002000553B0100553B0100553B01009D3B010044
:100030009D3B0100553B0100A9550100F957010006
:100040009D3B01009D3B01009D3B01009D3B01004C
:100050009D3B01009D3B01009D3B01009D3B01003C
:100060009D3B01009D3B01009D3B01009D3B01002C
:100070009D3B01009D3B01009D3B01009D3B01001C
:100080009D3B01009D3B01009D3B01009D3B01000C
:100090009D3B01009D3B01009D3B01009D3B0100FC
:1000A000D1360100E5360100B937010049380100B9
:1000B0009D3B01009D3B01009D3B010099590100C2
:1000C0009D3B0100C55A01009D3B0100F15B010011
:1000D0009D3B0100E95C01009D3B0100A936010048
:1000E0009D3B01009D3B01009D3B01009D3B0100AC
:1000F0009D3B01009D3B01009D3B01009D3B01009C
:100100000D370100253701003D370100553701004B
:100110009D3B0100B94701009D3B01009D3B010053
:100120009D3B01009D3B01009D3B01009D3B01006B
:100130009D3B01009D3B01009D3B01009D3B01005B
:100140009D3B01009D3B0100E15D01009D3B0100E5
:10015000D95E01009D3B01009D3B01009D3B0100DC
:100160009D3B0100BD360100F93601009D3B0100B9
:100170009D3B01009D3B01009D3B01009D3B01001B
:100180009D3B0100793701009D3B01009D3B010033
:100190009D3B01009D3B0100584B4CF2205210B595
:1001A0001A804DF628121A8000BF00BF13F0FAFC27
:1001B000534B4FF030621A60524A9A60524ADA60EA
:1001C000524B4FF470021A60514A136813F4807353
:1001D00004D150490B604FF4A85313604E4B1A786A
:1001E000110703D51A7842F008021A704B4B4C499C
:1001F0002A221A704B4A4C4B8B4204D252F8040FFD
:1002000043F8040BF8E7494B494900228B4202D2DC
:1002100043F8042BFAE74749474A002352F82300E2
:1002200041F823000133662BF8D1444B444A802126
:1002300003F8011B9342FBD1424B3E4A1A60424BEA
:100240008A221A70A3F5805324225A70A0221A70B1
:100250009A799207FCD59A79D406FCD43B4A9379D3
:1002600003F00C03082B394BF9D103221A714622F3
:100270005A719A799006FCD5344A9179334B4906E4
:10028000FBD5334A4FF08271116009215160202261
:100290001A709A7902F00C020C2AFAD12D4B2E4AD0
:1002A0001A602E4B2E4A1A6000225A60072243F829
:1002B000042C2C4AC3F80C2D62B613F02FFD154BFD
:1002C0001B68DA0705D5284813F016FD274B284A86
:1002D0001A60284B1B785B0609D5244C244B2268F6
:1002E0009A4204D1204813F007FD0023236015F043
:1002F000FDFE13F05DFC13F08DFBFEE70E200540C4
:1003000030800440823F04000100002B88ED00E0B3
:1003100010D0034014D0034002D0074000E0074053
:100320006014FF1F0CC20100F806FF1F6014FF1FBE
:10033000E8B6FF1F0002FF1F0000000000E400E01D
:1003400056E400E008ED00E00050064000400640A2
:100350004480044004800440C010050014E000E024
:10036000BFD4010000002020D5E4B4661CE00340A7
:10037000A5C3945A00F00740FFFFFFFFFFFFFFFFF8
:10038000FFFFFFFFFFFFFFFFFFFFFFFFFFFFFFFF7D
:10039000FFFFFFFFFFFFFFFFFFFFFFFFFFFFFFFF6D
:1003A000FFFFFFFFFFFFFFFFFFFFFFFFFFFFFFFF5D
:1003B000FFFFFFFFFFFFFFFFFFFFFFFFFFFFFFFF4D
:1003C000FFFFFFFFFFFFFFFFFFFFFFFFFFFFFFFF3D
:1003D000FFFFFFFFFFFFFFFFFFFFFFFFFFFFFFFF2D
:1003E000FFFFFFFFFFFFFFFFFFFFFFFFFFFFFFFF1D
:1003F000FFFFFFFFFFFFFFFFFFFFFFFFFFFFFFFF0D
:10040000FFFFFFFFFFFFFFFFFFFFFFFFDEF9FFFF23
:1004100010B5054C237833B9044B13B10448AFF33E
:1004200000800123237010BD6014FF1F0000000036
:1004300008C20100084B10B51BB108490848AFF3CA
:1004400000800848036803B910BD074B002BFBD0A0
:10045000BDE81040184700BF000000006414FF1FF3
:1004600008C201006014FF1F00000000034B586821
:1004700010B103681B681847704700BF3CB1FF1FED
:10048000034B986810B103681B681847704700BF9A
:100490003CB1FF1F034BD86810B103681B681847B5
:1004A000704700BF3CB1FF1F034B186910B10368D0
:1004B0001B681847704700BF3CB1FF1F034B5869CA
:1004C00010B103681B681847704700BF3CB1FF1F9D
:1004D000034B986910B103681B681847704700BF49
:1004E0003CB1FF1F034BD86910B103681B68184764
:1004F000704700BF3CB1FF1F034B186A10B103687F
:100500001B681847704700BF3CB1FF1F034B586A78
:1005100010B103681B681847704700BF3CB1FF1F4C
:10052000034B986A10B103681B681847704700BFF7
:100530003CB1FF1F034BD86A10B103681B68184712
:10054000704700BF3CB1FF1F034B186B10B103682D
:100550001B681847704700BF3CB1FF1F034B586B27
:1005600010B103681B681847704700BF3CB1FF1FFC
:10057000034B986B10B103681B681847704700BFA6
:100580003CB1FF1F034BD86B10B103681B681847C1
:10059000704700BF3CB1FF1F034B186C10B10368DC
:1005A0001B681847704700BF3CB1FF1F034B586CD6
:1005B00010B103681B681847704700BF3CB1FF1FAC
:1005C000034B986C10B103681B681847704700BF55
:1005D0003CB1FF1F034BD86C10B103681B68184770
:1005E000704700BF3CB1FF1F034B186D10B103688B
:1005F0001B681847704700BF3CB1FF1F034B586D85
:1006000010B103681B681847704700BF3CB1FF1F5B
:10061000034B986D10B103681B681847704700BF03
:100620003CB1FF1F034BD86D10B103681B6818471E
:10063000704700BF3CB1FF1F034B186E10B1036839
:100640001B681847704700BF3CB1FF1F034B586E33
:1006500010B103681B681847704700BF3CB1FF1F0B
:10066000034B986E10B103681B681847704700BFB2
:100670003CB1FF1F034BD86E10B103681B681847CD
:10068000704700BF3CB1FF1F034B186F10B10368E8
:100690001B681847704700BF3CB1FF1F034B586FE2
:1006A00010B103681B681847704700BF3CB1FF1FBB
:1006B000034B986F10B103681B681847704700BF61
:1006C0003CB1FF1F034BD86F10B103681B6818477C
:1006D000704700BF3CB1FF1F034BD3F8800010B13F
:1006E00003681B68184770473CB1FF1F034BD3F8E2
:1006F000840010B103681B68184770473CB1FF1FA6
:10070000034BD3F8880010B103681B681847704783
:100710003CB1FF1F034BD3F88C0010B103681B687A
:10072000184770473CB1FF1F034BD3F8900010B13E
:1007300003681B68184770473CB1FF1F034BD3F891
:10074000940010B103681B68184770473CB1FF1F45
:10075000034BD3F8980010B103681B681847704723
:100760003CB1FF1F034BD3F89C0010B103681B681A
:10077000184770473CB1FF1F034BD3F8A00010B1DE
:1007800003681B68184770473CB1FF1F034BD3F841
:10079000A40010B103681B68184770473CB1FF1FE5
:1007A000034BD3F8A80010B103681B6818477047C3
:1007B0003CB1FF1F034BD3F8AC0010B103681B68BA
:1007C000184770473CB1FF1F034BD3F8B00010B17E
:1007D00003681B68184770473CB1FF1F034BD3F8F1
:1007E000B40010B103681B68184770473CB1FF1F85
:1007F000034BD3F8B80010B103681B681847704763
:100800003CB1FF1F034BD3F8BC0010B103681B6859
:10081000184770473CB1FF1F034BD3F8C00010B11D
:1008200003681B68184770473CB1FF1F034BD3F8A0
:10083000C40010B103681B68184770473CB1FF1F24
:10084000034BD3F8C80010B103681B681847704702
:100850003CB1FF1F034BD3F8CC0010B103681B68F9
:10086000184770473CB1FF1F034BD3F8D00010B1BD
:1008700003681B68184770473CB1FF1F034BD3F850
:10088000D40010B103681B68184770473CB1FF1FC4
:10089000034BD3F8D80010B103681B6818477047A2
:1008A0003CB1FF1F034BD3F8DC0010B103681B6899
:1008B000184770473CB1FF1F034BD3F8E00010B15D
:1008C00003681B68184770473CB1FF1F034BD3F800
:1008D000E40010B103681B68184770473CB1FF1F64
:1008E000034BD3F8E80010B103681B681847704742
:1008F0003CB1FF1F034BD3F8EC0010B103681B6839
:10090000184770473CB1FF1F704700BF704700BFDA
:10091000D0F888328169027DF0B4D0F884620F6922
:10092000104C00EBC30501339E4298BF00232D6A93
:1009300000EBC3062F80C0F888324D2505FB02432B
:10094000F0691A5C02F01F031F2B09D012064ABF80
:10095000CA68102222F0100243F04003CA600B6004
:10096000F0BC7047B4B80100F8B50646044690F8EC
:100970005870002508E0042B1ED0022B26D001352C
:10098000082D04F1080416D0A0690028F7D0237FB1
:10099000032BF0D147FA05F3DA07F0D496F8583074
:1009A0002B41DB07EBD503681B6898470135082D01
:1009B00004F10804E8D1F8BD96F858307B402B418B
:1009C000DB07DCD503681B689847EFE747FA05F3B8
:1009D000D907D4D596F858302B41DA07CFD403681D
:1009E0001B689847E2E700BF40680368003118BF02
:1009F00001219B68184700BF30B44468057A69B983
:100A0000837A012B0DD094F85920012101FA05F3C6
:100A100022EA030384F8593030BC7047437A012B33
:100A2000F1D194F85920AB401343DBB284F859302C
:100A300030BC7047037A8B420CBF037B437B012B96
:100A400070B44468867A1CD0012594F8592005FAC0
:100A500006F322EA030384F85930427A4468C57ADF
:100A60008A420CBF037B437B012B10D094F85920A2
:100A7000012101FA05F322EA030384F8593070BC1E
:100A8000704794F85920B3401343DBB2E3E794F87E
:100A90005920AB401343DBB284F8593070BC704727
:100AA000037A8B4270B44468C67A24D0837A8B422E
:100AB00021D0837B012B21D0012594F8592005FA00
:100AC00006F322EA030384F85930427A4468057B2E
:100AD0008A4219D0837A8B4216D0837B012B16D0A1
:100AE00094F85920012101FA05F322EA030384F85E
:100AF000593070BC7047437B012BDDD194F85920ED
:100B0000B3401343DBB2DEE7437B012BE8D194F81B
:100B10005920AB401343DBB284F8593070BC7047A6
:100B200010B504468069174A0368DB68934282B0B7
:100B300020D1007913F0E0FC134922690B6801937E
:100B4000019B7AB161689B1A8B4209D3A0B9A16855
:100B50008B424FF0010234BF0023012363752275DD
:100B600002B010BD0028FBD10B680093009B2361ED
:100B700002B010BD9847DFE700232361237563753A
:100B800002B010BD5D0C000080B2FF1F30B483695D
:100B9000164C027F93F858302568016982B01341E2
:100BA000019503F00103019A81B14468521AA242EF
:100BB00009D3A3B981688A424FF0010334BF0022F0
:100BC00001224275037502B030BC7047002BFAD188
:100BD00023680093009B036102B030BC7047002380
:100BE00003610375437502B030BC704780B2FF1FCC
:100BF000C368DA0706D55B1041688268C858825816
:100C0000C81810474168826801EB6300104700BFB5
:100C1000C368DA0706D55B1041688268C8588258F5
:100C2000C81810474168826801EB6300104700BF95
:100C30004368074ADBB211F0FF0F52F833304FF030
:100C4000010214BF83F8802083F80021704700BFA1
:100C500010BD0100C9B2007913F05CBC08B5007981
:100C600013F04AFC08BD00BFD0F8843273B3037D93
:100C7000174970B4D0F88852846900EB830200EB06
:100C8000C500D268C56920684D2606FB03115309CB
:100C90004D5D9B00012103F1604302F01F0201FA48
:100CA00002F203F5614305F01F0140F040001F29E7
:100CB00020601A6009D02B064ABFE368102323F096
:100CC000100341F04001E360216070BC704700BF39
:100CD000B4B801000279034B53F83230012283F893
:100CE0008020704710BD01000279034B53F8323069
:100CF000012283F80021704710BD010038B5437B05
:100D00008568023B012BEA78A97902D90223EB70AE
:100D100038BDD2B2D40629D453062CD4C9B211F0AE
:100D2000500F044612D0AB7943F05003AB71826888
:100D3000937903F0DF03937183680222DA70036909
:100D40000BB1406D98470223A5686373636D3F2B19
:100D500004D85A1C626523442A791A75AB7943F08A
:100D60005003AB71A3680222DA7038BD102352061B
:100D7000EB701BD58568002343658365AB7943F031
:100D80002003AB718368C0229A7083681A79520875
:100D900080F85C209A7942F050029A71836842226E
:100DA000DA70826803239279437338BD826893793D
:100DB00043F05003937183680222DA7038BD00BF9C
:100DC0002DE9F04F00F5884395B093F858210023A2
:100DD0000F930E931093002A40F0918100F5355443
:100DE000103494F820308346A3B900F53556CE4F21
:100DF00030360EAD2368DB68BB4240F0A982207913
:100E000013F07AFBB0FA80F008344009B44205F8D8
:100E1000010BEFD142F29C0042F29E0142F2A0028D
:100E200042F2A2030BF502541C343BF800003BF8DD
:100E300001103BF802203BF8033094F88C4000018D
:100E4000090112011B01ADF83C00ADF83E10ADF8F0
:100E50004020ADF84230002C40F00B82B34B9FEDA8
:100E6000B44A9A785B780793B24B029303F10C0073
:100E7000043B0A920493023A0833D2B203930C3B28
:100E800005930B920BF58B430FAAA0F1180913AD34
:100E90001646D3ED015ADFEDA84A9FEDA86A9FEDF3
:100EA000A85A9FEDA82ADFEDA83ADFEDA82A9FED0A
:100EB000A83AA84BCDF824B0A0F12C01CB46A0F164
:100EC0001C0408950DF1380A00220195B14603F57E
:100ED000DB6696ED007A93F8046793F8077725EEC2
:100EE000877A002E00F03A81B9F80060C7F16307F5
:100EF00006FB07F607EE906AF8EEE76AF7EE007A6F
:100F0000E6EEE47AD3F80067002E27EE877A40F306
:100F10003A81039D4FF0000E85F800E00127029D05
:100F20008BF8007095F800E0BEF1000F04D19AF83C
:100F300000C0BCF1000F05D12778002F40F045819B
:100F40009AF80070022E00F0F981012E00F08781DE
:100F5000BEF1000F40F0D680002F00F0D380022EAB
:100F6000049D0CBF012600260CBFF0EE437AF0EE84
:100F7000637A2E70C1ED007A059DD1ED007A4FF0B5
:100F8000FF3E4FF0010C0026C0F800E084F800C0DE
:100F90002E7027EE867AB5EEC07AF1EE10FA40F2A6
:100FA0002B81B4EEC67AF1EE10FA80F22E81FDEEBE
:100FB000C76A67EE857A16EE908AFDEEE77AF8EE5C
:100FC000E66A17EE906A37EE667A08F101054FF48B
:100FD000B57C0CFB02FCE044AC445E4D05EB4808DC
:100FE00005EB4C0CB8F8605407EE905ABCF860540E
:100FF00001EE905AF8EE677AF8EE611AF6EE006AA2
:1010000071EEE71AE1EE877A77EEA67AFCEEE77AE0
:10101000CDED067ABDF818C011AD4FF0000825F8E7
:1010200012C0019D764585F800801FD04FEA821CD2
:10103000C2EB0C0E4FEA8E0E0EF5835E0EF11C0E07
:10104000444D066015F80EE0BEF1000F0ED0414D84
:10105000CF2EC2EB0C0C05EB8C0CD4BF26EAE67647
:10106000D0266644019D96F8A46F2E70029E019DC5
:1010700006F8017B0296049E01360496039E013613
:101080000396059E013201350136042A03F53573B6
:10109000019500F1040001F104010AF1010A04F1D3
:1010A00001040BF1010B09F1020905967FF40FAF62
:1010B000DDF824B0DDF820A00BF5365411AE38343D
:1010C0000BF536550BF537574FF001084FF0000977
:1010D00055F8043C36F8021B2878194112F036FF07
:1010E000237AA3B1E368643B002BE36040F3B08153
:1010F0001035AF4204F114040AF1010AE8D115B029
:10110000BDE8F08F079D012D7FF436AF27E79AF8F1
:101110000030002BECD054F8043C84F80880E360E5
:101120002046FFF7D7FDE3E75D0C0000BC14FF1F6E
:10113000462FBA358428FF1F9EF214340000504316
:1011400077FF50430000003400000000D9899D3B28
:10115000FEFF7F3FCC14FF1F00FE7F3FB9F8006009
:10116000C7F1630706FB07F607EE906AF8EEE76A39
:10117000F7EE007AE6EE847AD3F80067002E27EEC9
:10118000877A3FF7C6AE029D2E78002E46D19AF898
:101190000060002E00F098802678002E00F01B8161
:1011A0000B9D012D40F217810A9D002D40F0198200
:1011B000059D2E78002E00F01482039DD1ED007A5B
:1011C000D0F800E001272F70E3E6012E00F0C38085
:1011D000022E00F04381032E00F01E81D1ED007A33
:1011E000D0F800E09AF8007027EE867AB5EEC07A63
:1011F000F1EE10FA3FF6D5AE67EE857AFDEEE77AAE
:1012000017EE906AB3F860C406E767EE857AFDEEE4
:10121000E77A17EE906AB3F800C6FDE62678002E4E
:1012200040F0B180039D9AF800702E78002E00F0F7
:10123000AC80002F48D0049DC1ED003A00264FF04D
:10124000FF3EC0F800E02E70059D4FF0010C84F8C1
:1012500000C08BF800602E70039D2E7091E0049DFD
:101260004FF0000C85F800C0BEF1000F7FF44AAFCC
:1012700072E642F2A40042F2A60142F2A80242F251
:10128000AA033BF800403BF801003BF802103BF892
:10129000032040F265639C4294BF002401249842DD
:1012A00094BF00200120994294BF002101219A425D
:1012B00094BF002301238DF838408DF839008DF854
:1012C0003A108DF83B30C9E59BF800604EB1039DA4
:1012D00000268BF8006026702E70079D012D00F00F
:1012E0000B81D3F8FC76059D0126002F2E7065DD5D
:1012F000049D2E78002E61D003F5DC6603F2DC6ECF
:10130000D6ED006A2678DEED001A4FF0000E002EB2
:1013100040F0BF80D1ED007AB7EE007AF4EEC77AE4
:10132000F1EE10FA40F38F80002681ED007AD0F8BC
:1013300000E09AF800702670D0266CE7049D4FF00C
:10134000010C85F800C0BEF1000F7FF4DBAE03E6B0
:101350002046984756E5D1ED007A049D77EE277A2E
:10136000B7EE007AF4EEC77A0026F1EE10FAC1ED7E
:10137000007A2E7067DBD0F800E09AF80070C1EDBB
:10138000003A00263EE79AF80070002F9CD0059D99
:101390002F78002F98D19BF80070002F97D1D3F8A9
:1013A000FC7603F2DC6EDEED001A002F03F5DC6E36
:1013B000DEED006AC8BF4FF0010EA8DC2678D1ED43
:1013C000007A002EA8D077EE277A049D00262E7092
:1013D000C1ED007AA0E70A9D022D09D0D1ED007A77
:1013E000B7EE007AF4EEC77AF1EE10FAC0F2A08000
:1013F000C1ED003A049DD1ED007A00264FF0FF3E8A
:10140000C0F800E02E70059D012727708BF8006062
:101410002E70039D2E70BCE5049DD1ED007A2E78D0
:10142000002E6CD177EE277AB7EE007AF4EEC77A09
:10143000F1EE10FAC1ED007A05DB012681ED003AEC
:10144000F0EE437A2E70D0F800E09AF80070A0E534
:1014500084F808902046FFF747FC49E6D1ED007A72
:10146000049D77EEC77A0126F5EEC07AF1EE10FA08
:101470002E70C1ED007AE6D8D02681ED003A3546CF
:10148000D0F800E09AF800701FEDCD7A4FF0CF0849
:101490009DE5012F00F0AB80022F00F0C480032FE8
:1014A0007FF49CAE049DD1ED007A2E78002E00F0E2
:1014B000028177EEC77AC1ED007ABEF1000F0AD043
:1014C000F4EEE67AF1EE10FA05DB76EEC27A01264A
:1014D000C1ED007A2E70F4EEE71AF1EE10FAB2DDEB
:1014E000049DC1ED001A00262E70F0EE617AD0F84E
:1014F00000E09AF800704CE5C1ED003AF1E677EEB5
:10150000C77AB7EE007AF4EEC77AF1EE10FAC1EDC1
:10151000007A92DAF5EEC07AF1EE10FA93D5002651
:10152000C1ED003AD0F800E02E709AF8007028E77C
:1015300067EE867AF5EEC07AF1EE10FA40F2078196
:10154000F4EEC67AF1EE10FAC0F2C480FDEEE77A4E
:10155000B3F8007617EE908A4546002D3CDDB3F8CF
:1015600062C4B3F86064BC452CBF4FF0000E4FF06E
:10157000010EBE428CBF00260126B64540F0EE802B
:10158000BC4500F0EB80CDF834B003F2624C4FF074
:10159000010E0692CDF83090019DC34612E0BCF8D2
:1015A00000203CF8026FBA428CBF00220122B742F1
:1015B00094BF4FF000084FF0010842455CD1B7429C
:1015C0005AD0CE46DE450EF10109E8D1069ADDF883
:1015D0003090DDF834B00195DFED677AC1ED007A27
:1015E00008E7D1ED007AD0F800E00127D1E4D1ED91
:1015F000007A049D77EE277A0026C1ED007A2E70DE
:10160000BEF1000F3FF41FAFF4EEE67AF1EE10FAF0
:10161000FFF619AFC1ED001AF0EE617AD0F800E0E4
:101620009AF80070B5E4049DD1ED007A2E78A6B347
:1016300077EEC77AF4EEE67AF1EE10FAC1ED007AB1
:10164000C0F28F80BEF1000F70D076EEC27A012614
:10165000F4EEE17AF1EE10FAC1ED007A2E707FF52A
:10166000F2AE76EEC27A0126C1ED007AD0F800E043
:101670002E709AF800708CE4069ADDF83090DDF850
:1016800034B0019507EE90EAB8EEE77AF6EE007A0C
:1016900077EE277A67EEA27AA0E777EE277AF4EE64
:1016A000E67AF1EE10FAC1ED007AFFF6CCAEBEF1AB
:1016B000000FCAD1C7E677EE277AC1ED007ABEF1F6
:1016C000000F3FF4C0AEF4EEE67AF1EE10FABFF68A
:1016D000FCAEB8E6BDEEE71A4FF4B57611EE105A3F
:1016E00006FB0256254D05EB4607B8EEC17AB7F862
:1016F000605406EE905AB7F8625401EE905AF8EE34
:10170000666AF8EE611A77EEC77A71EEE61AB6EEFF
:10171000007AE7EEA16A11EE108A76EE877AFCEE87
:10172000E77ACDED067ABDF8187015E7F4EEE17AA8
:10173000F1EE10FA7FF587AE0026C1ED001A2E708B
:10174000F0EE617AD0F800E09AF8007021E4FDEE46
:10175000E77AB3F8607417EE908AFDE64FF0000E5A
:1017600090E7F4EEE17AF1EE10FA7FF56CAEBEF19F
:10177000000FE1D075E700BF00000000CC14FF1F90
:10178000F0B4E4298AB004462ED04E1EF7B20425E8
:101790002220012F8DF803108DF824308DF80420BD
:1017A0008DF800508DF8010004D9A1F11600012830
:1017B00000F26B8194F88150002084F8110184F8C4
:1017C0001001002D47D1162940F03D8194F8821078
:1017D00000294FD10525012F40F26481012284F8B0
:1017E000822084F881200FE090F881008DF80310AA
:1017F000182522218DF824308DF804208DF8005012
:101800008DF8011078BB1925D4F8A02094F8910028
:10181000D1788DF80200890664D5002000239370EA
:1018200000BFD4F8A01080228A70D4F8A0108B706A
:1018300000BFD4F8A0108A70D4F8A0201370D4F898
:10184000A0209378022143F04003937084F8A51000
:101850000AB0F0BC704794F8820058B916294FF0CE
:101860000505D1D1B7E794F882100029CBD019250E
:10187000E32603E0012F40F2DE800525162EC3D8B3
:1018800001A151F826F000BF311A00002B1A000008
:1018900009180000091800000918000009180000C4
:1018A00009180000091800000918000009180000B4
:1018B00009180000091800000918000009180000A4
:1018C0000918000009180000091800000918000094
:1018D000091800000918000009180000DD170000B1
:1018E000231A0000917801F0BF019170D4F8A01084
:1018F000012284F8A52042F21070CA7892060ED513
:101900000138FAD1887000BFD4F8A03080229A70D4
:1019100000BF012384F8A430D4F8A0207DE7B022D2
:101920008A70D4F8A02042F21071D078870603D4D0
:101930000139FAD19170E6E7D17889067FF56DAF6C
:10194000917841F030019170D4F8A00042F210710A
:10195000C27896060ED40139FAD1817000BFD4F84E
:10196000A03080229A7000BF012384F8A430D4F8FC
:10197000A02052E75B00DBB20371D4F8A02042F252
:101980001073D178880703D4013BFAD19370E5E74F
:1019900042F21073D178090603D4013BFAD1937057
:1019A000B1E70220D070D4F8A020937843F0100360
:1019B00093700DEB05076E46BE42D4F8A03044D0BC
:1019C00016F8012B1A71D4F8A03042F21071DA78AF
:1019D000920703D40139FAD1997094E7DA78D87074
:1019E000D3B203F0100202F0FF010225002A5FD1FA
:1019F000DB07E1D5D4F8A0300122DA7000BFD4F8BB
:101A0000A03084F8A450997000BFD4F8A030802290
:101A10009A70D4F8A0300222DA70D4F8A020002006
:101A2000FCE6002284F88220EEE6C4F88820EBE68B
:101A3000C4F88420E8E694F8801091424FF0050540
:101A40003FF61CAFE0E60525DEE60222DA70D4F8A8
:101A5000A020937803F0C7039370D4F8A02042F23B
:101A60001071D37898060ED50139FAD1917000BF64
:101A7000D4F8A03080229A7000BF012084F8A4001E
:101A8000D4F8A020CAE60120C8E694F88100002816
:101A9000D9D094F8820000287FF4EFAE1629D2D175
:101AA00005259BE694F8801091427FF6ADAE95E651
:101AB000D4F8A0301022DA7000BFD4F8A03003218F
:101AC000002284F8A4109A7000BFD4F8A0308022BD
:101AD0009A709EE7214B10B4D3F8C8201368506861
:101AE00019780478507A137A044201EA03011BD072
:101AF000937A03F0030309B143F0040343F00803AE
:101B00009910013B91720D2B0BD8DFE803F02107F0
:101B10001B070A152121150A071B0721D368013B62
:101B2000D3605DF8044B7047937A03F003030029F8
:101B3000E6D043F00403E3E7D3685DF8044B023BCF
:101B4000D3607047D3685DF8044B0233D3607047AD
:101B5000D3685DF8044B0133D360704734B0FF1F86
:101B6000214B10B45A681368506819780478507A79
:101B7000137A044201EA03011BD0937A03F00303B2
:101B800009B143F0040343F008039910013B91723B
:101B90000D2B0BD8DFE803F021071B070A152121C5
:101BA000150A071B0721D368013BD3605DF8044B7E
:101BB0007047937A03F003030029E6D043F004034F
:101BC000E3E7D3685DF8044B023BD3607047D3680A
:101BD0005DF8044B0233D3607047D3685DF8044B63
:101BE0000133D360704700BF34B0FF1F214B10B4E6
:101BF0009A681368506819780478507A137A044206
:101C000001EA03011BD0937A03F0030309B143F007
:101C1000040343F008039910013B91720D2B0BD87C
:101C2000DFE803F021071B070A152121150A071B0E
:101C30000721D368013BD3605DF8044B7047937A6A
:101C400003F003030029E6D043F00403E3E7D3687D
:101C50005DF8044B023BD3607047D3685DF8044BDA
:101C60000233D3607047D3685DF8044B0133D3600F
:101C7000704700BF34B0FF1F214B10B4DA681368FF
:101C8000506819780478507A137A044201EA030103
:101C90001BD0937A03F0030309B143F0040343F02C
:101CA00008039910013B91720D2B0BD8DFE803F06C
:101CB00021071B070A152121150A071B0721D368D5
:101CC000013BD3605DF8044B7047937A03F0030344
:101CD0000029E6D043F00403E3E7D3685DF8044B42
:101CE000023BD3607047D3685DF8044B0233D36086
:101CF0007047D3685DF8044B0133D360704700BF71
:101D000034B0FF1F214B10B41A691368506819785A
:101D10000478507A137A044201EA03011BD0937AC3
:101D200003F0030309B143F0040343F008039910DF
:101D3000013B91720D2B0BD8DFE803F021071B0745
:101D40000A152121150A071B0721D368013BD3601F
:101D50005DF8044B7047937A03F003030029E6D043
:101D600043F00403E3E7D3685DF8044B023BD36020
:101D70007047D3685DF8044B0233D3607047D36873
:101D80005DF8044B0133D360704700BF34B0FF1FD0
:101D9000214B10B45A691368506819780478507A46
:101DA000137A044201EA03011BD0937A03F0030380
:101DB00009B143F0040343F008039910013B917209
:101DC0000D2B0BD8DFE803F021071B070A15212193
:101DD000150A071B0721D368013BD3605DF8044B4C
:101DE0007047937A03F003030029E6D043F004031D
:101DF000E3E7D3685DF8044B023BD3607047D368D8
:101E00005DF8044B0233D3607047D3685DF8044B30
:101E10000133D360704700BF34B0FF1F214B10B4B3
:101E20009A691368506819780478507A137A0442D2
:101E300001EA03011BD0937A03F0030309B143F0D5
:101E4000040343F008039910013B91720D2B0BD84A
:101E5000DFE803F021071B070A152121150A071BDC
:101E60000721D368013BD3605DF8044B7047937A38
:101E700003F003030029E6D043F00403E3E7D3684B
:101E80005DF8044B023BD3607047D3685DF8044BA8
:101E90000233D3607047D3685DF8044B0133D360DD
:101EA000704700BF34B0FF1F214B10B4DA691368CC
:101EB000506819780478507A137A044201EA0301D1
:101EC0001BD0937A03F0030309B143F0040343F0FA
:101ED00008039910013B91720D2B0BD8DFE803F03A
:101EE00021071B070A152121150A071B0721D368A3
:101EF000013BD3605DF8044B7047937A03F0030312
:101F00000029E6D043F00403E3E7D3685DF8044B0F
:101F1000023BD3607047D3685DF8044B0233D36053
:101F20007047D3685DF8044B0133D360704700BF3E
:101F300034B0FF1F214B10B41A6A13685068197827
:101F40000478507A137A044201EA03011BD0937A91
:101F500003F0030309B143F0040343F008039910AD
:101F6000013B91720D2B0BD8DFE803F021071B0713
:101F70000A152121150A071B0721D368013BD360ED
:101F80005DF8044B7047937A03F003030029E6D011
:101F900043F00403E3E7D3685DF8044B023BD360EE
:101FA0007047D3685DF8044B0233D3607047D36841
:101FB0005DF8044B0133D360704700BF34B0FF1F9E
:101FC000214B10B45A6A1368506819780478507A13
:101FD000137A044201EA03011BD0937A03F003034E
:101FE00009B143F0040343F008039910013B9172D7
:101FF0000D2B0BD8DFE803F021071B070A15212161
:10200000150A071B0721D368013BD3605DF8044B19
:102010007047937A03F003030029E6D043F00403EA
:10202000E3E7D3685DF8044B023BD3607047D368A5
:102030005DF8044B0233D3607047D3685DF8044BFE
:102040000133D360704700BF34B0FF1F214B10B481
:102050009A6A1368506819780478507A137A04429F
:1020600001EA03011BD0937A03F0030309B143F0A3
:10207000040343F008039910013B91720D2B0BD818
:10208000DFE803F021071B070A152121150A071BAA
:102090000721D368013BD3605DF8044B7047937A06
:1020A00003F003030029E6D043F00403E3E7D36819
:1020B0005DF8044B023BD3607047D3685DF8044B76
:1020C0000233D3607047D3685DF8044B0133D360AB
:1020D000704700BF34B0FF1F214B10B4DA6A136899
:1020E000506819780478507A137A044201EA03019F
:1020F0001BD0937A03F0030309B143F0040343F0C8
:1021000008039910013B91720D2B0BD8DFE803F007
:1021100021071B070A152121150A071B0721D36870
:10212000013BD3605DF8044B7047937A03F00303DF
:102130000029E6D043F00403E3E7D3685DF8044BDD
:10214000023BD3607047D3685DF8044B0233D36021
:102150007047D3685DF8044B0133D360704700BF0C
:1021600034B0FF1F214B10B41A6B136850681978F4
:102170000478507A137A044201EA03011BD0937A5F
:1021800003F0030309B143F0040343F0080399107B
:10219000013B91720D2B0BD8DFE803F021071B07E1
:1021A0000A152121150A071B0721D368013BD360BB
:1021B0005DF8044B7047937A03F003030029E6D0DF
:1021C00043F00403E3E7D3685DF8044B023BD360BC
:1021D0007047D3685DF8044B0233D3607047D3680F
:1021E0005DF8044B0133D360704700BF34B0FF1F6C
:1021F000214B10B45A6B1368506819780478507AE0
:10220000137A044201EA03011BD0937A03F003031B
:1022100009B143F0040343F008039910013B9172A4
:102220000D2B0BD8DFE803F021071B070A1521212E
:10223000150A071B0721D368013BD3605DF8044BE7
:102240007047937A03F003030029E6D043F00403B8
:10225000E3E7D3685DF8044B023BD3607047D36873
:102260005DF8044B0233D3607047D3685DF8044BCC
:102270000133D360704700BF34B0FF1F214B10B44F
:102280009A6B1368506819780478507A137A04426C
:1022900001EA03011BD0937A03F0030309B143F071
:1022A000040343F008039910013B91720D2B0BD8E6
:1022B000DFE803F021071B070A152121150A071B78
:1022C0000721D368013BD3605DF8044B7047937AD4
:1022D00003F003030029E6D043F00403E3E7D368E7
:1022E0005DF8044B023BD3607047D3685DF8044B44
:1022F0000233D3607047D3685DF8044B0133D36079
:10230000704700BF34B0FF1F214B10B4DA6B136865
:10231000506819780478507A137A044201EA03016C
:102320001BD0937A03F0030309B143F0040343F095
:1023300008039910013B91720D2B0BD8DFE803F0D5
:1023400021071B070A152121150A071B0721D3683E
:10235000013BD3605DF8044B7047937A03F00303AD
:102360000029E6D043F00403E3E7D3685DF8044BAB
:10237000023BD3607047D3685DF8044B0233D360EF
:102380007047D3685DF8044B0133D360704700BFDA
:1023900034B0FF1F214B10B41A6C136850681978C1
:1023A0000478507A137A044201EA03011BD0937A2D
:1023B00003F0030309B143F0040343F00803991049
:1023C000013B91720D2B0BD8DFE803F021071B07AF
:1023D0000A152121150A071B0721D368013BD36089
:1023E0005DF8044B7047937A03F003030029E6D0AD
:1023F00043F00403E3E7D3685DF8044B023BD3608A
:102400007047D3685DF8044B0233D3607047D368DC
:102410005DF8044B0133D360704700BF34B0FF1F39
:10242000214B10B45A6C1368506819780478507AAC
:10243000137A044201EA03011BD0937A03F00303E9
:1024400009B143F0040343F008039910013B917272
:102450000D2B0BD8DFE803F021071B070A152121FC
:10246000150A071B0721D368013BD3605DF8044BB5
:102470007047937A03F003030029E6D043F0040386
:10248000E3E7D3685DF8044B023BD3607047D36841
:102490005DF8044B0233D3607047D3685DF8044B9A
:1024A0000133D360704700BF34B0FF1F214B10B41D
:1024B0009A6C1368506819780478507A137A044239
:1024C00001EA03011BD0937A03F0030309B143F03F
:1024D000040343F008039910013B91720D2B0BD8B4
:1024E000DFE803F021071B070A152121150A071B46
:1024F0000721D368013BD3605DF8044B7047937AA2
:1025000003F003030029E6D043F00403E3E7D368B4
:102510005DF8044B023BD3607047D3685DF8044B11
:102520000233D3607047D3685DF8044B0133D36046
:10253000704700BF34B0FF1F214B10B4DA6C136832
:10254000506819780478507A137A044201EA03013A
:102550001BD0937A03F0030309B143F0040343F063
:1025600008039910013B91720D2B0BD8DFE803F0A3
:1025700021071B070A152121150A071B0721D3680C
:10258000013BD3605DF8044B7047937A03F003037B
:102590000029E6D043F00403E3E7D3685DF8044B79
:1025A000023BD3607047D3685DF8044B0233D360BD
:1025B0007047D3685DF8044B0133D360704700BFA8
:1025C00034B0FF1F214B10B41A6D1368506819788E
:1025D0000478507A137A044201EA03011BD0937AFB
:1025E00003F0030309B143F0040343F00803991017
:1025F000013B91720D2B0BD8DFE803F021071B077D
:102600000A152121150A071B0721D368013BD36056
:102610005DF8044B7047937A03F003030029E6D07A
:1026200043F00403E3E7D3685DF8044B023BD36057
:102630007047D3685DF8044B0233D3607047D368AA
:102640005DF8044B0133D360704700BF34B0FF1F07
:10265000214B10B45A6D1368506819780478507A79
:10266000137A044201EA03011BD0937A03F00303B7
:1026700009B143F0040343F008039910013B917240
:102680000D2B0BD8DFE803F021071B070A152121CA
:10269000150A071B0721D368013BD3605DF8044B83
:1026A0007047937A03F003030029E6D043F0040354
:1026B000E3E7D3685DF8044B023BD3607047D3680F
:1026C0005DF8044B0233D3607047D3685DF8044B68
:1026D0000133D360704700BF34B0FF1F214B10B4EB
:1026E0009A6D1368506819780478507A137A044206
:1026F00001EA03011BD0937A03F0030309B143F00D
:10270000040343F008039910013B91720D2B0BD881
:10271000DFE803F021071B070A152121150A071B13
:102720000721D368013BD3605DF8044B7047937A6F
:1027300003F003030029E6D043F00403E3E7D36882
:102740005DF8044B023BD3607047D3685DF8044BDF
:102750000233D3607047D3685DF8044B0133D36014
:10276000704700BF34B0FF1F816842F21073CA780F
:1027700092060BD5013BFAD18B7000BF8268802195
:10278000917000BF0122027318467047B0238B700E
:10279000826842F21073D178890603D4013BFAD1E2
:1027A0009370EAE7D378C3F340131846704700BF2D
:1027B00001380B463A2800F25C82DFE810F0530241
:1027C0004C0245023E0237023002290222021B025D
:1027D000AE01A701A001990192018B0184017D0145
:1027E00076016F01680161015A0153014C014501F5
:1027F0003E0137013001290122011B0113010B01A8
:102800000301FB00F300EB00E300DB00D300CB008F
:10281000C300BB00B300AB00A3009B0093008B0080
:1028200083007B0073006B0063005B0053004B0070
:1028300043003B00BC48BD49C0F8EC201A463B2091
:1028400011F0DAB9B848BA49C0F8E8201A463A2077
:1028500011F0D2B9B448B749C0F8E4201A4639207B
:1028600011F0CAB9B048B449C0F8E0201A4638207F
:1028700011F0C2B9AC48B149C0F8DC201A46372083
:1028800011F0BAB9A848AE49C0F8D8201A46362087
:1028900011F0B2B9A448AB49C0F8D4201A4635208B
:1028A00011F0AAB9A048A849C0F8D0201A4634208F
:1028B00011F0A2B99C48A549C0F8CC201A46332093
:1028C00011F09AB99848A249C0F8C8201A46322097
:1028D00011F092B994489F49C0F8C4201A4631209B
:1028E00011F08AB990489C49C0F8C0201A4630209F
:1028F00011F082B98C489949C0F8BC201A462F20A3
:1029000011F07AB988489649C0F8B8201A462E20A6
:1029100011F072B984489349C0F8B4201A462D20AA
:1029200011F06AB980489049C0F8B0201A462C20AE
:1029300011F062B97C488D49C0F8AC201A462B20B2
:1029400011F05AB978488A49C0F8A8201A462A20B6
:1029500011F052B974488749C0F8A4201A462920BA
:1029600011F04AB970488449C0F8A0201A462820BE
:1029700011F042B96C488149C0F89C201A462720C2
:1029800011F03AB968487E49C0F898201A462620C6
:1029900011F032B964487B49C0F894201A462520CA
:1029A00011F02AB960487849C0F890201A462420CE
:1029B00011F022B95C487549C0F88C201A462320D2
:1029C00011F01AB958487249C0F888201A462220D6
:1029D00011F012B954486F49C0F884201A462120DA
:1029E00011F00AB950486C49C0F880201A462020DE
:1029F00011F002B94C486949C2671A461F2011F00C
:102A0000FBB84948664982671A461E2011F0F4B89F
:102A10004548644942671A461D2011F0EDB8424806
:102A2000614902671A461C2011F0E6B83E485F492A
:102A3000C2661A461B2011F0DFB83B485C4982662B
:102A40001A461A2011F0D8B837485A4942661A4631
:102A5000192011F0D1B83448574902661A46182097
:102A600011F0CAB830485549C2651A46172011F00E
:102A7000C3B82D48524982651A46162011F0BCB8D9
:102A80002948504942651A46152011F0B5B8264824
:102A90004D4902651A46142011F0AEB822484B4940
:102AA000C2641A46132011F0A7B81F48484982642F
:102AB0001A46122011F0A0B81B48464942641A4633
:102AC000112011F099B81848434902641A461020A1
:102AD00011F092B814484149C2631A460F2011F010
:102AE0008BB811483E4982631A460E2011F084B813
:102AF0000D483C4942631A460D2011F07DB80A4842
:102B0000394902631A460C2011F076B80648374955
:102B1000C2621A460B2011F06FB803483449826232
:102B20001A460A2011F068B83CB1FF1FF5080000F2
:102B3000E1080000CD080000B9080000A508000069
:102B4000910800007D080000690800005508000099
:102B5000410800002D0800001908000005080000C9
:102B6000F1070000DD070000C9070000B5070000FD
:102B7000A10700008D07000079070000650700002D
:102B8000510700003D07000029070000150700005D
:102B900001070000ED060000D9060000C506000090
:102BA000B10600009D0600008906000075060000C1
:102BB000610600004D0600003906000025060000F1
:102BC00011060000FD050000E9050000D505000024
:102BD000C1050000AD050000990500008505000055
:102BE000710500005D050000490500003505000085
:102BF000210500001F48204942621A46092010F0B2
:102C0000FBBF1C481D4902621A46082010F0F4BFA1
:102C100018481B49C2611A46072010F0EDBF15483D
:102C2000184982611A46062010F0E6BF114816497D
:102C300042611A46052010F0DFBF0E4813490261B9
:102C40001A46042010F0D8BF0A481149C2601A463B
:102C5000032010F0D1BF07480E4982601A460220B7
:102C600010F0CABF03480C4942601A46012010F018
:102C7000C3BF70473CB1FF1F0D050000F904000001
:102C8000E5040000D1040000BD040000A904000018
:102C900095040000810400006D04000008B513468F
:102CA00040680A461946FFF783FD08BDF0B5002AC3
:102CB0009DF8144029DB002B27DBFF2825DC3F296A
:102CC00023DCFF2AA8BFFF2220EAE0703F2BA8BF29
:102CD0003F23824221EAE1761D4616DB591C891BFF
:102CE000DFF828C0571C09024FEA062EB54208DB60
:102CF00000EB0E0262440023D45403F580738B4230
:102D0000FAD10130B842F1D1F0BDF0BD3070FF1FF3
:102D1000F0B5002A9DF8145028DB002B26DBFF2895
:102D200024DC3F2922DCFF2AA8BFFF2220EAE0762C
:102D30003F2BA8BF3F23B24221EAE17716DBDC1B21
:102D400064080134DFF828C064024FEA072EBB4252
:102D500008DB06EB0E0060440021455401F50071CC
:102D60008C42FAD10236B242F1DAF0BDF0BD00BFBA
:102D70003070FF1FF6EE007A30EE270A30B4BDEE59
:102D8000C07A70EEA70A17EE104AFF2C31EE271A10
:102D900071EEA71ABDEEE06A03D816EE103A3F2B8B
:102DA0006BD9FDEEC17A17EE902AFDEEE17AFF2A8B
:102DB00017EE901A01D83F295AD931EE407A71EEB8
:102DC000E07AF0EEC76AF0EEE75AF4EEE56AF1EE6B
:102DD00010FA23DB9FED316AF4EEC66AF1EE10FAC9
:102DE0001AD4B4EEC10AF1EE10FA4DDC23469A4231
:102DF000C7EE876A10DD2A4CFF2B08D8FDEEE07A7B
:102E000017EE901A3F2904EB012198BFC8540133F3
:102E1000934270EEA60AEFD130BC7047F4EEE10A9F
:102E2000F1EE10FA1ADC16EE103AF0EE476A8B4219
:102E300086EEA77AF0DA1A4DFDEEC07A30EE070A78
:102E400017EE902AFF2A04D805EB03243F2B98BFE6
:102E5000A05401338B42EFD130BC704770EE416A11
:102E60000B4670EEE17AB0EE410A16EE101ADEE77C
:102E70000B4B03EB012398549FE7094B16EE102AE6
:102E800003EB022318558CE770EEE17A134630EE1F
:102E9000417A2246F0EE610AA9E700BFACC52737A8
:102EA0003070FF1F2DE9F04F854B9BB0DD6A1B682A
:102EB0001193834B002D5C68064640F38181032DFE
:102EC00056DC304613F0DCF93278002A59D000285D
:102ED0004FF0000EACBF07466FF00047F446711E7E
:102EE000012011F8013F33B99FB911F8013F4FF0AC
:102EF000FF37002BF8D00A2B04D01F2BF1D90EF18D
:102F0000060EEEE7F445B8BFF44601304FF0000E70
:102F1000E7E76B4BF445996A6346B8BF734605FB18
:102F200003F308311793664B00FB01F005FB00F734
:102F3000D86801282CD0022800F04581604B1B691D
:102F4000012B30D0022B08BFE41B5D4B1199D3F845
:102F500018E01B6ADFF868C103EB0E0841450B4619
:102F600003DA17990B449E4522DB1BB0BDE8F08FB6
:102F7000534B03253046DD6213F082F93278002A84
:102F8000A5D14F4B1792D86801284FEAC507D2D177
:102F9000179B119903EBD373A1EB63031193484B78
:102FA0001B69012BCED107EBD773A4EB6304CCE7ED
:102FB000DCF81CE0DCF8243073449C42D5DA27446A
:102FC000BE45D2DA002AD0D00996CDF864C00A2ACC
:102FD000099B00F0E0851E460021134602E00A2B03
:102FE00000F0A0831F2B16F8013F88BF0131002B92
:102FF000F5D101EB41014FEA410E189605FB0EFE9B
:103000002F4B9B6A083305FB03FC0128ACEBC5067C
:1030100000F09383022800F0B685119B0693284B9D
:103020001B7D002B40F0D4800CEB04030E93022D8B
:1030300006EB0403109300F08A83032D40F0FD801B
:10304000002A00F0AC810A2A00F0A9811C4B1C4820
:10305000109CD3F81890196AD3F81CB05B6A007AF8
:1030600002905B4420020393831C0A93A31C0B93DE
:10307000631C1493A2F12003DBB26B2B09EB010A52
:1030800000F226830F4A52F823301E780A9A0699D6
:10309000059310460C4BDDF82CE0DDF850C0109F76
:1030A00000EB01089844002304934B1C07938B1CEE
:1030B000089318460A4607994446002335E000BFA6
:1030C000782AFF1FDCAD01003070FF1F814500F33F
:1030D0007181824540F36E81894540F34582BB454D
:1030E00005DC039DBD42C4BF9DF808502570E34533
:1030F00006DC039D654503DD9DF8085084F800510A
:10310000F34506DC039D754503DD9DF8085084F802
:1031100000520133062B02F1030204F1030401F112
:10312000030100F1030000F0658146FA03F5ED07A5
:10313000EFD59145CADC824500F37181814540F3AA
:103140009481894500F37081924540F30382BB4529
:1031500000F38782039DBD4240F383829DF80850AF
:1031600004F8025C8A4506DD9DF8085004F8015C0D
:10317000924540F3E181E34500F3DE81039D65451F
:1031800040F3DA819DF8085084F8FE508A4540F3F8
:10319000AD829DF8085084F8FF50924540F322819B
:1031A000F345B6DC039D7545B3DD9DF8085084F802
:1031B000FE518A45ADDD9DF8085084F8FF51A8E71F
:1031C0000125DD627DE6119B17995B1A1193B5E627
:1031D00019998869D1F81C800B6A4F6A4A7D069953
:1031E00000920CEB04020E920A46724400EB030EAE
:1031F000013A0EF1FF3E724508EB07030E9FA8BF90
:103200007246884203F1FF33B8BF0846013FA0452C
:103210004146B8BF2146BB42A8BF3B46FFF746FD2B
:1032200033191093099B022D1A7800F09082032D18
:103230003FF406AF002A00F0B2800A2A00F0AF8007
:10324000B94BB94899691E6AD3F81CB05B6A007A19
:10325000069D07905B440593109B180205350E44AC
:10326000069003F10807A2F12003DBB26B2B96BF97
:10327000AE4AAF4C52F82340069B109A039558195A
:10328000AC4B013C05F1FF3E1844A5F1050AA5F140
:103290000409A5F10308A5F1020CCDF810E0029491
:1032A000029C14F8013F0294DC070FD551450DDC58
:1032B00056450BDD934509DC059C944206DD039CD5
:1032C000041BA6469DF81C400EF80A409D070FD52A
:1032D00049450DDC4E450BDD934509DC059C9442C8
:1032E00006DD039C041BA6469DF81C400EF8094011
:1032F0005C070FD541450DDC46450BDD934509DCE8
:10330000059C944206DD039C041BA6469DF81C40C8
:103310000EF808401D070FD58C450DDBB4450BDAC0
:10332000934509DC059C944206DD039C041BA646DC
:103330009DF81C400EF80C40DC0611D5049DA942F6
:103340002C460DDCAE420BDD934509DC059C944216
:1033500006DD039C041BA6469DF81C400EF80540A4
:103360009B060CD5039B994209DC9E4207DD9345E1
:1033700005DC059B9342C4BF9DF81C3003700132ED
:10338000974200F580708BD1099B039D13F8012FA4
:10339000099322B10A2A05F106057FF464AF189B50
:1033A0000E9C1A78002A3FF4E0AD09935E4BDD6A6B
:1033B000D8680CE689453FF7ACAE8A457FF7A9AEE1
:1033C000BB4506DC039DBD4203DD9DF8085004F8B3
:1033D000015CE34506DC039D654503DD9DF808506F
:1033E00084F8FF50F3453FF794AE039D75453FF7D2
:1033F000E2AE8EE6049B0333182B049308F5407865
:103400000EF1030E07F103070CF1030C00F04D81E0
:10341000059B089813F8016F0593069A4BE68145C2
:1034200051DD4945BFF690AE92457FF772AEBB4580
:1034300006DC039DBD4203DD9DF8085004F8025CE4
:10344000E34506DC039D654503DD9DF8085084F8DF
:10345000FE50F3453FF75DAE039D75457FF759AECE
:103460009DF8085084F8FE5153E68945DCDC92450E
:1034700040F34381BB4500F34B81039DBD4240F3C4
:1034800047819DF8085004F8025C8A4506DD9DF8E6
:10349000085004F8015C924540F31D81E34500F3B8
:1034A0001A81039D654540F316819DF8085084F804
:1034B000FE508A4540F32F819DF8085084F8FF5054
:1034C00092458FDD6CE68A457ADC924540F3D980DF
:1034D000BB450CDC039DBD4209DD9DF8085004F896
:1034E000025C9DF808502570924540F3D080E3457A
:1034F0000DDC039D65450ADD9DF8085084F8FE50FB
:103500009DF8085084F8005192457FF7F9ADF345D6
:103510003FF7FFAD039D75457FF7FBAD9DF8085064
:1035200084F8FE51F1E500BF782AFF1FDCAD0100F1
:1035300004B401003070FF1F8A4507DDE3453FF703
:103540002CAE039D65457FF728AE22E692457FF7B6
:10355000E0AD25E68A45F9DDBB453FF709AE039DA1
:10356000BD427FF705AEFFE58A457EDDBB450BDC3E
:10357000039DBD4208DD9DF8085004F8015C9DF8EC
:10358000085025708A4575DDE3450DDC039D6545D2
:103590000ADD9DF8085084F8FF509DF8085084F823
:1035A00000518A457FF7ACADF3453FF7B2AD039DBF
:1035B00075457FF7AEAD9DF8085084F8FF51A4E53E
:1035C000924542DDBB4540DC039DBD423DDD9DF89B
:1035D000085004F8025C89453EDD039DBD4202DDD2
:1035E0009DF80850257092451FDDE3451DDC039DC5
:1035F00065451ADD9DF8085084F8FE5089451BDDAD
:10360000039D654503DD9DF8085084F800519245FF
:1036100017DDF34515DC039D754512DD9DF8085057
:1036200084F8FE518945C6DD6CE5894537DCE34504
:10363000EDDC039D6545EADD9DF8085084F8FF50F8
:10364000E1E789453FF75CADAEE789452ADCBB453C
:10365000C9DC039DBD42C6DD9DF8085004F8015C3D
:10366000BEE78A453FF778AF85E5BB4502DC039DA1
:10367000BD4284DCE3453FF743AD039D65458CDCEB
:103680003EE5BB4503DC039DBD423FF72AAFE34562
:103690003FF736AD039D65453FF732AF30E5E34573
:1036A000B5DCADE7BB459EDC97E7099B13F8012F1E
:1036B0000993069B12330693002A3FF470AE0A2A40
:1036C0003FF46DAEA2F12003DBB26B2B7FF6DAACD8
:1036D0009C4B0026DAE48A457FF738AFE3453FF795
:1036E000EFAE039D65457FF7EBAEE5E692453FF70C
:1036F00057AD8A453FF776AE0BE58A457FF726AF93
:10370000BB453FF7C8AE039DBD427FF7C4AEBEE6E2
:103710008A45F5DCC2E692453FF742AD8A457FF720
:10372000F8AC5FE601EB41014FEA410E189605FB4C
:103730000EFE33460133189362E4179B1199CEEBCA
:10374000030303EBD37301EB6303069367E4002ADF
:103750003FF425AE0A2A3FF422AE7B4B7A48196A21
:103760009C69DE695B6A90F8089006EB0308069B8B
:1037700004EB010B591C039119460B330F930B46B5
:103780000A330D930B4609330C930B46083304930D
:103790000B4607310B91991D0A91591D0691191D70
:1037A0000891D91C0791991C0591C2461099C846E9
:1037B0009946A2F12003DBB201316B2B149100F288
:1037C0004481624A52F823502978109A149B02953A
:1037D00000208CE0CD0711D5039DA542C0F2A18148
:1037E000A14580F2E5815D4508DAB34206DB534529
:1037F00004DA574F07EB032707F805808D0713D529
:10380000079DAC42059D00F37781AC4240F3CA812D
:10381000079DAB4508DD9E4206DC9A4504DD4C4F12
:1038200007EB032707F805804F0713D5069DAC4229
:10383000089D00F30D81AC4240F3BD81069DAB4570
:1038400008DD9E4206DC9A4504DD414F07EB032765
:1038500007F805800D0713D50B9DA5420A9DC0F200
:103860000C81AC4240F3AB810B9D5D4508DA9E4272
:1038700006DC9A4504DD364F07EB032707F8058081
:10388000CF0613D50C9DAC42049D00F30B81AC42D6
:1038900040F399810C9DAB4508DD9E4206DC9A45BC
:1038A00004DD2B4F07EB032707F805808D0613D5A2
:1038B0000F99A1420D99C0F20A818C4240F36F81A9
:1038C0000F9D5D4508DA9E4206DC9A4504DD2049DD
:1038D00001EB032101F805800130082802F1020202
:1038E00003F102037DD0029D15F8011F0295964257
:1038F0003FF770AF924513DCCF077FF57FAF039D95
:10390000A542C0F22C81A14580F24F815D45BFF6F2
:1039100075AF9E423FF772AF9A457FF76FAF68E78A
:103920000B4F0B4DDDF80CC0CDF8549007EB022780
:1039300005EB032512971395CE460027029D16929C
:1039400022E000BF04B40100782AFF1FDCAD0100B3
:103950003070FF1FDE4502DA129A02F80E806445CD
:103960001BDDDE4509DA9E4204DC9A45C4BF139A8A
:1039700002F80E80644540F3EE800137062F0CF10B
:10398000020C0EF1020E21D041FA07F919F0010FD5
:10399000F3D0A645DEDA6445EFDCE34540F3D5809D
:1039A000129AA64502F80C8080F2D2809E42E4DC96
:1039B0009A45C8BF139A07F10107C8BF02F80C80E7
:1039C000062F0CF1020C0EF1020EDDD1169ADDF875
:1039D000549002950130082802F1020203F102031B
:1039E00081D1099B13F8012F099309F10C09002AD1
:1039F0003FF4D5AC039B0C3303930F9B0C330F9315
:103A00000D9B0C330D930C9B0C330C93049B0C33CC
:103A100004930B9B0C330B930A9B0C330A93069B6A
:103A20000C330693089B0C330893079B0C330793C6
:103A3000059B0A2A03F10C0305933FF4B0ACA2F1F5
:103A40002003DBB26B2B7FF6BCAE614D0021BCE6E0
:103A5000AC423FF7FFAEAB457FF7FCAE9E4207DCC2
:103A60009A4505DD5B4D05EB0327089D07F80580AA
:103A7000069DAC423FF7EEAEE0E6AC423FF700AF4A
:103A8000AB457FF7FDAE9E4207DC9A4505DD514D03
:103A900005EB03270A9D07F805800B9DA542FFF65D
:103AA000EFAEE1E6AC423FF701AFAB457FF7FEAECC
:103AB0009E4207DC9A4505DD464D05EB0327049D34
:103AC00007F805800C9DAC423FF7F0AEE2E68C4271
:103AD0003FF702AF8B457FF7FFAE9E4207DC9A456A
:103AE00005DD3C490D9D01EB032101F805800F998F
:103AF000A142FFF6F1AEE3E6AC423FF795AEAB452F
:103B00007FF792AE9E4207DC9A4505DD314D05EB0D
:103B10000327059D07F80580079DAC423FF784AE5B
:103B200076E6A145FFF66AAED945BFF667AE9E427E
:103B300006DC9A4504DD274D05EB032707F80980CD
:103B4000039DA542FFF65AAE4DE6A645FFF615AF1A
:103B5000DE45FFF608AFE3453FF728AF0DE7A14587
:103B6000FFF64CAED945BFF649AE9E4206DC9A45FB
:103B700004DD184D05EB032707F80980039DA542D6
:103B8000FFF63CAEC2E6179B1199CEEB03030B4444
:103B90000693FFF744BA18934FF0000ECAE58B4521
:103BA0009BDC8DE6AB45ADDC32E6D945DDDBADE631
:103BB000D945BCDB17E6AB453FF750AF3EE6AB451A
:103BC0003FF761AF50E6AB453FF772AF62E600BF2B
:103BD00004B401003070FF1FF0B5DFED3C7AB4EEA5
:103BE000E70AF1EE10FA83B0054639D5B5EEC00A02
:103BF000F1EE10FA65DD9FED367A364C364B374ADA
:103C0000DFF8E0E0F6EE007AE0EE077AFDEEE77A24
:103C100017EE901ACE1784FB010483FB0103C6EB59
:103C2000A414C6EB631382FB040C82FB0327E0178A
:103C30008EFB0121DA17C0EBAC00C2EBA70200EB50
:103C4000800002EB8202A4EB4000A3EB4202C6EB31
:103C50002131303030323031C0B2D2B2C9B202E09C
:103C60003922104611461E4B8DF806204FF0010EEA
:103C700000224FF480774026022430298DF804106A
:103C80008DF80500C3F82CE01F625E62DC609A626A
:103C90001A611A755A759A61DA611A728DF80720DD
:103CA00007D0152201A883E82400FFF7FBF803B032
:103CB000F0BD202230288DF8042008BF8DF80520A3
:103CC000EFE7302210461146CDE700BF00C079442F
:103CD0000000C842D34D62101F85EB5167666666CF
:103CE000782AFF1FAD8BDB6891420B46A8BF1346B5
:103CF000002B4ADB531A002BB8BF5B42012B54DD6B
:103D0000914230B434DC002937DBD02A44DC00EBAC
:103D1000410400EB4203A4899D894B1C07EE904AA5
:103D2000B8EE677A07EE905A511A06EE901AF8EE3E
:103D3000E77AB8EEE66A77EEC77A9A42C7EE866A05
:103D400014DD511D00EB430303F10A0200EB4101B6
:103D5000B6EE006A37EE267A77EE067AFCEEE77A60
:103D600017EE903A22F8023F8A42F3D130BC7047F6
:103D70000B46114600291A46C7DA00EB420101231F
:103D80008C8984818D890021C8E791420B46B8BF98
:103D90001346D02BAEDD704700EB41024B1C9589DA
:103DA000A0F8AC519489D022B8E77047F8B54FF429
:103DB000D172044600210C3012F0C0F9D12200214A
:103DC00004F5D77012F0BAF92022002104F52D7005
:103DD00012F0B4F9194B1A4AC4F884324FF0FF318B
:103DE0000023012000254FF07A574FF07D56A16047
:103DF000C4F8802234219C2284F8B332C4F888723B
:103E0000C4F88C62C4F8A05284F8AE0184F8B00201
:103E100023606360C4F8A432C4F8A832C4F8AC329A
:103E200084F8B13284F8B232C4F89812C4F890120F
:103E3000C4F89C22C4F89422F8BD00BFCDCC4C3EFF
:103E40000000A040D0ED017A9FED866ADFED866A22
:103E5000B8EEE77AF6EE007AE7EE067AF0B4FDEE19
:103E6000E77A0568F8EEE77A421967EEA67A00EB82
:103E70004506FDEEE77A012117EE904A05F5D77366
:103E800082F8AE11C2182946B48105E0D02900F3AA
:103E9000B08012F8014D1CB90139F7D54FF0FF3150
:103EA00003442E4605E0D02E00F3A58013F8012F21
:103EB0001AB90136F7D54FF0FF368D422B46A8BF11
:103EC0000B46002BC0F2A0806A1A82EAE273A3EBD1
:103ED000E273012B39DD8D42AABF0C462C462946E0
:103EE000002CC0F2B780D02900EB440200F3AB8075
:103EF00000EB410392899F89631C07EE902AB8EE7C
:103F0000677A07EE907A0C1BB8EEE76A07EE904AE4
:103F100036EE476AF8EEE77A9942C6EE276A14DD74
:103F200000EB43034C1D03F10A0200EB4404B6EE20
:103F3000006A37EE267A77EE067AFCEEE77A17EE1D
:103F4000903A22F8023FA242F3D1B5422B46A8BFD5
:103F50003346002B65DB721B82EAE273A3EBE2734C
:103F6000012B34DDB54237DD002E3ADBD02D00EBDE
:103F7000460261DC00EB450392899989731C07EEC8
:103F8000902AB8EE677A07EE901AAE1B06EE906A9A
:103F9000F8EEE77AB8EEE66A77EEC77A9D42C7EEAA
:103FA000866A14DD00EB4303691D03F10A0200EB8E
:103FB0004101B6EE006A37EE267A77EE067AFCEE1D
:103FC000E77A17EE903A22F8023F9142F3D10123AB
:103FD00080F8B132F0BC704733462E46002E1D46A5
:103FE000C4DA00EB450101238A8982818989002690
:103FF000C5E7D12154E78D422B46A8BF0B46002BC5
:104000004FF0D106BFF660AF8D422B46B8BF0B46CE
:10401000D02B7FF759AFB5422B46A8BF3346002BB4
:1040200099DAB5422B46B8BF3346D02B93DD012336
:1040300080F8B132F0BC70479189A0F8AC11731CC4
:104040009289D0259BE79789A0F8AC71631C92896F
:10405000D02152E700EB41040123A2898281A78984
:1040600000244AE7FA007A3CEC118342F8B58468F0
:10407000CF29D4BF21EAE175D025002C056022DBD1
:10408000174606464FF4D17207F10C010C300FF0C1
:10409000C7FC07F5D771D12206F5D7700FF0C0FC29
:1040A000A54211DB04F5D77333440022D02C04F170
:1040B0000104D8BF1A70AC4203F10103F6DD3046AB
:1040C000FFF7C0FEF8BDF8BD23462C461D46E9E7C4
:1040D00010B5D1220446002112F030F8202204F15C
:1040E000DC00002112F02AF80023012284F8D820F5
:1040F000C4F8D43084F8D93010BD00BF41F2E832A2
:10410000F0B5825804464FF4357341F22F4003FB5B
:1041100002F303F58A61255C214483B0081D234422
:10412000002D6CD041F23C46D3F85454A759444E6C
:10413000ED1B05F5514585FB06672F44EE17C6EBD1
:10414000E716D12707FB165525EAE575C3F8545441
:1041500091ED017ADFED3B6AB8EEC77AC7EE267AB9
:1041600067EEA67AF5EEC07AF1EE10FA60D9F4EEB9
:10417000E67AF1EE10FA54DABDEEE76A4FF4B57361
:1041800016EE101A03FB021304EB43010B46B1F8C1
:104190006014B3F8623407EE101A06EE903AB8EEE7
:1041A000C66AB8EE477AF8EE666A77EEC67A76EEB9
:1041B000C76AB6EE006AA7EEA67A37EE067AFCEE7C
:1041C000C77ACDED017ABDF804304FF4357101FBAB
:1041D0000242C2F858348368002B01DBFFF732FE3D
:1041E00041F23C4504F5A25041F22E4141F22F42EA
:1041F0000023635103606354A35403B0F0BD41F244
:104200003C45D3F8543465595B1B4FF43575D02BBE
:1042100005FB0245D4BF23EAE373D123C5F8543428
:1042200096E74FF4357303FB0243B3F80036CCE74F
:104230004FF4357303FB0243B3F86034C5E700BFA6
:1042400061E1C89C0000504341F2E832F0B5825869
:1042500004464FF4357341F22F4003FB02F303F59C
:104260008A61255C214483B0081D2344002D00F0A1
:10427000BD8041F23C46D3F85454A7596C4EED1B17
:1042800005F5514585FB06672F44EE17C6EBE7168B
:10429000D12707FB165525EAE575C3F8545491ED6F
:1042A000017ADFED646AB8EEC77AC7EE267A67EE68
:1042B000A67AF5EEC07AF1EE10FA40F2B280F4EE92
:1042C000E67AF1EE10FA80F2A380BDEEE76A4FF4D1
:1042D000B57316EE101A03FB021304EB43010B46F1
:1042E000B1F86014B3F8623407EE101A06EE903A93
:1042F000B8EEC66AB8EE477AF8EE666A77EEC67A26
:1043000076EEC76AB6EE006AA7EEA67A77EE067A70
:10431000FCEEE77ACDED017ABDF804304FF435714B
:1043200001FB0242C2F858348368002B01DBFFF71F
:1043300089FD41F2324241F23C46A15C04F5A253B0
:1043400041F22E4541F22F400022A2511A606255DF
:104350002254002963D041F2E83104F5A15061589C
:10436000354E41F230474FF435730025E25103FBDF
:1043700001F1456141F2384704F5A25504F5A65014
:1043800001F203631A3001F58C61E25123442144A8
:1043900096466E60044602224FF6ED7705E0D12A7C
:1043A00003F1010301F102011AD014F8015F013297
:1043B000002DF4D01D78002DF1D04E88751EADB2C1
:1043C000BD42ECD90D88B542E9D18E88AE4208BF16
:1043D00083F800E0D12A03F1010301F10201E4D1E5
:1043E000002103B0BDE8F04011F0A8BE41F23C4509
:1043F000D3F8543465595B1B4FF43575D02B05FB4E
:104400000245D4BF23EAE373D123C5F8543446E709
:104410004FF4357303FB0243B3F800367EE703B075
:10442000F0BD4FF4357303FB0243B3F8603475E716
:1044300061E1C89C00005043CDCCCC3D41F2E83353
:104440002DE9F04F50F803800288B0F840304FF467
:10445000357606FB080606F58A6606F104099B1AFE
:104460001BB283B00446D9F80470002B00F097808B
:1044700090F855107268002900F0638141F28D4177
:104480000120605403EB83034FEA430A0AEB020363
:104490004FF4357BCF2B0BFB08FBD8BF23EAE37A25
:1044A00004EB0B03C8BF4FF0D00AD3F85C54C3F839
:1044B00054A4002D27DB03F58C604FF4D17204F176
:1044C0008C010FF0ADFA04EB0B0000F20260D12278
:1044D00004F22E210FF0A4FAAA45C0F246814FF44F
:1044E000357202FB08F20021D02D02EB0503D8BF84
:1044F0001B1905F10105D8BF83F802165545F3DDF8
:104500004846FFF79FFCD6ED017ADFEDB96AB8EEB9
:10451000E77AC7EE267A67EEA67AF5EEC07AF1EE74
:1045200010FA40F23D81F4EEE67AF1EE10FA80F2F4
:104530001581BDEEE76A4FF4B57316EE102A03FB42
:10454000082304EB43021346B2F86024B3F8623444
:1045500007EE102A06EE903AB8EEC66AB8EE477A31
:10456000F8EE666A77EEC67A76EEC76AB6EE006A4D
:10457000A7EEA67A37EE067AFCEEC77ACDED017A81
:10458000BDF804204FF4357303FB0843C3F85824E7
:10459000D9F80830002B02DB4846FFF753FCB4F88B
:1045A000423062889B1A1BB2002B70D094F85620C0
:1045B000002A00F0BD8041F28E4101226254104673
:1045C00083EAE371A1EBE371302904DD5B0083EA48
:1045D000E371A1EBE371022914DD03EB430383EAEA
:1045E000E371A1EBE37110290CDD002B40F3D380C4
:1045F0000122A1F108035B0002FB03F383EAE371EC
:10460000A1EBE371082907DD002B40F3BF800122F5
:104610000B1F5B0002FB03F310B1652202FB03F3E7
:1046200003EB83133B44A3F165014FF635729142CE
:1046300015D807EE903A9FED6C6ADFED6C6AF8EEE4
:10464000E77AB6EE007AA7EE867AFDEEC77AF8EE44
:10465000E77A67EEA67AFDEEE77A17EE903A4FF624
:10466000FE7293424FF4357202FB0842D4BF23EA34
:10467000E3734FF6FF73C2F85834D9F80830002BB3
:1046800002DB4846FFF7DEFB4846FFF7DBFB94F80A
:1046900055300BB9637D43BB94F8563013BBA37DF3
:1046A00003B341F28E43E35CE3B941F22542A15CDE
:1046B00000295ED104F18000814504D04FF43572A9
:1046C00049460FF0ADF941F225430122E254484634
:1046D000FFF7B8FB4FF4357303FB0844D4F85434A8
:1046E000C4F85C3403B0BDE8F08F41F22243E35CD0
:1046F000002BD1D141F28D43E35C002BCCD141F2B0
:104700002540215C002952D041F2E8314FF4357246
:104710006158235402FB014304F180014FF0FF3044
:104720008945C3F85C04B7D048460FF079F9B3E780
:1047300094F85F20002A7FF43EAF41F28E42A05CE5
:104740003EE790F85E1000297FF498AE41F28D416B
:104750009A46415C00293FF499AE93E64FF43573D5
:1047600003FB0843B3F800260CE75346AA461D4650
:10477000B5E641F2E8314FF435706158A35400FBBF
:1047800001444FF0FF33C4F85C34ABE714BF4FF083
:10479000FF3200223CE714BF4FF0FF32002228E72F
:1047A0004FF4357303FB0843B3F86024EAE64FF493
:1047B000357303FB08F3E018D0F85424D02A35D819
:1047C0008518D01800F2026085F8021620441146C0
:1047D00002E010F8015D15B911F1FF31F9D213446F
:1047E00003F20263234408E0FA007A3CEC118342AE
:1047F0000000504313F8010F10B90132D12AF9D14A
:104800004846FFF771FA4FF4357303FB08434FF442
:10481000B572D3F8541402FB081204EB42020121D2
:10482000B2F86024C3F8582483F8051796ED017A8E
:104830005FED116AB8EEC77AC7EE267A67EEA67A00
:10484000F5EEC07AF1EE10FA43D9F4EEE67AF1EE25
:1048500010FA14DB4FF4357303FB0843B3F800265A
:104860004FF4357303FB0843C3F85824D9F80830D4
:10487000002BFFF611AF4846FFF7E4FA0CE7BDEE58
:10488000E76A4FF4B57316EE102A03FB082304EB16
:1048900043021346B2F86024B3F8623407EE102ADC
:1048A00006EE903AB8EEC66AB8EE477AF8EE666A57
:1048B00077EEC67A76EEC76AB6EE006AA7EEA67AFB
:1048C00077EE067AFCEEE77ACDED017ABDF80420AA
:1048D000C6E74FF4357303FB0843B3F86024BFE722
:1048E0002DE9F0479FED8A6ADFED8A5A9FED8A5ADB
:1048F000DFED8A4A00F5A4560F3600F1440800F1B6
:10490000040C044600F2D46700F59E5E01460025C3
:1049100038F8023F3CF8022F9B1A1BB2002B44D000
:1049200094F86520002A4FD194F86920002A4BD1D1
:104930003278002A4AD194F86120002A4ED19EF89C
:104940000090B9F1000F5CD091F804A791F8072707
:10495000BAF1000F0CBF4FF0FF3A4FF0010AC2F15D
:104960006302112B02FB0AF200F3AC8013F1110F6A
:10497000B8BF6FF011031A44622A00F39A8012F153
:10498000620FC0F2A68082EAE273A3EBE2736FEAE1
:104990000209C3F16303DBB24FEAD979012281F83E
:1049A000049781F8073781F805270135042D01F5B3
:1049B000357107F535770EF1010E04F1010406F1AA
:1049C0000106A5D1BDE8F0870122327003EB830315
:1049D00094F8612003EB83039B005AB100F5A159C1
:1049E00000F5A0524FF0010A89F801A04FF0FF39FD
:1049F000C2F81090002BD8D09EF80090B9F1000FAB
:104A0000A2D107EE103AD7ED007AB8EEC77AF0EEF1
:104A1000676AE7EE066AF4EEE56AF1EE10FA2ADD5F
:104A200077EE877AF4EEC57AF1EE10FA33D5F4EE2C
:104A3000C67AF1EE10FA47DDF4EEE57AF1EE10FAFF
:104A4000C7ED007A49DAF2EE046AF4EEE67AF1EEA6
:104A500010FAB6EE007A4DDBA7EEA67AF7EE006A02
:104A6000FDEEC77AF8EEE77A67EE867AC7ED007A50
:104A700086EEA77A15E0E7EE247AB2EE047AF4EE39
:104A8000477AF1EE10FAC8BFF0EE667AF4EEC57A16
:104A9000F1EE10FACBD49FED227ADFED1F7AC7ED4D
:104AA000007A01F5DB63012283ED007A81F80527A6
:104AB0007BE70023012281F8049781F8073781F80A
:104AC000052772E7122356E79FED167ADFED167A77
:104AD000E5E74FF000094B46ECE7B6EE007A77EEDB
:104AE000877AF7EE006AFDEEE77AF8EEE77A86EE6F
:104AF000A77AD4E7A7EEA57AF7EE006AFDEEC77AAB
:104B0000F8EEE77A67EEA47A86EEA77AC7E700BFE9
:104B1000CDCCCC3D0000C84200C079440AD7233C2C
:104B20000534833A01002041CCCCCC3D2DE9F04F37
:104B30002DED028B00F5A15BDFED918A9FED918A4F
:104B400083B006460BF1050B00F1600800F1210768
:104B5000002518F8013FEBB93B788BB106F5A1535E
:104B6000013306F5A0541B7810341BB92268AA4201
:104B700000F0AB802368AB4204BF4FF0FF332360EB
:104B80000135042D07F10107E3D103B0BDEC028B21
:104B9000BDE8F08F3B78002BF2D19BF800206AB182
:104BA00006F59F5A8BF80030DAF808304FF435726A
:104BB00002FB03634FF0FF32C3F85C2406F5A054F8
:104BC000103422684FF0000906F5A1534A4583F8D6
:104BD00001906FDBAA4267D03046FFF78FFA06F5E7
:104BE000A15312331B78002B4BD006F59F5A4FF47C
:104BF0003573DAF8081003FB01F106F5A65306F544
:104C0000A15A184606F5A25201F203631A3001F5C3
:104C10008C61CAF81090CAED058ACAF81890019004
:104C200082ED018A33443144864602224FF6ED7A02
:104C300005E0D12A03F1010301F102011DD01EF8A4
:104C4000010F01320028F4D018780028F1D0B1F813
:104C500002C00CF1FF3080B25045EAD908886045A7
:104C6000E7D1B1F804C0844504BF00201870D12AF0
:104C700003F1010301F10201E1D10198002111F0DA
:104C80005DFA06F5A0531846D4F800E0C3F814E026
:104C900019468561012008771A46002106F5A153BF
:104CA0008E455177187007DB98F80030002B7FF4A1
:104CB00067AF51E706F5A153002225601A7098F8F6
:104CC0000030002B7FF45CAF46E79BF800206AB110
:104CD00006F59F5A8BF80030DAF808304FF4357239
:104CE00002FB03634FF0FF32C3F85C2406F5A153C7
:104CF0001A78CAB906F59F5909F10C09D9F800309C
:104D0000CBB1013B06F59F5A012B0AF1080A1BD9CA
:104D100098F80030CAF80050002B7FF431AF3B7890
:104D2000002B7FF427AF2BE700221A703B78002B73
:104D30007FF420AF24E706F59F530122C9F8002035
:104D400003F1080A1A61E3E7DAF80030AB420ED04B
:104D500006F5A150C271027282713046FFF774FAF3
:104D600006F59F530122C9F800201A61D0E706F525
:104D70009F53C9F8002030461A61FFF765FAC7E76C
:104D800000000000CDCCCC3DF8B54FF6FF710446D5
:104D900000F18A0300F50B75002033F8022F9142D1
:104DA000A8BF11469042B8BF1046AB42F5D1268845
:104DB000B4F840506288B4F84230AD1B2DB29B1A53
:104DC0002E461AB2002D00F0C38094F85530002B07
:104DD00000F0068141F28D460127A75505EB8505B8
:104DE0006E0041F23C456559AD1BD12D00F30A819F
:104DF0006FF0D107BD42B8BF3D4641F23C47E55197
:104E0000002A40F0A680002E00F0C38004F5A257CF
:104E10003B68DFEDD05ADFEDD06A07EE903AF8EE4E
:104E2000E77A41F2E83267EEA55A07EE901AF8EEFB
:104E3000E77AA65837EEA55A4FF4357303FB0643BD
:104E400007EE100AB4EEE65A0122F1EE10FA83F8EA
:104E50000527B8EEC77A40F16A81B5EEC05A77EE01
:104E6000255AF1EE10FAF4EEE65A40F39E81F1EE87
:104E700010FA00F13581B4EEE65AF1EE10FAF0EED8
:104E8000665A80F23981F4EEC77AF1EE10FA00F139
:104E9000C78077EEC77ADFEDB16ADFEDB23A4FF443
:104EA0003573F4EEE67A03FB06F303F25E47F1EEA8
:104EB00010FA03F2016305F22E2135EE655AD8BFD0
:104EC000F0EE667A2744E01821442A4605F1D10C19
:104ED000B7EE004AF6EE004A13E0B7EE006AF0EED5
:104EE000656AE5EE066A0132944501F1010176EE4C
:104EF000A46AFDEEE66A16EE903A27F8023F00F04B
:104F00008380D02A94BF91F800E04FF0000ECF2AA2
:104F10004FF0D003D8BF22EAE27300F801EF04EBB0
:104F20004303B3F88C3006EE903AF8EE666A76EEFC
:104F3000C76A86EEA76AB4EEC46AF1EE10FACCD561
:104F4000B5EEC06AF1EE10FAD8BFB0EE636AC6E7FC
:104F5000EAB194F856308BB341F28E430125E55403
:104F600004F5A25702EB82023B68520013443B60F7
:104F7000002E00F0E88041F23C42A55849E706D0F7
:104F80004FF4357303FB0646012386F8D23694F8B6
:104F900055303BB9637D2BB141F22243E35C002BDA
:104FA00000F0E28094F856303BB9A37D2BB141F27A
:104FB0008E43E35C002B00F0F480F8BD94F85F3082
:104FC000002BC9D141F28E43E35C002BC8D104F51C
:104FD000A25741F23C453B68655913443B6018E7D2
:104FE00094F85E70002F7FF4F5AE41F28D47E75DD7
:104FF000002F7FF4F3AE41F23C456559AD1BD12D36
:105000007FF7F6AED225F8E6002DB8DD4FF4357304
:1050100003FB0646012386F8023694F85530B8E7BC
:1050200037EE677ADFED4D6ADFED4E3A4FF43573B8
:10503000B4EEE67A03FB06F303F25E47F1EE10FAF4
:1050400003F2016305F22E2175EEC55AD8BFB0EE0A
:10505000667A2744E01821442A4605F1D10CB7EEC0
:10506000004AF6EE004A12E0B7EE006AF0EE456A3A
:10507000E5EE866A0132624501F1010176EEA46A2D
:10508000FDEEE66A16EE903A27F8023FBCD0D02A31
:1050900094BF91F800E04FF0000ECF2A4FF0D003FC
:1050A000D8BF22EAE27300F801EF04EB4303B3F840
:1050B0008C3006EE903AF8EE666A76EEE76A86EE97
:1050C000876AB4EEC46AF1EE10FACDD5B5EEC06AC7
:1050D000F1EE10FAD8BFB0EE636AC7E79FED215A30
:1050E000DFED1D6AF5EEC05AF1EE10FAB4EEE65AA5
:1050F00063DDF1EE10FA0BDBDFED176A9FED186A46
:1051000076EEE76A66EE866AFDEEE66AC7ED006A4D
:10511000F5EEC05AF1EE10FA3FF6B5AEDFED106ACB
:1051200067EE666AFDEEE66AC7ED006AABE677EE0B
:10513000255AB0EE665AF4EEE65AF1EE10FACFD4E4
:10514000F0EE665AD8E7002A3FF421AF41F23C4224
:10515000A5585EE60000004400FF7F47BD37863556
:105160000000003B0000000041F28D43E35C002B97
:105170007FF418AF41F2E8334FF43572E05802FB88
:10518000004000F2544004F18001884201D00EF04A
:1051900047FC41F23C430022E2502046FFF754F81E
:1051A00000E72046FFF750F8F8BDF1EE10FA95D46D
:1051B000F0EE665A1FED155A65E6F1EE10FA5FED56
:1051C000175A99DAAAE700BFF8B50446B0F842309A
:1051D0004088B4F84010228894F855C01B1A1BB2BE
:1051E0008A1A03FA82F2002A4FD0BCF1000F00F0B5
:1051F000E28041F28D430121E15402EB8202520030
:1052000094F8563023B994F85F30002B00F0DF801B
:1052100041F28E430121E15402EB8202520041F23D
:105220003C4163589B1A002B635004DAD133FDD400
:1052300041F23C41635042B341F2E8321D1BA25897
:10524000DFF89CE1C2EB82129200A01802F58356AF
:1052500041F27D01AD1A0123143602F6A3724354C4
:10526000A5F6D2652644A018D127291881FB0E2364
:105270000B44CA17C2EBE31307FB1313234493F841
:10528000543300F8013FB042EFD1BCF1000F02D11E
:10529000637D002B6DD194F856302BB9A37D1BB1E3
:1052A00041F28E43E35C33B194F85930002B57D16F
:1052B000637E002B54D02046FEF720FF41F232439C
:1052C000E35C002B54D041F2E8324FF43573A2581E
:1052D000424E04F5A15003FB02F241F23047002593
:1052E0004FF0000E02F2036302F58C62E551A11843
:1052F000C0F814E004F5A25241F2384704F5A65074
:105300001A30E55123445660AE46044602224FF659
:10531000ED7705E0D12A03F1010301F102011AD072
:1053200014F8015F0132002DF4D01D78002DF1D06A
:105330004E88751EADB2BD42ECD90D88B542E9D19B
:105340008E88AE4208BF83F800E0D12A03F1010342
:1053500001F10201E4D10021BDE8F84010F0EEBEF9
:1053600094F85C3023B9237F13B1637F002BA2D064
:10537000F8BD41F22243E35C002B8CD141F28D4316
:10538000E35C002B87D141F2E83304F55571E35813
:10539000C3EB831304EB830000F6A470884202D0B1
:1053A000FC220EF03DFB41F23C430022E25020463D
:1053B000FEF74AFF6FE794F85E30002B7FF419AFD9
:1053C00041F28D43E35C002B3FF41AAF15E741F245
:1053D0008E43E35C002B3FF422AF1DE7CDCCCC3DE8
:1053E00061E1C89C90F86130002B40F0968190F804
:1053F0006230002B40F0918190F86330002B40F038
:105400008C8190F86430002B40F08781F0B541F238
:10541000EC3383B0C358022B044605D090F85C20CF
:10542000002A51D003B0F0BD41F22843C35C002BE9
:1054300055D141F22643C35C002B50D141F22743A2
:10544000C35C002B4BD141F22E43C35C002B46D1F1
:1054500041F22F43C35C002B41D190F85C30002B0C
:105460003DD1037F002B3AD0437F002B37D141F24F
:10547000E833C358C3EB8315AD0005F57A620244E7
:10548000D2F8D820002A2ADD4FF4357202FB03033C
:105490000544D3F8541403F2544042F210720B4600
:1054A0000EE0D12BA8BF0023EE1896F8A46F002EB3
:1054B00040F09281994200F09081013A00F0A08181
:1054C0000133EED5D023EFE7027F002AAAD0427F36
:1054D000002AA7D1012B00F07781022BA2D1B4F8CA
:1054E00042206188B4F840002388521A12B2C31ACD
:1054F00002FA83F3002B56D041F2E8324FF43575AF
:10550000A65894F8552005FB064505F58A652F1D1C
:10551000696822B994F85E20002A00F03D8141F2CA
:105520008D420120A05403EB83035B0094F85620C6
:1055300022B994F85F20002A00F0278141F28E42C0
:105540000120A05403EB83035B00194404F18002A3
:105550003846FEF78BFD95ED017ADFEDAC6AB8EECB
:10556000C77AC7EE267A67EEA67AF5EEC07AF1EE34
:1055700010FA40F22281F4EEE67AF1EE10FAC0F26F
:10558000CD804FF4357303FB0643B3F800264FF488
:10559000357303FB0643C3F85824BB68002B02DBBA
:1055A0003846FEF74FFC94F85630002B40F0A380AD
:1055B000A37D002B00F09F8041F28E43E35C002B23
:1055C00040F0998041F2E8324FF43573A25803FB62
:1055D0000243D3F854049301CF28A3EB020140F314
:1055E000E28041F2740004EB8101D025095C81F076
:1055F000010081420ED0991A04EB810141F27D062F
:1056000001278F5541F27807CE59002800F0E1803C
:105610000136CE519B1A04EB83032B4483F8A40F6D
:1056200094F85A300BB3A37EFBB941F22542A15C3A
:10563000002940F09D802046FEF760FD41F2E833EE
:105640004FF43572E15802FB014141F2274641F225
:105650002E4301F2544104F18000002701258842C5
:10566000A755E55401D00EF0DBF994F85D30002B1E
:105670003FF4D8AE617F00297FF4D4AE41F2E83325
:10568000E358C3EB831204EB820202F57A62D2F88C
:10569000D820002A7FF7C6AE41F22542A05C40B177
:1056A0004FF4357000FB03434FF0FF30A154C3F8B3
:1056B0005C042046FEF722FD41F2E83341F2274721
:1056C000E358C3EB831104EB810141F2264641F21A
:1056D0002F4201F6A47104F555700023012588427C
:1056E000E355A355A5543FF49DAEFC2203B0BDE89D
:1056F000F0400EF095B994F85530002B90D1637DB1
:10570000002B8DD041F22243E35C002B88D141F283
:105710008D43E35C002B83D154E77047BDEEE76A0D
:105720004FF4B57316EE102A03FB062304EB430275
:105730001346B2F86024B3F8623407EE102A06EE7E
:10574000903AB8EEC66AB8EE477AF8EE666A77EE37
:10575000C67A76EEC76AB6EE006AA7EEA67A77EE4C
:10576000067AFCEEE77ACDED017ABDF804200EE76B
:1057700041F2E8314FF435706158A35400FB014306
:105780004FF0FF32C3F85C2455E741F28E42A25C31
:10579000002A3FF4DAAED5E641F28D42A25C002A3F
:1057A0003FF4C4AEBFE620EAE07504EB8101294472
:1057B00091F8A41F81F001001BE74FF4357303FB40
:1057C0000643B3F86024E2E641F2EC330222E250F1
:1057D00085E6013ECE511DE7194604F18002FEF731
:1057E00045FC94F85C306BB941F2EC33227FE3580E
:1057F000002A3FF472AE627F002A7FF46EAE69E643
:105800001146EAE741F2EC33E35866E60000504304
:105810002DE9F04341F2E83290F85B30845883B0D0
:10582000064623BBC27E002A00F0108190F820506B
:105830008DB941F23242825C002A40F0238141F26C
:105840002F42825C002A40F01D8141F22E42825C90
:10585000002A40F0178141F22842B15C002940F053
:10586000F980002D00F0588203B0BDE8F08341F2CA
:10587000284190F86020415C002A00F0C68096F82C
:105880002020002A40F0C1804FF4357303FB0463ED
:105890000121D3F8002783F805175242002AC3F8E4
:1058A000002740F0EC80C3F8001741F22F414FF47D
:1058B0003573755C03FB04F341F2284103F58A62FA
:1058C00041F2264E4FF0010C41F2274706F801C085
:1058D0003244002106F80E10101DF1553344002DFE
:1058E00000F0DE8141F23C45D3F854147759764DEF
:1058F000C91B01F5514181FB058901EB0907CD1752
:10590000C5EBE715D12707FB151121EAE171C3F8B3
:10591000541492ED017ADFED6E6AB8EEC77AC7EEE5
:10592000267A67EEA67AF5EEC07AF1EE10FA40F22A
:105930003182F4EEE67AF1EE10FAC0F2C3814FF450
:10594000357303FB0463B3F800264FF4357303FB90
:105950000464C4F858248368002B01DBFEF772FA54
:1059600041F2324241F23C45B15C06F5A25341F2AC
:105970002E4441F22F40002272511A6032553254A7
:10598000002900F0868041F2E83141F2304471583C
:10599000325106F5A1504FF435734FF0000EC0F8A8
:1059A00014E003FB01F106F5A25441F2384706F575
:1059B000A65001F20363454DF25101F58C611A3096
:1059C0009446656033443144044602224FF6ED7E2E
:1059D00005E0D12A03F1010301F1020156D014F8C8
:1059E000015F0132002DF4D01D78002DF1D04F88D9
:1059F0007D1EADB27545ECD90D88BD42E9D18F88C9
:105A0000AF4208BF83F800C0E3E700293FF42CAFA2
:105A10004FF4357202FB0462D2F80017002959DDF9
:105A2000002B7FF421AFF37E002B3FF41DAF96F8DF
:105A30002030002B7FF418AF01310329C2F8001782
:105A40007FF712AF0123C2F800370DE741F2284279
:105A5000825C4AB196F86020002AD9D096F82020BE
:105A6000002A3FF411AFD3E790F86030002B3FF4E9
:105A7000FBAE90F82030002B3FF406AFF4E67FF742
:105A8000F3AE12E73046FEF7DFFBEDE6002110F043
:105A900055FB41F22543F25C62B141F2E8324FF42A
:105AA0003571B25801FB026200204FF0FF31F05413
:105AB000C2F85C1441F2EC3141F2F0320123735030
:105AC000B35003B0BDE8F08361E1C89CCDCCCC3DC0
:105AD0000000504341F22F41715C002940F0C98021
:105AE00041F22E41715C002940F0C380ABB9F07ED9
:105AF000002800F0668196F8203073B9D2F8FC16C1
:105B00000029C0F2668101310125032982F8055779
:105B100000F36781C2F8FC160346B6F840203188CE
:105B2000521A12B21546002A48D096F8551000298C
:105B300040F03F8196F85E10002940F03A8141F232
:105B40008D41715C002940F038814FF4357000FBC5
:105B500004600122D0F8E41680F805274FF4357070
:105B600000FB04606A18CF2AD0F8E8161FED287AE7
:105B7000D4BF22EAE272D0228A42D8BF114607EE91
:105B8000901AF8EEE77AC0F8E426C7EE876A4FF479
:105B9000357202FB0462C8BFC0F8E41602F2DC6092
:105BA00002F5DC61C0ED006AD2F8E82607EE902A23
:105BB000F8EEE77AC7EE876AC1ED006AB6F84220D0
:105BC0007188521A12B21546002A46D096F856101D
:105BD000002940F0E68096F85F10002940F0E1804F
:105BE00041F28E41715C002940F0DF804FF4357046
:105BF00000FB04600122D0F8E81680F805274FF476
:105C0000357000FB04606A18D0F8E4161FED507A76
:105C100007EE901AF8EEE77ACF2AC7EE876AD4BF6C
:105C200022EAE272D022C0F8E8268A424FF43572A6
:105C300002FB0462B8BFC0F8E81602F2DC6002F5AD
:105C4000DC61C0ED006AD2F8E82607EE902AF8EE93
:105C5000E77AC7EE876AC1ED006A002B3FF404AE15
:105C60004FF4357303FB0463D3F80037002B3FF781
:105C7000FBAD4FF4357303FB0464D4F8FC36002B02
:105C80003FF7F2AD41F2284041F2264141F227426E
:105C90000023335473543046B354FEF7D5FA09E762
:105CA00041F23C41D3F8543471585B1A4FF43571CA
:105CB000D02B01FB0461D4BF23EAE373D123C1F8E5
:105CC000543426E6BDEEE76A4FF4B57316EE102A9B
:105CD00003FB042306EB43021346B2F86024B3F837
:105CE000623407EE102A06EE903AB8EEC66AB8EEB5
:105CF000477AF8EE666A77EEC67A76EEC76AB6EE4F
:105D0000006AA7EEA67A77EE067AFCEEE77ACDED8A
:105D1000017ABDF8042018E641F2264041F22741FD
:105D20000123355475543046B354FEF78DFA41F2D1
:105D30002543F25C5AB141F2E8324FF43571B25862
:105D4000F55401FB02634FF0FF32C3F85C2441F2CB
:105D5000F03141F2EC3001224FF43573325003FB45
:105D600004637250D3F8001700293FF77DADD3F8D4
:105D7000FC16002927DB4FF4357303FB0464D4F8C9
:105D8000FC36002B7FF470AD0123C4F8FC3684F898
:105D9000053769E54FF4357303FB0463B3F86024FA
:105DA000D3E541F28E410120705402EB820255008E
:105DB0001CE741F28D410120705402EB8202550034
:105DC000C3E60123A9E64942C3F8FC1683F8052778
:105DD000D1E749420125C2F8FC16034682F805576F
:105DE0009BE641F22841C2F8FC36735495E600BFA9
:105DF0002DE9F04F2DED048B90F8573089B0044613
:105E0000002B40F0B680C37D002B00F0B280237ED3
:105E1000002B00F0438141F23043E35C002B40F063
:105E2000958194F854302BB941F22643E35C002B62
:105E300040F0A98041F23243E35C2BB141F22F43A1
:105E4000E35C002B00F01A8341F23043E35C002B4B
:105E500040F0AC8041F22643E35C002B00F08480EC
:105E600041F2E831B4F84030228865584FF4357675
:105E70009B1A06FB05461BB206F254461946002B38
:105E800000F0A08141F22742A25C002A00F0A0822B
:105E900004F5A357D7ED067AF5EEC07AF1EE10FAC5
:105EA00007F1180740F32D8304F5A05393ED037A0F
:105EB00077EEC77AF5EEC07AF1EE10FAC7ED007A08
:105EC00094BF4FF001084FF000084FF4357303FB07
:105ED000054303F2F463B4F84420A188D3ED007ABB
:105EE00001234FF4357000FB0540C0F8F826002B65
:105EF00040F0BE8141F23143E35CABBB4FF43573FC
:105F000003FB05439FEDAE7AD3F8EC0607EE900A4B
:105F1000F8EEE77A03F2F46087EE876A80ED006AB4
:105F2000D3F8EC0607EE900AF8EEE76AC6EE877A39
:105F300067EE877AF5EEC07AF1EE10FA40F2178438
:105F4000F4EEC77AF1EE10FAC0F21C83B3F8003613
:105F5000994200F007849A1A002AA3EB010140F34A
:105F60000F84002940F3548309B0BDEC048BBDE8D5
:105F7000F08F94F85830002B3FF44DAF237E002B68
:105F80007FF449AF8AE041F28943E35C002B7FF460
:105F900051AF94F85A301BB1A37E002B3FF44AAFA7
:105FA00041F23043E35C002B3FF45AAF41F23143FE
:105FB000E35C002B3FF44EAF94F8521041F23245AF
:105FC00041F2334201F0020301260020665503F03E
:105FD000FF0EA0541BB941F2384344F803E0B4F972
:105FE0004E30002BFFF636AFB4F95020002AFFF6F2
:105FF00031AF07EE903ADFED6A6A9FED6A7A9FED66
:106000006A6AF8EEE77AA7EEA67AF0EE477AC7EE6C
:10601000866AB7EE007AF4EEC76AF1EE10FA08D598
:106020009FED627AF4EEC76AF1EE10FAC8BF36EE61
:10603000877A07EE902A9FED5A6ADFED5D6ADFED01
:106040005D5AF8EEE77A04F5A257E7EE866A103754
:10605000F7EE007A86EEA56A87ED007AB4EEE76A7D
:10606000F1EE10FA08D5DFED517AB4EEE76AF1EE01
:1060700010FAC8BF76EE277A04F5A25808F1140882
:10608000CB07C8ED007A40F13F8241F2334104F57D
:10609000A153494A012060545A61DBE641F226438C
:1060A00041F2284041F22741012200252554655440
:1060B0002046E254FEF7C8F841F22542A35C002BCB
:1060C00040F0538241F2E833E358DFED3D6A41F29C
:1060D000EC3541F2F03001224FF43571625101FB91
:1060E00003432250D3F8EC2607EE902AF8EEE77A25
:1060F00003F2F46287EEA67A82ED007AB4F84420C7
:10610000C3F8F82694F85830002B3FF484AE217E73
:1061100000297FF480AE41F22643E35C002B3FF47C
:106120007AAE41F23042A35C83F00103A354002B0A
:1061300000F02183214B1B680493049B41F25C40D7
:1061400041F2274203F5FA732350A15494F85330D7
:10615000DBB91A4B41F25C421B680593059BA258C0
:106160009B1A002B7FF75DAE002A3FF45AAE204603
:10617000FEF76AF841F23043E35C002B3FF451AE86
:1061800094F85330002B3FF44CAE41F23143E15CC4
:10619000002900F07D8141F231430122E25440E6C2
:1061A000D54C07380AD723BD1E856B3F0000000081
:1061B0000AD7A3BD0BD7633F8FC2753D80B2FF1FC7
:1061C00000005043B4F84230618841F227425B1A24
:1061D0001BB2A25C002B00F03D81002A7FF458AE78
:1061E00094F8562022B994F85F20002A00F0F48138
:1061F00041F28E420121A15403EB83035B004FF473
:10620000357202FB05424FF43571D2F8F02601FBDE
:1062100005411344CF2BD1F8EC26D4BF23EAE37316
:10622000D0239342C1F8F03601DAC1F8F02607EE28
:10623000902A5FED1D6AB8EEE77A4FF43573C7EE2A
:10624000267A03FB054303F2F463C3ED007AB4F846
:106250004420A18891423FF487AE4FF4357000FB93
:10626000054000239846C0F8F826002B3FF442AEC4
:106270001FED2D7A67EE877A04F5A357B946FDEE38
:10628000E78A183709F11409B4F84430A288934218
:1062900004F5A05100F02481D64891ED036A3860DE
:1062A00007EE903AB8EE677A07EE902AF8EEE76AC2
:1062B000DFEDD15A9FEDD15A77EE667A76EE254A18
:1062C000F0EEE77A67EEA57AF7EE006A87EEA47A39
:1062D00037EE267AC5EE076AC9ED006A4FF43573CA
:1062E00003FB054303F2F462D2ED007A9FEDC77A17
:1062F000E6EE867AC2ED007AD3F8F03606EE903AF2
:10630000B8EEE66AC6EE076AF4EEE67AF1EE10FA47
:106310004EDDF6EE007AE6EE877AC2ED006AFDEE1B
:10632000E77A17EE907A04F1800239463046FDF79D
:106330009DFE4FF4357303FB05434FF6FE72D3F811
:10634000F83693424FF4357202FB0542D4BF23EA7C
:10635000E3734FF6FF73C2F85834B368002B02DBC7
:106360003046FDF76FFD3046FDF76CFD4FF4357399
:1063700003FB0545D5F8F0369F42FFF6F5AD41F237
:10638000284141F2264241F227400023235463541E
:106390002046A354FDF7B2FE41F2EC3141F2F03257
:1063A00001236350A35009B0BDEC048BBDE8F08F0E
:1063B000F6EE006AE7EE876A18EE902AFDEEE67ABE
:1063C00017EE907ABA42AED1B8F1000FD4D0AAE756
:1063D00094F8552022B994F85E20002A00F0038139
:1063E00041F28D420121A15403EB830359004FF484
:1063F000357303FB0543DFED856AD3F8EC268B1874
:106400004FF4357101FB0541CF2BD1F8F026D4BFF5
:1064100023EAE373D0239342D8BF1A4607EE902AAB
:10642000F8EEE77AC1F8EC3687EEA67A4FF43573CA
:1064300003FB054303F2F463C8BFC1F8EC2683ED08
:10644000007AB4F8423062889B1A1BB2002B7FF4AA
:10645000C7AE02E0002A7FF41BADB4F84420A18847
:1064600091423FF481AD4FF4357000FB054000F2DE
:10647000F4600023D0ED007A984632E52046FDF71F
:10648000E3FE41F23043E35C002B3FF4E3AC8DE5E7
:106490005B4B5C4F1B68069341F2E8334FF4357554
:1064A000E358069A05FB0343D026C3F8EC16C3F85D
:1064B000F06604F5A25503F2F463002041F2584E51
:1064C000A2F51C521860103AA860E86004F5A650C6
:1064D00044F80E201A306F60D1220FF02FFE5AE6DA
:1064E000D7ED006A9FED487A91ED036AF4EEC76A32
:1064F000F1EE10FA3FF6D4AEF0EE476A89ED007A7D
:10650000ECE64FF00008E0E43D4A41F258431268DF
:106510000792E358079904F5A052C3EB010904F56B
:10652000A25392ED036AD3ED016A04F5A25576EE0B
:10653000C66A2E46B9F1320F05F1080506F10C06C0
:1065400041F25842F5EEC06AC4BF85ED007AC6ED4F
:10655000007AF1EE10FAA150C3ED016A40F2A78073
:1065600085ED007AC6ED007A74E441F2E8334FF429
:106570003571E358A55401FB03424FF0FF31C2F8D7
:106580005C14A2E5FDEEE75A4FF4B57315EE900AE0
:1065900003FB050304EB43000346B0F86004B3F8C3
:1065A000623407EE100A06EE903AF8EEE55AB8EEBD
:1065B000477AF8EE666A77EEE57A76EEC76AF6EE27
:1065C000005AA7EEA67A37EE257AFCEEC77ACDED13
:1065D000017ABDF80430BBE441F28E42A25C002A8D
:1065E0003FF40DAE08E641F28D42A25C002A3FF472
:1065F000FEAEF9E6CDCC4C3DACC527370AD7233EDD
:1066000080B2FF1FCDCCCC3D000000000000504305
:106610003FF4AAAC1FED038AD64BB6EE009AF0EE1B
:10662000497AE6EE087A04F5A3594F4641F227422B
:10663000FDEEE78A09F1140918370120A05418EE7D
:10664000901AC9F8003004F180023B603046FDF733
:106650000DFDF8EEE87A87EE887A27EE087AB5EE37
:10666000C07AF1EE10FA40F2C280B4EEC87AF1EED0
:1066700010FAC0F294804FF4357303FB0543B3F86E
:1066800000264FF4357303FB0543C3F85824B36861
:10669000002B02DB3046FDF7D5FB3046FDF7D2FB81
:1066A00041F22743E35C002B7FF4EEAD5CE441F262
:1066B000E8324FF43573A158BEF1000F00F09E8010
:1066C00003FB014341F2384BD3F8EC26D3F8F03604
:1066D00007EE902A06EE903AF8EEE77AF8EEE66AD0
:1066E00054F80B2076EEE76AE6EE877AFDEEE77A5D
:1066F00017EE903ACF2BD4BF23EAE37A4FF0D00ABB
:10670000002A00F01781B9F1320F22DD41F2E8339F
:1067100054F803E04FEA8E11CEEB010004EB800049
:1067200000EB0A0393F8A43F5BB941F2780C41F205
:106730007D0950F80C30013340F80C30012300F88B
:106740000930CEEB010304EB83035344012183F8AA
:10675000A41F41F238430132E25097ED007AD8EDA0
:10676000007AFDE691427FF455AFFFF7F4BBB3F832
:106770006034FFF7EDBB2046FDF766FDFFF74BBB2E
:1067800014BF4FF0FF320022002940F3C0800123E4
:1067900003FB02F301333FF43DAFFFF7E5BBBDEE72
:1067A000C76A4FF4B57316EE102A03FB052304EBFA
:1067B00043021346B2F86024B3F8623407EE902A1D
:1067C00006EE903AF8EE677AB8EEC66AF8EE666AB8
:1067D00037EE467A76EEE76AE7EE267A77EE897A42
:1067E000FCEEE77ACDED017ABDF8042049E74FF4DD
:1067F000357303FB0543B3F8602442E703FB01F361
:10680000E2181346D2F8EC06D2F8F026D5ED005A7D
:1068100006EE900A06EE102AF8EEE66AB8EEC66AB0
:10682000B0EE665A36EE666A03F2544BA5EE865A0F
:10683000E6EE076AFDEEC55A15EE909AB9F1CF0F54
:106840006ADCFDEEE66A29EAE97916EE902ACF2A9B
:1068500000F3838022EAE272914540F387804FF093
:10686000FF3302F1FF3A1846914571D0C9EB02039C
:1068700083EAE372A2EBE37296ED008A06EE902AB9
:1068800037EEC86AF8EEE66A86EE269AD1453FF4FE
:1068900067AE4FF4357202FB014304F180020195AB
:1068A0000296039705465F461646DFED338A9B4600
:1068B000324649463846FDF7D9FB68EE287A4FF64E
:1068C000FE73FDEEE77A4FF6FF7117EE902A9A42BB
:1068D000D8BF22EAE271CBF85814BA68002A3846C9
:1068E00001DBFDF7AFFA3846FDF7ACFA09F5A65221
:1068F0001A32A9440121D14538EE098AA154D7D1D1
:1069000001ADE0CDD8ED007A97ED007A28E63FF4AE
:106910002BAB4FF0FF333BE7FDEEE66A16EE902A15
:10692000CF2A1EDD4FF0D0094A464FF0D10A01238D
:10693000184699E7C1EB811104EB810000F6A470C1
:10694000FDF7C6FB54F80B20002A3FF4DFAEDAE671
:10695000B0EE678A9FED099A98E74FF0D10AD022EE
:10696000E5E722EAE2724FF0D00978E702F1010A86
:10697000DDE700BFCDCC4C3D00FF7F4700000000AD
:106980002DE9F04190F85A3082B0044633B990F8BE
:106990005920002A4ED1427E002A4BD0A27E002AE6
:1069A00048D141F2EC32A258012A00F0878041F22E
:1069B000264141F2274241F22840002323546354E8
:1069C0002046A354FDF79AFB94F85A2041F2EC308C
:1069D00041F2F0310123235063505AB3A37E4BBBE5
:1069E00041F22542A15C59B141F2E8314FF43570D2
:1069F0006158A35400FB01434FF0FF32C3F85C24FD
:106A00002046FDF77BFB41F2E8334FF43572E15845
:106A100002FB014141F2274641F22E4301F254416B
:106A200004F18000002701258842A755E55401D0D4
:106A30000CF0F6FF94F85D30002B3CD0617FD1BBA9
:106A400041F2E833E358C3EB831204EB820202F510
:106A50007A62D2F8D820002A2DDD41F22542A05CCE
:106A600040B14FF4357000FB03434FF0FF30A154A9
:106A7000C3F85C042046FDF741FB41F2E83341F2E4
:106A80002747E158C1EB811104EB810141F2264611
:106A900041F22F4201F6A47104F55570002301253F
:106AA0008842E355A355A55405D0FC2202B0BDE8A9
:106AB000F0410CF0B5BF02B0BDE8F08141F22842D0
:106AC000A25C002A7FF473AF41F22642A25C002A46
:106AD0007FF46DAF41F22742A25C002A7FF467AFDA
:106AE00041F22E42A25C002A7FF461AF41F22F42B4
:106AF000A25C002A7FF45BAF002B7FF458AF41F219
:106B0000E8334FF43572E55802FB05F202F58A6866
:106B1000A04408F104064FF0FF33B768B360D8F81B
:106B200004C02244614608E0531893F8023613B1BA
:106B3000BEF1010F12D18C4510D0481C48D4D0288A
:106B400048DD00218E460123134493F80236002BC2
:106B5000EAD1531893F80236002BECD004F18002EE
:106B60003046FDF783FAD8ED016ADFED3A7AF8EEA8
:106B7000E66A86EEA77A27EE277AB5EEC07AF1EEBE
:106B800010FA5AD9B4EEE77AF1EE10FA2BDB4FF493
:106B9000357303FB0543B3F800364FF4357202FB3F
:106BA0000542C2F85834B368002B02DB3046FDF7CB
:106BB00049F9002FFFF6FBAE3046FDF743F94FF4DD
:106BC000357303FB0545D5F85434C5F85C34EEE65F
:106BD000D021BEE7D0B35318D02893F802E633D0C3
:106BE0008B1C0146B0E7BDEEC76A4FF4B57316EED5
:106BF000102A03FB052304EB43021346B2F860247A
:106C0000B3F8623407EE902A06EE903AB8EEC66A00
:106C1000F8EE677AF8EE666A37EE467A76EEE76A5D
:106C2000B6EE006AE7EE267A77EE867AFCEEE77A31
:106C3000CDED017ABDF80430AFE74FF4357303FBB7
:106C40000543B3F86034A8E7014682E7014686466B
:106C5000012379E700005043FE2843D0431E03F090
:106C6000FE03FE2B22D0D12B22DCA92B22DC872B8A
:106C700022DC692B22DC512B22DC3D2B22DC2B2B4E
:106C800022DC1F2B22DC152B22DC0D2B22DC092B16
:106C900022DC052B22DC032B22DC012BD4BF0023BA
:106CA0000123C2074CBF581CD84370470F23F8E795
:106CB0000E23F6E70D23F4E70C23F2E70B23F0E7AE
:106CC0000A23EEE70923ECE70823EAE70723E8E7CE
:106CD0000623E6E70523E4E70423E2E70323E0E7EE
:106CE0000223DEE76FF00F00704700BF2DE9F04F81
:106CF0002DED028B05468DB04022002140300FF073
:106D00001DFAFF2385F8793085F87A304FF4D17277
:106D1000002105F18C000FF011FAD122002105F2BB
:106D20002E200FF00BFA2022002105F54D700FF0F8
:106D300005FA4FF0FF32F04BC5F8882000244FF0E1
:106D4000010834224FF07A504FF07D51C5F80033DE
:106D5000DFF8AC93C5F808039C230027C5F80C1393
:106D600085F82E82214685F83083C5F88040C5F825
:106D70008440C5F82443C5F82843C5F82C4385F85A
:106D8000314385F8324385F83343C5F81823C5F8F5
:106D90001023C5F81C33C5F81433D122C5F8049369
:106DA000C5F8207305F555700FF0C8F9214605F5B3
:106DB000866020220FF0C2F9264685F82C84C5F89B
:106DC000284485F82D4405F57B6805F58C644FF45F
:106DD000D172002120460FF0B1F9D122002104F533
:106DE000D1700FF0ABF92022002104F52A700FF0CA
:106DF000A5F94FF0FF3A012134229C23DFF8F8C2B5
:106E0000C4F878924FF07A5E4FF07D50C4F89472D7
:106E1000C4F89862C4F89C62C4F8A06284F8A562C1
:106E200084F8A66284F8A76284F8A412C4F874C235
:106E3000C4F88C22C4F88422C4F89032C4F8883292
:106E4000C4F87CE2C4F8800244F80C6C44F8086C86
:106E500084F8A21144F804AC04F535744445B6D165
:106E600005F59C53143305F6A47B5E460893002772
:106E70009846D122002130460FF060F906F1DC007F
:106E8000202200210FF05AF90123C6F8D47086F8A9
:106E9000D97086F8D830FC3646454FF00004E8D16A
:106EA00041F2D4329FED958AAC5005F59E534FF0D8
:106EB000FF32DA611A625A6283ED068A4022214665
:106EC00028460FF03BF941F2E83705F5A15305F5E7
:106ED000A050009341F2943A4FF0FF3341F2104931
:106EE00085F839300146EC5105F59F5685F83A3062
:106EF00005F5A3524FF0FF3386ED078A41F2EC38D7
:106F000080ED008A80ED018A41F2F03C81ED028A39
:106F100041F21D4EC5F8504441F2144745F80A406D
:106F200041F2184082ED058A41F21E4145F80930D0
:106F300041F22446009B45F8084041F22E4241F2BE
:106F40002F4941F21C4A45F80C4041F23C481C7064
:106F500005F5A25C05F80E4041F2264305F80A400B
:106F600041F2284EEC5141F2274A2C5041F225477C
:106F70006C5441F22140AC5541F22241AC5441F2F3
:106F80001F4605F80940DFF87C9145F80840CCF829
:106F90000040EC5405F80E4005F80A40EC552C541E
:106FA0006C54AC55D9F800300A9341F2234241F2B7
:106FB000F83C41F2F43E41F25C460A9FD9F80030B9
:106FC000AC5405F5A35041F2844145F80C700B9385
:106FD00045F80E7041F27C42AC5141F28B4380ED9A
:106FE000068AFF2068500B99A95041F28A4AEC5456
:106FF00041F2884941F2294841F22A4C41F22B4E94
:1070000041F22C4741F22D4641F2944041F289432E
:1070100041F29841EC5441F2714205F80A4041F2C4
:107020006C4305F8094005F8084005F80C4005F8E0
:107030000E40EC55AC552C5041F268406C5441F276
:107040008D4AAC5441F28E49EC5041F28F482C509D
:1070500041F2904C41F2914005F80A4005F8094090
:1070600041F2304A05F8084005F80C402C5441F232
:10707000924005F5A2572C5441F2324105F80A40DE
:1070800041F2334241F2314AB84605F5A15341F28B
:10709000644605F80A40BE466C5405F5A35CAC5442
:1070A000DFF8649083ED058A05F5A5504FF0FF33B6
:1070B0008CED008A2222AB51214687ED028A1830DE
:1070C0008EED038AC8F804900FF038F805F5A65045
:1070D0001A30D12221460FF031F805F59C5305F501
:1070E0009D501833049300F11703039300F11B0321
:1070F0000593C31D06930BE00000A04000000000B4
:10710000CDCC4C3E80B2FF1FCDCCCC3DCDCC4C3E47
:1071100000F10B0307930346133305F5A4580093BE
:1071200000F11F034FF0050C01935FED088A88F80A
:1071300000C005F59E5300F10F0A05F585572E4650
:10714000029309954FF4D172002106F58C600EF080
:10715000F5FFD122002106F202600EF0EFFF20229F
:10716000002106F5E1600EF0E9FF06F2D46E4FF063
:10717000010806F5DB604FF0FF35DFF810C1C6F8F7
:107180005444C6F8584486F80286C6F85C54342144
:10719000CEF800C09C22C0ED008A06F2DC6E06F537
:1071A000DC60C6F8EC16C6F8E416C6F8F026C6F899
:1071B000E8264FF07A5C06F2F4624FF07D514FF012
:1071C0000009CEF800C0016082ED008A4946D12254
:1071D00086F80487C6F8F846C6F8FC46C6F80047A5
:1071E00086F8054786F8064786F8074758460EF0A2
:1071F000A5FF2022A7F1200049460EF09FFF049B27
:1072000007F8248C4FF07E5247F8284C07F8234C9F
:1072100043F8042B0493029B43F8045F0293039BFF
:1072200003F8014F0393059B03F8014F0593069B59
:1072300003F8014F0693079B03F8014F0793009B48
:107240000AF8014F03F8014F0093019B03F8014F27
:107250000193089B0BF1FC0B9B4506F5357607F176
:10726000FC077FF46FAF099D41F2704141F28C42FF
:1072700041F29343284605F8018005F8029005F88D
:1072800003900DB0BDEC028BBDE8F08F0000A04074
:107290002DE9F04F2DED068B8FB04FF4357E9DF824
:1072A0008040DDF878B007949DF88440DDF87CA03C
:1072B00002940EFB0BFE9DF8884003940EF58A683D
:1072C0009DF88C4008941D469DF8904009940AEB67
:1072D00008039DF8944004930F460433D6449DF868
:1072E00098C00A940EF58C619DF8A0400593EB1BA5
:1072F0009DF89C600B94814606910AEE103A08EEC8
:10730000102ABCF1000F00F0A7810BF59E630AEB79
:1073100083035B68002BC0F29F81034407EE903A21
:1073200006EE905AF8EEE77AB6EE007A77EE877AB4
:10733000F8EEE66A06EE107AFDEEE77A76EE876AF8
:10734000F8EEC68A1AEE103A38EE877A17EE902ACF
:1073500017EE900AFDEEE67A202B17EE903AFDEE3E
:10736000C77A4FF0770E17EE901ACDF800E040F391
:10737000C183FBF7CDFC002E00F088800AF5A153F5
:10738000D3ED057AF5EEC07AF1EE10FA7EDD41F22A
:10739000E8334FF435725AF8033002FB03A30AF5C1
:1073A000A252D3F8EC16D3F8F036D2ED046A07EE09
:1073B000103A07EE901AB8EEC77AF8EEE77A0AF5B7
:1073C000A25237EE677AD2ED059AE6EE877AF7EEAB
:1073D000006AFDEEE77A07EE105A17EE903ACF2BCF
:1073E000D4BF23EAE373D023F4EEE69A4B44F1EEE4
:1073F00010FA07EE903AF8EEC7AA00F1E586F0EE33
:10740000669AF8EEE77AB6EE009A77EE897A3AEE67
:10741000895AFDEEE77A78EE895A17EE902A17EE30
:10742000900AFDEEC57A772617EE903AFDEEE57AE2
:10743000009617EE901AFBF739FC78EEEA7AB0EE78
:107440006A7AA7EEA97A009607EE909AB8EEE76AF4
:1074500077EE097AF8EEC85AFDEEE77A75EE895AAA
:10746000F8EEE77A36EE097A77EE897AFDEEE56A8C
:10747000FDEEE77ABDEEC77A16EE902A17EE100AF7
:1074800017EE903A17EE901AFBF710FC029B002BB8
:1074900040F07781039B002B40F08682079B002BF6
:1074A00040F00B81B8EECA9A07EE909A069E9FEDC7
:1074B000C61AC2489FEDC20A0B9CB8EEE74A49467D
:1074C00009F1D00EF6EE004AF7EE001A338807EE07
:1074D000103A36F8023F07EE903AB8EEC77AF8EE67
:1074E000E77AF0EE616AE7EE416A0131B0EE617A67
:1074F000A7EEC17AF0EE685A74EE247AE7EE095AE4
:10750000B0EE686A07EE101AA6EE896AB8EEC74AAE
:10751000BDEEE77A36EE246A17EE108AB8F1FF0F57
:10752000BDEEC62A75EEA45A34EE247A07D812EEC0
:10753000103A3F2B9CBF00EB032303F80840FDEEFD
:10754000C76A16EE902AFDEEE56AFF2A16EE90CA8B
:1075500005D8BCF13F0F9CBF00EB0C239C5477EE89
:10756000676A35EEC65AF0EEE63AF0EEC50AF4EE7A
:10757000E03AF1EE10FA74DBF4EEC03AF1EE10FAF4
:1075800023D4F4EEC77AF1EE10FA40F3948077EE4C
:10759000C76A36EE655A1346B0EE656A42469A42AD
:1075A000C5EE267A11DDFF2B0AD8BDEEC67A17EE9E
:1075B00010CABCF13F0F00EB0C2C98BF0CF8034035
:1075C0000133934236EE276AEDD18E457FF47EAFCC
:1075D0000A9BC3B3049B5B6841F2E83209EB0301E9
:1075E00007EE901A5AF80220CF2BF8EEE77AC2EB9A
:1075F000821206EE905AB6EE007A0AEB8202D4BFEF
:1076000023EAE373D023134477EE877AF8EEE66A31
:10761000FDEEE77A76EE876A93F8A43F17EE902A9C
:1076200017EE900A38EE877A6624FDEEE67A002B94
:1076300000F0CC8017EE903AFDEEC77A009417EE7A
:10764000901AFBF733FB089B002B40F0CC800FB067
:10765000BDEC068BBDE8F08F07EE907AF8EEE78A76
:1076600089E6B4EEE56AF1EE10FA21DD634636EE06
:10767000655A12EE10CA77EEC76AF0EE477A9C455B
:1076800086EE857AA1DDFDEEE76A77EE877A16EE63
:10769000902AFF2A05D800EB03283F2B98BF08F853
:1076A000024001336345EED18E457FF40FAF8FE783
:1076B00012EE103AE3E7434671E7099B002B40F0D6
:1076C0009C81B8EECA9A059BDFED3F6A93ED017A83
:1076D000049B4FF4357202FB0BA2B8EEC77AF7EEAB
:1076E000007AE7EE667AD2F854145B680A444B4499
:1076F000B0EE687AA7EE897A92F8022607EE903A01
:10770000B8EEE7AA002A00F0B98107EE909AF8EEE9
:10771000C85AF6EE009A75EEA95AB8EEE76A37EE47
:10772000297AFDEEE57A36EE296ABDEEC77A17EEC4
:10773000902AFDEEC67A662617EE103A17EE101A5A
:1077400017EE900A0096FBF7B1FA07EE105A7AEEA0
:10775000297AB8EEC77AFDEEE77A37EE297A78EE25
:10776000A96A17EE902A17EE900AFDEEC77A0096E6
:1077700017EE903AFDEEE67A17EE901AFBF796FABE
:1077800092E64FF4357303FB0BA3D3F8E816D3F856
:10779000E42609EB010803994A44002940F00F81CF
:1077A000D3F8FC36022B00F00D85032B00F0EA82A3
:1077B000012B7FF473AE88263BE200BF3070FF1FC1
:1077C000ACC52737000050438000803717EE903A51
:1077D000FDEEC77A009417EE901AFBF799FA089B12
:1077E000002B3FF434AF4FF4357303FB0BA34FF082
:1077F0006608D3F8EC66D3F8F046CDF800804E4426
:10780000324630462B463946FBF782FAFF2E4C446F
:107810000ED83F2D40F203826A1E3F2A40F2F681C5
:10782000AA1E3F2A40F2E981EA1E3F2A40F2DF8188
:10783000731EFF2B0AD83F2D40F2D081691E3F29CD
:1078400040F2C381A91E3F2940F2B981B31EFF2B2C
:1078500006D83F2D40F2AA81691E3F2940F2A0813F
:10786000033EFF2E02D83F2D40F294816626394612
:1078700000962B4622462046FBF74AFAFF2C0ED8EC
:107880003F2D40F27F816A1E3F2A40F27281AA1E7C
:107890003F2A40F26581EA1E3F2A40F25B81631C69
:1078A000FF2B0AD83F2D40F24C81691E3F2940F240
:1078B0003F81A91E3F2940F23581A31CFF2B06D82A
:1078C0003F2D40F22681691E3F2940F21C8103347E
:1078D000FF2C02D83F2D40F2108141F231431AF8BB
:1078E0000330002B7FF4B3AE4FF4357303FB0BAAC8
:1078F0005FED4B6ADAF8F8361FED4E5A07EE903A14
:10790000F8EEE77AB7EE007AA7EEE67A0AF2F46AC2
:10791000662407EE909AF0EE686AB8EEE76AE7EE42
:10792000096A9AED007A0094F0EE467AE7EE057A5D
:10793000F8EEC85AF6EE009A75EEA95AB0EE678ACC
:1079400036EE296AFDEEE57A76EEA96A17EE902A00
:10795000FDEEE66AFDEEC67A16EE903A16EE901A45
:1079600017EE900AFBF7D4F907EE905AF8EEE76AA3
:1079700038EE297A76EEA97A38EEA93AFDEEE77A62
:10798000BDEEC77A17EE903AFDEEC37A17EE102AD5
:1079900017EE100A17EE901A1E940FB0BDEC068B6E
:1079A000BDE8F04FFBF7B4B94FF4357303FB0BA3FD
:1079B000D3F8E426D3F8E8364A4409EB03084FF439
:1079C000357303FB0BA3D3F8FC36022B00F0548372
:1079D000032B00F04D83012B00F02A8166262B46F5
:1079E000104639460096FBF761F900962B46424651
:1079F00040463946FBF75AF950E5059B5FED8E6A24
:107A00005B680293DDED027A049BF8EEE77AB7EE4D
:107A1000007AA7EEE67A5B68B8EECA9AF0EE686A7A
:107A2000E7EE096A4B4407EE903AB0EE667AF8EE5C
:107A3000E77AF6EE006A37EE267A77EEA67AF0EE6F
:107A4000006A77EE265A37EE667A37EEA66ABDEE02
:107A5000C77A77EEE67A17EE101AFDEEE56ABDEE0C
:107A6000C67AFDEEE77A8823009317EE102A16EE09
:107A7000903A17EE900AFBF719F924E607EE909A70
:107A8000F8EEC85AF6EE009A75EEA95AB8EEE76A13
:107A900037EE297AFDEEE57A36EE296ABDEEC77A31
:107AA00017EE902AFDEEC67A662617EE103A17EE0C
:107AB000101A17EE900A0096FBF72AF907EE105AF3
:107AC0007AEE297AB8EEC77AFDEEE77A37EE297AB0
:107AD00078EEA96A17EE902A17EE900AFDEEC77AA3
:107AE000009617EE903AFDEEE67A17EE901AFBF745
:107AF0000FF9D9E4FBF7DAF83DE4A14B03EB0523DA
:107B000066221A55E9E69E4A02EB01226621D1540B
:107B1000DDE69B4A02EB05226621D154691E3F290E
:107B2000F1D9D4E6964A02EB01226621D154C4E68B
:107B3000934A02EB01226621D154A91E3F29F1D9B3
:107B4000BBE68F4A02EB05226621D154691E3F290C
:107B5000EED9AEE68A4B03EB022366221A559EE667
:107B6000874B03EB022366221A55EA1E3F2AF1D9FE
:107B700095E6834B03EB022366221A55AA1E3F2A81
:107B8000EED988E67E4B6A1E03EB05233F2A1E557D
:107B9000EFD97CE67A4B03EB052366229A5565E61E
:107BA000774A02EB01226621D15459E6744A02EB6E
:107BB00005226621D154691E3F29F1D950E6704A49
:107BC00002EB01226621D15440E66D4A02EB01220C
:107BD0006621D154A91E3F29F1D937E6684A02EB44
:107BE00005226621D154691E3F29EED92AE6644B4D
:107BF00003EB022366229A551AE6614B03EB02233C
:107C000066229A55EA1E3F2AF1D911E65C4B03EB36
:107C1000022366229A55AA1E3F2AEED904E6584B43
:107C20006A1E03EB05233F2A03F80680EED9F7E529
:107C30006626FF2A1AD83F2D03D8514B03EB0523A4
:107C40009E54691E3F2903D84D4B03EB01239E54DC
:107C5000A91E3F2903D84A4B03EB01239E54E91E7A
:107C60003F2903D8464B03EB01239E54531EFF2BA1
:107C700013D83F2D03D8424901EB0521CE54681E8D
:107C80003F2803D83E4901EB0021CE54A81E3F28CF
:107C900003D83B4901EB0021CE54931EFF2B0CD897
:107CA0003F2D03D8364901EB0521CE54681E3F28ED
:107CB00003D8334901EB0021CE54D11EFF2905D84A
:107CC0003F2D03D82E4B03EB05235E54B8F1FF0F75
:107CD0001ED83F2F04D82A4B03EB072303F8086074
:107CE000791C3F2904D8264B03EB012303F80860D5
:107CF000B91C3F2904D8224B03EB012303F8086089
:107D0000F91C3F2904D81E4B03EB012303F808603C
:107D100008F10103FF2B13D83F2F03D8184901EBBB
:107D20000721CE54781C3F2803D8154901EB0021C8
:107D3000CE54B81C3F2803D8114901EB0021CE5482
:107D400008F10203FF2B0CD83F2F03D80C4901EB9D
:107D50000721CE54781C3F2803D8094901EB0021A4
:107D6000CE5408F10301FF2905D83F2F03D8044B57
:107D700003EB07235E54039B002B3FF48FAB2EE6EF
:107D80003070FF1F8826FF2A1AD83F2F03D8B94B1F
:107D900003EB07239E54791C3F2903D8B54B03EB13
:107DA00001239E54B91C3F2903D8B24B03EB012396
:107DB0009E54F91C3F2903D8AE4B03EB01239E547C
:107DC000511EFF2913D83F2F03D8AA4B03EB0723DB
:107DD0005E54781C3F2803D8A64B03EB00235E5467
:107DE000B81C3F2803D8A34B03EB00235E54901E1E
:107DF000FF280ED83F2F03D89E4B03EB07231E54BA
:107E000007F1010EBEF13F0F03D89A4B03EB0E238F
:107E10001E54D31EFF2B1C460C9305D83F2F03D8AE
:107E2000944B03EB07231E55B8F1FF0F24D83F2DC9
:107E300004D8904B03EB052303F8086005F1FF3EDF
:107E4000BEF13F0F04D88B4B03EB0E2303F8086001
:107E5000A5F1020EBEF13F0F04D8864B03EB0E23B3
:107E600003F80860A5F1030EBEF13F0F04D8814B63
:107E700003EB0E2303F8086008F10103FF2B1DD864
:107E80003F2D05D8DFF8ECE10EEB052E0EF8036070
:107E900005F1FF3CBCF13F0F05D8DFF8D8E10EEB50
:107EA0000C2E0EF80360A5F1020CBCF13F0F05D8B3
:107EB000DFF8C0E10EEB0C2E0EF8036008F10204AF
:107EC000FF2C029413D83F2D05D8DFF8A8E10EEB64
:107ED000052E0EF8046005F1FF3CBCF13F0F06D8FB
:107EE000DFF890E1029C0EEB0C2E0EF8046008F116
:107EF0000304FF2C0D9407D83F2D05D8DFF874E15B
:107F00000EEB052E0EF80460FF2A28D83F2D05D869
:107F1000DFF860E10EEB052E0EF8026005F1FF3C84
:107F2000BCF13F0F05D8DFF84CE10EEB0C2E0EF83C
:107F30000260A5F1020CBCF13F0F05D8DFF834E177
:107F40000EEB0C2E0EF80260A5F1030CBCF13F0FF6
:107F500005D8DFF820E10EEB0C2E0EF80260FF29A9
:107F60001DD83F2D05D8DFF80CE10EEB052E0EF8DD
:107F7000016005F1FF3CBCF13F0F05D8DFF8F4E0EC
:107F80000EEB0C2E0EF80160A5F1020CBCF13F0FB8
:107F900005D8DFF8E0E00EEB0C2E0EF80160FF28AC
:107FA0000ED83F2D03D8334901EB05210E5405F1BE
:107FB000FF3EBEF13F0F03D82E4901EB0E210E54B8
:107FC0000C98FF2805D83F2D03D82A4901EB05213D
:107FD0000E54B8F1FF0F1ED83F2F04D8254901EBEE
:107FE000072101F80860781C3F2804D8214901EBDB
:107FF000002101F80860B81C3F2804D81D4901EB96
:10800000002101F80860F81C3F2804D8194901EB49
:10801000002101F80860FF2B13D83F2F03D8154922
:1080200001EB0721CE54781C3F2803D8114901EBFE
:108030000021CE54B81C3F2803D80E4901EB002183
:10804000CE54029BFF2B0ED83F2F04D81946094B64
:1080500003EB07235E54791C3F2904D8054B03EB3F
:10806000012302995E540D99FF293FF684AE7CE608
:10807000662688E63070FF1F6626FF2A1AD83F2F33
:1080800003D8574B03EB07239E54791C3F2903D891
:10809000534B03EB01239E54B91C3F2903D8504B8B
:1080A00003EB01239E54F91C3F2903D84C4B03EBEF
:1080B00001239E54531EFF2B13D83F2F03D848494A
:1080C00001EB0721CE54781C3F2803D8444901EB2B
:1080D0000021CE54B81C3F2803D8414901EB0021B0
:1080E000CE54931EFF2B0CD83F2F03D83C4901EBF5
:1080F0000721CE54781C3F2803D8394901EB0021D1
:10810000CE54D11EFF2905D83F2F03D8344B03EBA3
:1081100007235E54B8F1FF0F1ED83F2D04D8304B13
:1081200003EB052303F80860691E3F2904D82C4B94
:1081300003EB012303F80860A91E3F2904D8284B4C
:1081400003EB012303F80860E91E3F2904D8244B00
:1081500003EB012303F8086008F10103FF2B13D898
:108160003F2D03D81E4901EB0521CE54681E3F2840
:1081700003D81B4901EB0021CE54A81E3F2803D889
:10818000174901EB0021CE5408F10203FF2B0CD854
:108190003F2D03D8124901EB0521CE54681E3F281C
:1081A00003D80F4901EB0021CE5408F10301FF2948
:1081B0003FF6E1AD3F2D3FF6DEAD094B03EB052366
:1081C0005E54D8E5882658E7F5EEC09ADFED056ADB
:1081D000F1EE10FAD8BFF0EE669AFFF712B900BFC1
:1081E0003070FF1F000000002DE9F04F2DED028BD5
:1081F000BC4C9FEDBD8ADFEDBD8A89B001F5A35768
:108200000391043701F59E5A01F2D46826460125F0
:108210004FF000093B684B4500F0348198F833E09B
:1082200098F83030CEF1630E0BB9CEF1000E9AF80B
:108230000030AF4A002B14BF00217721106807904F
:10824000BEF1000F4FF0010B40F341812B228DF85E
:108250001C20BEF1000FB8BFCEF1000EBEF1090F19
:1082600040F33D81A34A4FEAEE7082FB0EC2C0EBA1
:10827000A20230328DF81D209E4A019382FB0E32FD
:10828000C0EBA20202EB8202AEEB420E2172002290
:108290000EF1300E01214FF480708DF81EE0E16286
:1082A0004FF0400E0221A262226122756275A26126
:1082B000E26120622B2207A86560C4F824E0E16037
:1082C00022600292FAF7EEFD019BC3B18A4B029A3B
:1082D0001B6813F0010F12D1884B1B680693069B95
:1082E000C3F30803B3F5807F09D92021EE2307A843
:1082F000326075608DF81C103372FAF7D3FDD8ED3B
:10830000007A9AF80030BBF1000F00F03A81002BA0
:108310000CBF4FF0000E4FF0770EF4EEC87AF1EE7E
:1083200010FA40F1AA80F5EEC07AF1EE10FA40F3AF
:108330002E81B6EE007AA7EEA87A714B6420FDEE8E
:10834000C77A17EE902A83FB0231D317C3EB611172
:1083500000FB11204FF0010C84F808E04FF4807E00
:108360000023C4F82CC0C4F820E04FF0400C4FF0BC
:10837000020E0929A362236123756375A361E3617A
:10838000C4F824C0C4F80CE03BDC5A4A8DF8153020
:1083900082FB00E24FEAE07ECEEBA20202EB820E0D
:1083A000A0EB4E00303100F1300E30328DF8141059
:1083B00007A815218DF81E308DF81DE08DF81C20C2
:1083C00031607560FAF76EFD0B234E4886E8280091
:1083D000FAF768FD062305A886E82800FAF762FD8B
:1083E00009F10109B9F1040F0AF1010A05F10B05C0
:1083F00008F535787FF40EAF09B0BDEC028BBDE80F
:10840000F08F632900F38480DFF8E8C08DF81E3018
:108410008CFB01EB4FEAE17ECEEBAB0E8CFB00BC9C
:10842000C017C0EBAC0C38488DF8153080FB02B09B
:108430000EEB8E0ED217A1EB4E0EC2EBA0120CF17A
:10844000300C0EF1300E3032152105A88DF814C015
:108450008DF81DE08DF81C2031607560FAF722FD63
:108460001123284886E82800FAF71CFD0C2307A8EA
:1084700086E82800FAF716FDB2E7002040F2E7315F
:10848000224A67E7039B03F5A35393ED007AF2EECC
:108490000E7A67EE277AFDEEE77A17EE903ADB0761
:1084A0007FF5BCAE98F833E098F83030CEF1630E2B
:1084B000002B7CD09AF8003063B90D4ABEF1000F52
:1084C000106807909B464FF077013FF7BFAE6AD127
:1084D0007046D1E6D8ED007A4FF0770E1DE74FEAEF
:1084E000EE70C9E6782AFF1F00C079440000C84238
:1084F0000CAD0100676666665029FF1F80B2FF1F42
:108500001F85EB51F8B00100D34D62103C8601008D
:1085100028488DF81F3080FB02E04FEAE27CDFF84C
:108520009CE0CCEBA0138EFB030B8EFB010ED81747
:10853000C0EBAB000190204880FB020201984FEA9B
:10854000E17B00EB8000CBEBAE0ECCEB2232A3EB59
:1085500040000EEB8E0E3032D2B23030A1EB4E0125
:10856000C0B23031302A8DF81C208DF81D008DF8F6
:108570001E1010D0152307A884E82800FAF792FCF3
:108580002EE7002B3FF42CAF4FF0770EC5E600200E
:1085900001460246DEE6202330288DF81C3008BF55
:1085A0008DF81D30E6E72D228DF81C2051E6CEF126
:1085B000000E7FE7D34D6210AD8BDB6867666666A1
:1085C0000B69002B00DA7047F0B587B000242D4A04
:1085D00003940F2102A80294049405940DF0FCFD6D
:1085E000FF2300939E222A2314216220FAF75EFBC8
:1085F0002C236122122160200094FAF757FB1323E9
:10860000122160200094A022FAF750FB1E49234655
:10861000204603F594521F3203F58073B3F5D85FFB
:108620008854F6D10023184603F5955203F580735C
:10863000B3F5D85F88544FF00004F5D100942C2393
:10864000A0222B216020FAF731FB104B4FF48072EF
:108650004FF0400E1F211A6202A80122FF270226B6
:1086600080251C759C61DC611C72C3F824E05F7579
:10867000DE621D6059609A62DA601A61FAF712FCD4
:1086800007B0F0BDFCB001003070FF1F782AFF1F5B
:108690002DE9F04F97489BB0894600F58045772437
:1086A000A0F5807313F8011FFF2918BF1C709842B2
:1086B000F8D100F580708542F2D1002A00F0F780F1
:1086C00041F2144241F2184359F8022059F803309C
:1086D00041328020413300218DF824208DF825007F
:1086E0008DF826308DF827109A244FF066089922CD
:1086F00067209B2765264FF0FF0A0025CDF800A0D4
:108700002A231421FAF7D2FA424630462C231221AA
:108710000095FAF7CBFA3A4630461323122100951A
:10872000FAF7C4FA20463A462C2312210095724CDF
:10873000FAF7BCFA3A4630462C232B210095FAF77B
:10874000B5FA0126022180221F234FF0400B4FF47F
:10875000807809A884F815A0E16284E80C00C4F8C8
:1087600024B02575A561E5612572C4F82080A66254
:10877000E6602661FAF796FBDFF880C1E662BCE8A6
:108780000F000DF12C0EAEE80F00BCE80F00AEE8B4
:108790000F00BCE80F00AEE80F009CE8070009F5E9
:1087A000A0531F461E3325608EE8070065600693C0
:1087B0003B1DC4F824B0AA46A946C4F82080E56051
:1087C00025612575A561E561A66207930DF12C0B66
:1087D000069B84F808901B7843FA0AF3FF22DB0714
:1087E000F3EE047A627560D5079B93ED007A67EE2D
:1087F000277A1546FDEEE77A17EE903A13F001035B
:1088000003D13D491D464B750A72DBF808300493CD
:1088100018460DF035FDDBF80030DBF804600095FC
:1088200000EB400003EB40051F462A461846314640
:1088300006F108030597013F0397FAF737FA039B00
:10884000CDF8009006F1FF3806F1090701351A4608
:10885000184641463B46FAF729FA2A46434641461E
:108860000398CDF80090FAF721FA41462A462846A7
:108870003B46CDF80090FAF719FA2A460398CDF84E
:1088800000903B463946FAF711FA059B04980AF125
:10889000010A84E84800FAF705FBBAF1050F0BF16D
:1088A0000C0B95D11BB0BDE8F08F1546ADE741F23A
:1088B0001843632659F803308DF82B206524612076
:1088C000202241336C2572218DF824608DF82640DA
:1088D0008DF827008DF829208DF82A308DF8255045
:1088E0008DF82810B1244FF04F08B0225020B22745
:1088F0004E2600E72F71FF1F782AFF1F10AD0100E1
:108900002DE9F04F2DED028B91F83530ABB0002BF7
:1089100040F0CD8091F836308A46002B40F05E81E1
:1089200091F83730002B40F0B281CB6B002B55D043
:10893000A34A4FF0FF3102F580700023D15003F5B8
:108940008073B3F5804F4FF0FF34F7D10432824289
:10895000F3D1FF230093C2222C2313213D200025B5
:10896000FAF7A4F93C2210462D2312210095FAF7BC
:108970009DF912231946C3223C200095FAF796F977
:10898000C32210462D2312210095FAF78FF92D23CB
:108990001946C3223C200095FAF788F9894B8A4F83
:1089A0001B681893189A3D604FF48070C2F3080258
:1089B0000123402182427D60BD61FD617C753D7275
:1089C00038627962FB623B75BB62FB603B6100F21F
:1089D000A3802BB0BDEC028BBDE8F08F91F8343052
:1089E000002B40F0B08041F2B843CC5C002C40F04A
:1089F000B68141F28943CB5C002B40F02D8241F2DD
:108A00008C43CB5C002B40F00B8241F271438346D8
:108A1000CB5C63B16B4A41F2F43113681493149B3D
:108A20005AF801105B1AB3F5FA7F00F2C68141F2E1
:108A3000EC335AF80330002B00F07A845A1E012AD6
:108A400040F24C8341F21C431AF80320002A40F004
:108A5000B28041F21D431AF80330002B40F0AB8086
:108A600041F2EC335AF80330032B00F0A68541F2B3
:108A70008B431AF80330002BABD0534B00220AF57E
:108A8000A45001214FF480764025FF241830DA608D
:108A90001A611E625D625C75D9621975996219600E
:108AA00059609A61DA611A72FAF7FCF991E7444A5F
:108AB0004FF0FF3402F580700023D45003F580732B
:108AC000B3F5804F4FF0FF31F7D104328242F3D13A
:108AD0003C4A3D4B12681592159859754FF48075B4
:108AE000C0F30800012100224024A8421D625C62FC
:108AF000D96219759962D96019611A605A609A61D0
:108B0000DA611A727FF665AF7F211F222F4883E852
:108B10000600FAF7C7F95CE77F241A232C487B602C
:108B20003C60FAF7BFF9DAF83C002A4B3C60A842F7
:108B300008BF184624237B60FAF7B4F92BB0BDECCC
:108B4000028BBDE8F08F1E4A4FF0FF3102F58070B6
:108B50000023D15003F58073B3F5804F4FF0FF34FD
:108B6000F7D104328242F3D1164A1B4B1268199294
:108B70000FCB1AAF87E80F00199E134D2AAAC6F330
:108B8000C11302EB83034FF4807253F8400C6C75F1
:108B9000002301212A6240240222EB602B616C62D7
:108BA000E962A9622B75AB61EB612B722A606A6086
:108BB000FAF778F90DE751465846FFF769FD4FE798
:108BC0003070FF1F80B2FF1F782AFF1F84B10100A1
:108BD000C4B1010000B101005CAD0100984A4FF042
:108BE000FF3102F580700023D15003F58073B3F597
:108BF000804F4FF0FF34F7D104328242F3D1FF238C
:108C00000093C2222C2313213D200025FAF74EF8B1
:108C10003C2210462D2312210095FAF747F8122323
:108C20001946C3223C200095FAF740F8C3221046AB
:108C30002D2312210095FAF739F82D231946C32266
:108C40003C200095FAF732F87E4A7F4B1268169264
:108C500016991D604FF48076C1F30801012240206F
:108C6000B1425D609D61DD615C751D721E6258627E
:108C7000DA621A759A62DA601A617FF6AAAE7F210B
:108C80001F22724883E80600FAF70CF9A1E66C4A45
:108C90004FF0FF3102F580700023D15003F580734F
:108CA000B3F5804F4FF0FF34F7D104328242F3D155
:108CB000FF230093C2222C2313213D20F9F7F6FF56
:108CC00000263C22104600962D231221F9F7EEFFD4
:108CD000122319460096C3223C20F9F7E7FFC3226E
:108CE000104600962D231221F9F7E0FF2D23564D53
:108CF00000961946C3223C20F9F7D8FF7F270123AD
:108D00004FF4807E40211B2251486C75C5F820E04D
:108D100069626A60EB622B75AB62EB602B61AE61DE
:108D2000EE612E722F60FAF7BDF84A4B454C2F606A
:108D30000FCB246817941AAC84E80F00179B2AAA5B
:108D4000C3F3C11302EB8303232253F8400C6A6080
:108D5000FAF7A8F82BB0BDEC028BBDE8F08F384ACB
:108D60004FF0FF3402F580700023D45003F5807378
:108D7000B3F5804F4FF0FF31F7D104328242F3D187
:108D8000314B0AF5A55000224FF4807E4027022681
:108D90007F251F24597518300121C3F820E05F6238
:108DA000DE621D605C601A759A61DA611A729962FE
:108DB000D9601961FAF776F80BE612681A9241F257
:108DC000844341F26C425AF803005AF802401A9B5D
:108DD0001C1BFDF741FF1A4A0028CBBF0025FF25C9
:108DE000FF26002602F58070002165F3070165F378
:108DF0000F2165F3174165F31F610023D15003F57F
:108E00008073B3F5804FF9D1043282420C4BEBD121
:108E1000C4F3053203EB0223C4F307141E55D8E54F
:108E2000074A4FF0FF3102F580700023D15003F55F
:108E30008073B3F5804FF9D104328242F5D1C8E591
:108E40003070FF1F80B2FF1F782AFF1FA0B1010002
:108E5000B0B101004CAD010021464FF4807286484C
:108E60000DF06CF921464FF4807284480DF066F9DC
:108E700021464FF4807282480DF060F921464FF48C
:108E8000807280480DF05AF921464FF480727E4876
:108E90000DF054F921464FF480727C480DF04EF9E4
:108EA00021464FF480727A480DF048F921464FF47C
:108EB000807278480DF042F921464FF4807276486E
:108EC0000DF03CF9754A4FF0FF3002F58074002335
:108ED000D05003F58073B3F55C5F4FF0FF31F7D1ED
:108EE0000432A242F3D16E4F6E48397200244FF41F
:108EF00080750123FF2102223D627C604025FC60D9
:108F00003C61FB62BB6279753A607D623C75BC6115
:108F1000FC61F9F7C7FF2A4621461AA83C720DF0FA
:108F20000DF99AF87130604D002B40F0F7820AF588
:108F3000A45494F800E05D495D4A6E785D485E4B4C
:108F4000BEF1020F18BF0A46002E08BF034600926A
:108F50003F215A4A1AA80DF03FF91C2302221AA8F1
:108F600087E80C00F9F79EFFAB78012B00F0C08476
:108F7000002B00F0D182524A5249022B14BF1346F3
:108F80000B46267849484A494F4A032E18BF0146E6
:108F900000911AA83F210DF01FF9022225231AA8DB
:108FA00087E80C00F9F77EFF2B7940482578404987
:108FB000052B96BF454A464B52F82330454A042DAF
:108FC00018BF014600911AA83F210DF005F92E2384
:108FD00002221AA887E80C00F9F764FF41F28443E3
:108FE0005AF80330FE2B00F08084013B03F0FE03AF
:108FF000FE2B00F0E082D12B00F3DB82A92B00F3E3
:10900000D682872B00F3D182692B00F37285512B16
:1090100000F36C853D2B00F366852B2B00F36085F8
:109020001F2B00F35A85152B00F354850D2B00F3ED
:109030004E85092B00F34885052B00F3F584032B9F
:1090400000F3EF84012BD4BF0023012301332478E4
:1090500016481749204A052C18BF014600911AA846
:109060003F210DF0B9F8022237231AA887E80C0037
:10907000F9F718FFADE400BF3070FF1F3071FF1F1C
:109080003072FF1F3073FF1F3074FF1F3075FF1FDA
:109090003076FF1F3077FF1F3078FF1F3079FF1FBA
:1090A000782AFF1FD4B10100BC14FF1F9CBF010030
:1090B00028B101002CB1010034B1010028B2010037
:1090C00050B1010048B1010044B20100A0AF01005D
:1090D00058B101005CB2010070B2010041F2E83207
:1090E000022B5AF8022000F0378400254FF4357324
:1090F00003FB02A3D3F80017002940F325840027BF
:1091000041F228431AF80330002B00F0068141F2A7
:109110002643002D00F005841AF80340002C40F08F
:109120000381264600230C9341F225431AF80330AD
:10913000002B00F0F08085F0010E0AEB020141F2F5
:10914000A833A94A11F803C002F580704FF0FF312F
:109150000023D15003F58073B3F5804FF9D1043269
:109160008242F5D141F2EC3341F2E8385AF803304B
:10917000CDF820C0022B5AF808200C98039714BF92
:1091800000217721012302900A9100920993FF2286
:10919000382300210795CDF818E005960494CDF802
:1091A00004A02E20FEF774F85AF80870BA01D11BFB
:1091B000890001F57A63534493F8DC301BBB8B487C
:1091C00041F28443C35813F0010300F030844FF0A0
:1091D000AA09D71B0AEB870707F6A3774FF02E08DB
:1091E00004E008F10108B8F1FF0F10D017F8013FB3
:1091F000002BF6D0CDF800903E2342463A2140465F
:10920000F9F754FDEDE74FF00009E2E70D9C784FC8
:1092100041F2EC3340225AF803007A624FF4807333
:10922000022201213B6290424FF00003F962B962D1
:109230003B757B75BB61FB61FA603A6107D041F217
:109240002F431AF80330002B0CBF772300232B2267
:109250003B7268483A6040237B60F9F723FE002E9A
:1092600000F089830AF5A153D3ED057AF5EEC07AB3
:10927000F1EE10FA43DD41F2E8334FF435725AF85B
:10928000033002FB03A30AF5A252D3F8EC16D3F87D
:10929000F036D2ED046A07EE103A07EE901AB8EEF7
:1092A000C77AF8EEE77A37EE677AE6EE877AFDEE70
:1092B000E77A17EE903ACF2BDCBF23EAE37300EE98
:1092C000103A0AF5A25393ED057AC8BF9FED4A0AFA
:1092D000F7EE007AB4EEE77AD8BFB8EEC00AF1EE46
:1092E00010FA00F1D0834FF47A742D20FAF774FC51
:1092F00007EE904A3820B8EEE70AFAF76DFC5146BF
:109300005846FEF771FF0AF59E5114315846FFF793
:1093100057F9FFF797BB9E460FE741F226431AF82D
:109320000340002C00F0E98285F001060024F9E6F4
:109330002D4A4FF0FF3102F580700023D15003F524
:109340008073B3F5804FF9D104328242F5D10AF52A
:109350009D5307330AF59E590D939FED284ACDF88A
:109360004CA00AF58C6309F1040957460C934FF0A1
:10937000000807F583531C330D9A1B78002B08F166
:1093800002031146109308F10D030F9308F10C032B
:1093900011F8012F119308F103030E920D910CBFE8
:1093A0004FF0AA0A4FF0220A07F6A3762E240025D2
:1093B000129311E015F0010F0F9B1099CDF800A04A
:1093C0002246204603D0119B129922462046F9F7E7
:1093D0009FFC0134FF2C15D016F8013F0135002BFE
:1093E000E8D11D46F5E700BF3070FF1FCC14FF1F0A
:1093F000782AFF1F84B201000000504380008037AC
:109400000000384208F10E0306EE903A0E9B002B46
:109410007DD0D9F80030002B79DB2E3307EE903A5F
:10942000F8EEE77AB6EE007A77EE877AF8EEE66A3B
:1094300006EE108AFDEEE77A76EE876AF8EEC64A07
:1094400017EE902A34EE877A17EE900AFDEEE67A50
:10945000772417EE903AFDEEC77A009417EE901A33
:10946000F9F724FC1FED1A5A0C9D2E24B7EE003A92
:10947000F2EE0C3A2B8807EE103AB8EEC77A35F8C0
:10948000023FF0EE436AE7EE446A0134002007EE43
:10949000903AF8EEE77AB0EE667AF0EE436AE7EEDD
:1094A000C46AB0EE450AF0EE667A06EE904AB8EE6F
:1094B000E65AF0EE640AF0EE641AE7EE230AE7EEED
:1094C000A31AB0EE451AF9F755FCFE2CD2D10C9B2D
:1094D00008F1100803F53573B8F1400F07F1FC07E8
:1094E0000C9309F104097FF444AFDDF84CA0584611
:1094F0005146FEF779FE0AF59E5114315846FFF7A2
:109500005FF841F2EC335AF80330FFF797BA07EEF1
:10951000908AF8EEE74AA5E7C14B32E52B78002B9D
:1095200041D0012B00F0E781BE4ABF49022B14BF96
:1095300013460B460AF5A454BC4E2178DFF8888305
:10954000BB4A002914BF3146414600911AA83F2169
:109550000CF042FE0A2302221AA887E80C00F9F751
:10956000A1FC9AF87130002B3FF4E3AC95F8009021
:10957000B04BB9F1020F7FF4DCAC2178DA78012925
:1095800008BF4646642302FB03330096AA4A3F21E4
:109590001AA80CF021FE13231AA8C7F800907B60CC
:1095A000F9F780FCC5E4A54BC4E70C234EE50D2379
:1095B0004CE50E234AE50F2348E5A14A002102F5B8
:1095C00080700023D15003F58073B3F5804F4FF0C6
:1095D0000004F7D104328242F3D19A4F9A48FC60DA
:1095E000FF264FF4807E40230125314625223C6131
:1095F000C7F820E07B62FD62BD627E753C75BC6190
:10960000FC613C720CF09AFD314625228F480CF02B
:1096100095FD314625228E480CF090FD31462522DD
:109620008C480CF08BFD314625228B480CF086FDD2
:109630003146252289480CF081FD31462522884893
:109640000CF07CFD3146252286480CF077FD314632
:10965000252285480CF072FD4FF0370861238348BE
:1096600087E80801F9F71EFC31462B2280480CF0F0
:1096700065FD31462B227F480CF060FD31462B22E0
:109680007D480CF05BFD31462B227C480CF056FDEA
:1096900031462B227A480CF051FD31462B22794875
:1096A0000CF04CFD31462B2277480CF047FD31463B
:1096B0002B2276480CF042FD31462B2274480CF0E8
:1096C0003DFD9123734887E80801F9F7EBFB31462C
:1096D000492271480CF032FD314649226F480CF0A6
:1096E0002DFD314649226E480CF028FD31464922B5
:1096F0006C480CF023FD314649226B480CF01EFDEE
:109700003146492269480CF019FD31464922684822
:109710000CF014FD3146492266480CF00FFD31462D
:10972000492265480CF00AFD41F2294341F22A41E1
:109730001AF80360614A624B1AF801006149C7F8E0
:109740000480A64218BF1346A0420CBF1846084624
:109750000F223A60F9F7A6FB09230AF59E580AF58D
:109760009F5928227B620AF5A053CDF830B0FD60E6
:109770003D61A3463A6208F1140809F11C0902256B
:109780000F93B3EE048ACDF840A005F108030E93C1
:109790002B1D0D93DDF830A05E460524F1EE008A06
:1097A00019E00092204604F127020E9B87F808E09A
:1097B0002946BC61FD61F9F779FA0D9B7B605AF887
:1097C000040B04F1140329343B60F9F76BFBFB2C09
:1097D00006F101067AD00F9B99ED007AD3ED007A5D
:1097E000D8F80010F5EEC07AF1EE10FAD4BF67EEAB
:1097F000287A67EE887AB142FDEEE77A4FF0FF02F1
:1098000017EE903A03F0010383F001034FF0000ECE
:10981000C7D173451CBF72464FF0FF0EC1E700BFB2
:1098200040B1010020B1010018B101009CBF01004E
:10983000E4B10100BC14FF1F08B2010004B1010033
:109840003070FF1F782AFF1F8EA7FF1F8EA8FF1FF3
:109850008EA9FF1F8EAAFF1F8EABFF1F8EACFF1FAE
:109860008EADFF1F8EAEFF1F8EAFFF1F88B20100AF
:10987000BEA7FF1FBEA8FF1FBEA9FF1FBEAAFF1FD6
:10988000BEABFF1FBEACFF1FBEADFF1FBEAEFF1FB6
:10989000BEAFFF1F90B201003CA7FF1F3CA8FF1FF7
:1098A0003CA9FF1F3CAAFF1F3CABFF1F3CACFF1FA6
:1098B0003CADFF1F3CAEFF1F3CAFFF1F6CB1010072
:1098C00060B1010078B1010028B101000C9B0BF1DF
:1098D000060B1833BBF11E0F05F10A050C937FF43C
:1098E00054AFDDF840A0FFF7C2B81023FFF7AFBBBD
:1098F000814BFFF746BB814B1CE6002D7FF411AC7A
:1099000041F22E431AF80330BBB941F22F432C46E3
:109910001AF803302E46002B7FF404AC01230C937D
:1099200002E41AF803301BB13C460126FFF7FABBEC
:109930003C4637B12E46FFF7F5BB2C462E46FFF7C7
:10994000F1BB3E46FFF7EEBBD3F8FC76002FD4BF49
:1099500000270127FFF7D4BB41F22E431AF803304A
:10996000002B7FF4C2AB41F22F431AF8035085F06D
:109970000105FFF7BBBB4CBB0C9B13B9002D3FF49B
:10998000BEAC41F2E8334FF435725AF8033002FBB3
:1099900003A303F58A6393ED010A9C682D20B8EEBA
:1099A000C00AFAF719F94FF47A73554A03FB04F326
:1099B00082FB03121A44DB17C3EBE23300EE103ACA
:1099C0003820B8EEC00AFAF707F998E441F2E83215
:1099D0004FF435735AF80220494E03FB02F30AEBA9
:1099E000030707F58C65D7F8E43635F813304FF4E4
:1099F0007A7404FB03F386FB03121A44DB17C3EBF0
:109A0000E23300EE103A2D20B8EEC00AFAF7E4F87F
:109A1000D7F8E83635F8133004FB03F386FB03125E
:109A2000C8E70223FFF712BB0323FFF70FBB01F6C2
:109A3000A3710AEB01081F464FF02E090D9413E0A5
:109A400017F0010F4FF03D034A464FF03B014846E7
:109A500010D0AA240094F9F75BF9013709F1010944
:109A6000B9F1FF0F3FF4D2AB18F8013F002BE7D15B
:109A70001F46F3E7AA2300934A463E233A2148466D
:109A8000F9F746F9E9E7DFED1F7AB4EEE77AF1EE90
:109A900010FA17DDDFED1C6A194CE7EE267A4FF459
:109AA0007A72B6EE007A77EE877AFDEEE77A17EEF5
:109AB000903A02FB03F384FB03241C44DB17C3EB43
:109AC000E43412E4002410E40423FFF7BFBA0523B2
:109AD000FFF7BCBA0623FFF7B9BA0723FFF7B6BAF8
:109AE0000823FFF7B3BA0923FFF7B0BA0A23FFF739
:109AF000ADBA0B23FFF7AABA3CB1010010B10100C7
:109B0000018000800000000000FF7F47F8B5D0F81A
:109B1000E432DE4E044618460D4650F8302F0978E0
:109B20001268B24240F0E08493F838005F6B93F81B
:109B30003B20884200F0388393F83A00884200F0D6
:109B4000338393F83EE0BEF1010F00F033834FF012
:109B5000010E97F859000EFA02F220EA020287F885
:109B6000592093F83920586B93F83C708A4200F0E2
:109B7000468493F83A208A4200F0418493F83E30BC
:109B8000012B00F04184012190F8592001FA07F3DC
:109B900022EA030380F85930D4F8E4326978184691
:109BA00050F8402F1268B24240F0998493F8480070
:109BB0005F6C93F84BC0884200F0148493F84A20FD
:109BC0008A4200F00F8493F84E20012A00F00F849F
:109BD0004FF0010E97F859000EFA0CF220EA02023B
:109BE00087F8592093F84920586C93F84C708A42B2
:109BF00000F0348493F84A208A4200F02F8493F8CE
:109C00004E30012B00F02F84012190F8592001FAE9
:109C100007F322EA030380F85930D4F8E432A97834
:109C2000184650F8502F1268B24240F0608493F802
:109C300058005F6D93F85BC0884200F0038493F88E
:109C40005A208A4200F0FE8393F85E20012A00F039
:109C5000FE834FF0010E97F859000EFA0CF220EA3D
:109C6000020287F8592093F85920586D93F85C70D8
:109C70008A4200F0DC8393F85A208A4200F0D783AE
:109C800093F85E30012B00F0D783012190F8592022
:109C900001FA07F322EA030380F85930D4F8E432DA
:109CA000E978184650F8602F1268B24240F01A84E2
:109CB00093F868005E6E93F86BE0884200F0AB8327
:109CC00093F86A208A4200F0A68393F86E20012A56
:109CD00000F0A683012796F8590007FA0EF220EA51
:109CE000020286F8592093F86920586E93F86C6048
:109CF0008A4200F06C8393F86A208A4200F06783FE
:109D000093F86E30012B00F06783012190F8592001
:109D100001FA06F322EA030380F85930D4F8E4028A
:109D20005B4E036829791B68B34240F0D6834768CD
:109D300090F808E0002940F03F83817A012900F083
:109D40003F83012397F8592003FA0EF322EA030315
:109D500087F85930D4F8E4326979184650F80C2F56
:109D60001268B24240F0CA8318691F7D002940F092
:109D70001883997D012900F01883012390F8592058
:109D8000BB4022EA030380F85930D4F8E432A979C1
:109D9000184650F8182F1268B24240F0AD83D869C7
:109DA00093F82070002940F0F08293F822100129E6
:109DB00000F0F082012390F85920BB4022EA03030F
:109DC00080F85930D4F8E422E979104650F8243F5D
:109DD0001B68B34240F08E83906A92F82C60002991
:109DE00040F0C88292F82E30012B00F0C882012189
:109DF00090F8592001FA06F322EA030380F859305B
:109E0000D4F83801297B03681B689847D4F8E4220A
:109E1000687BD2F8801092F88460002840F09F821E
:109E200092F88630012B00F09F82012091F8592092
:109E300000FA06F322EA030381F85930D4F8E42249
:109E4000A87BD2F88C1092F89060002840F07C82B9
:109E500092F89230012B00F07C82012091F8592079
:109E600000FA06F322EA030381F85930D4F8E42219
:109E7000E87B516F92F87860002840F05A8292F89F
:109E80007A30012B00F05A8204E000BFA10A0000E2
:109E9000F9090000012091F8592000FA06F322EA9E
:109EA000030381F85930D4F8E432287C93F8BC10CD
:109EB000D3F8B86093F8BEE081420CBF93F8C0209D
:109EC00093F8C120012A00F0D582012796F8591095
:109ED00007FA0EF221EA020286F8592093F8BD2013
:109EE000D3F8B81093F8BF6082420CBF93F8C0302B
:109EF00093F8C130012B00F0EA82012091F859203B
:109F000000FA06F322EA030381F85930D4F8E43268
:109F1000687C93F89C10D3F8986093F89EE0814297
:109F20000CBF93F8A02093F8A120012A00F0C8826A
:109F3000012796F8591007FA0EF221EA020286F874
:109F4000592093F89D20D3F8981093F89F6082428F
:109F50000CBF93F8A03093F8A130012B00F0AA8237
:109F6000012091F8592000FA06F322EA030381F850
:109F70005930D4F8E432A87C93F8AC10D3F8A86038
:109F800093F8AEE081420CBF93F8B02093F8B12073
:109F9000012A00F08882012796F8591007FA0EF27C
:109FA00021EA020286F8592093F8AD20D3F8A810D0
:109FB00093F8AF6082420CBF93F8B03093F8B130A1
:109FC000012B00F06A82012091F8592000FA06F373
:109FD00022EA030381F85930D4F8E432687D93F81B
:109FE000CC10D3F8C85093F8CE7081420CBF93F8D0
:109FF000D02093F8D120012A00F04982012695F85B
:10A00000591006FA07F221EA020285F8592093F85E
:10A01000CD20D3F8C81093F8CF5082420CBF93F8EC
:10A02000D03093F8D130012B00F02B82012091F831
:10A03000592000FA05F322EA030381F85930A66893
:10A0400094F862503046F8F78FFBA8B1B268937865
:10A0500043F030039370B26842F21071D3789806DF
:10A0600000F110810139F9D1917000BFB3688022ED
:10A070009A7000BF01233373A068816842F21073A5
:10A08000CA78120600F1D480013BF9D18B7000BF71
:10A09000836880229A7000BF01230373A0688268DE
:10A0A000937803F0C7039370816842F21072CB7803
:10A0B0009D0600F19180666E94F8BE503046F8F728
:10A0C00053FBA8B1B268937843F030039370B26841
:10A0D00042F21071D378980600F1F1800139F9D17C
:10A0E000917000BFB36880229A7000BF0123337360
:10A0F000606E816842F21073CA78120600F1AD807A
:10A10000013BF9D18B7000BF836880229A7000BF39
:10A1100001230373606E8268937803F0C703937022
:10A12000816842F21072CB789D064AD4D4F8C060A0
:10A1300094F81A513046F8F717FBA8B1B268937833
:10A1400043F030039370B26842F21071D3789806EE
:10A1500000F1D2800139F9D1917000BFB36880223B
:10A160009A7000BF01233373D4F8C000816842F2B3
:10A170001073CA78170646D4013BFAD18B7000BF22
:10A18000836880229A7000BF01230373D4F8C00053
:10A190008268937803F0C7039370816842F210726B
:10A1A000CB789B0624D4F8BD93F83DE0BEF1010FB7
:10A1B0007FF4CDAC97F859000EFA02F20243D2B206
:10A1C000CDE4013AAFD18A7000BF836880229A70D3
:10A1D00000BF01230373A9E7013A7FF468AF8A70D7
:10A1E00000BF836880229A7000BF0123037362E777
:10A1F000013AD5D18A7000BF836880229A7000BF6F
:10A2000001230373F8BD022394F81951CB708268BF
:10A21000937843F01003937083681D71826842F253
:10A220001073D1788E0758D4013BFAD19370A6E70A
:10A23000022394F86150CB708268937843F0100346
:10A24000937083681D71826842F21073D1788F0712
:10A2500060D4013BFAD1937019E7022394F8BD5002
:10A26000CB708268937843F01003937083681D71FC
:10A27000826842F21073D1788F0711D4013BFAD172
:10A28000937040E76B00DBB21371B26842F2107357
:10A29000D17889073FF5F0AE013BF9D19370E4E640
:10A2A000D3780221DBB2D17013F0100240F05C8150
:10A2B000DE0700F1318183680222DA702AE76B0041
:10A2C000DBB21371B26842F21073D17889073FF59F
:10A2D0000FAF013BF9D1937003E7D3780221DBB2D2
:10A2E000D17013F0100240F02381DD0700F12E81C0
:10A2F00083680222DA7049E76B00DBB21371B2683F
:10A3000042F21073D17889073FF52EAF013BF9D1A6
:10A31000937022E7D3780221DBB2D17013F01002E0
:10A3200040F01A81DE0700F1EB8083680222DA70C8
:10A33000B4E692F87930012B7FF4ACAD91F8592056
:10A34000B3401343DBB2ACE592F89130012B7FF4BC
:10A3500084AD91F85920B3401343DBB284E592F801
:10A360008530012B7FF461AD91F85920B340134340
:10A37000DBB261E592F82D30012B7FF438AD90F817
:10A380005920B3401343DBB238E593F8211001297B
:10A390007FF410AD90F8592001FA07F31343DBB2B4
:10A3A0000EE5597D01297FF4E8AC90F8592001FAB7
:10A3B00007F31343DBB2E6E4417A01297FF4C1AC31
:10A3C00097F8592001FA0EF31343DBB2C0E493F877
:10A3D0006D30012B7FF499AC90F85920B3401343B2
:10A3E000DBB299E493F84D20012A7FF4F1AB97F8A2
:10A3F000590002FA0CF20243D2B2FFF7F1BB93F814
:10A400003D30012B7FF4BFAB90F85920BB40134384
:10A41000DBB2FFF7BFBB93F86D20012A7FF45AAC83
:10A4200096F8590002FA0EF20243D2B259E493F8B8
:10A430005D30012B7FF429AC90F85920BB401343C9
:10A44000DBB229E493F85D20012A7FF402AC97F88F
:10A45000590002FA0CF20243D2B202E493F84D30F2
:10A46000012B7FF4D1AB90F85920BB401343DBB2F2
:10A47000FFF7D1BB96F8591002FA0EF20A43D2B296
:10A480002AE591F85920AB401343DBB2D5E595F8A6
:10A490005910BA400A43D2B2B7E591F85920B340F7
:10A4A0001343DBB296E596F8591002FA0EF20A430E
:10A4B000D2B277E591F85920B3401343DBB256E5A9
:10A4C00096F8591002FA0EF20A43D2B237E591F823
:10A4D0005920B3401343DBB216E598473AE490475E
:10A4E000FFF79BBB904719E49047FFF755BB904798
:10A4F000FFF7D4BB984783E4904763E4904744E474
:10A5000083680125DD7000BF836801739A7000BF06
:10A51000836880229A7008E783680125DD7000BF98
:10A52000836801739A7000BF836880229A70C2E6C4
:10A5300083681022DA7000BF836803210022017350
:10A540009A7000BF836880229A70D1E683680125E3
:10A55000DD7000BF8368F2E783681022DA7000BF05
:10A56000032183680022D0E783681022DA7000BFDD
:10A57000032183680022D4E730B54568AA6883B018
:10A5800042F21071D3789B065ED50139FAD19170F1
:10A5900000BFAB6880229A7000BF01232B73436811
:10A5A0005A7B012A00F0E3809A6D596D8A42C0F00F
:10A5B0008F800023056E80F85C30AA6842F210712B
:10A5C000D3789B0620D50139FAD1917000BFAB68D2
:10A5D00080229A7000BF01232B73036E5A7B012ADD
:10A5E0007BD09A6D596D8A426DD30023D0F8E0423A
:10A5F00080F8B83034B1236820461B689847E46877
:10A60000002CF8D103B030BDB02190F8BA30917071
:10A61000AA68D478A40642F2107104D40139D4D0C7
:10A62000D478A406FAD5D1788906D6D5917841F0A8
:10A6300030019170A96842F21074CA78920623D44E
:10A64000013CFAD18C70C1E7B02190F85E30917076
:10A65000AA68D478A40642F2107104D4013996D0C5
:10A66000D478A406FAD5D1788C0698D5917841F0A3
:10A6700030019170A96842F21074CA78920612D41F
:10A68000013CFAD18C7083E75B0043F00103DBB23D
:10A690000B71AA6842F21073D17889079DD4013BEF
:10A6A000FAD1937092E75B0043F00103DBB20B71C8
:10A6B000AA6842F21073D1788C073FF570AF013B66
:10A6C000F9D1937064E7511C1A449965137D8DE7A5
:10A6D000511C1A449965137D6CE700228DF8062001
:10A6E0009C689DF8062042F21072E1780D060AD4AB
:10A6F000013AFAD1A27000BF9A688021917000BF20
:10A7000001221A7371E7A27802F0E702A2709A6838
:10A710001179C9B28DF80610917841F00801917055
:10A720009A680221D1709A6842F21071D478A40715
:10A7300003D40139FAD19170DDE7917801F0C701B6
:10A740009170996842F21072CC78A50659D5013AF9
:10A75000FAD18A7000BF996880248C7000BF0124F0
:10A7600099681C73022413460A79CC703EE70022D4
:10A770008DF807209C689DF8072042F21072E1785E
:10A7800009060AD4013AFAD1A27000BF9A68802162
:10A79000917000BF01221A730BE7A27802F0E70262
:10A7A000A2709A681179C9B28DF80710917841F0BA
:10A7B000080191709A680221D1709A6842F2107172
:10A7C000D478A50703D40139FAD19170DDE79178E7
:10A7D00001F0C7019170996842F21072CC78A4061A
:10A7E00013D5013AFAD18A7000BF996880248C7021
:10A7F00000BF012499681C73022413460A79CC70A7
:10A80000D8E602220B79CA70F0E602220B79CA70F0
:10A81000D0E600BF2DE9F84F80460D4648F8041BEE
:10A82000E94FEA4EC0F8108000210446456081607F
:10A830008161C760466140221C300BF07FFC2323FE
:10A8400084F85E30AA68937803F0BF039370A06821
:10A8500001236B7358B10368DD495B688B4204F1D7
:10A860000C0240F0AF8240680221F7F7A1FF256893
:10A8700094F85C3084F85D30002104F160094022D6
:10A88000A7662667C4F86C9025666166616704F167
:10A8900078000BF053FC242384F8BA30AA6893782C
:10A8A00003F0BF039370606E01236B7358B10368AC
:10A8B000C7495B688B4204F1680240F07F824068C0
:10A8C0000221F7F775FF94F8B830C24AC24984F8FC
:10A8D000B930002505264FF4FA771E2004F1BC0399
:10A8E000C4F8BC10C4F8C000C4F8D050C4F8D450A8
:10A8F00084F8D85084F8D950C4F8C420C4F8DC30A7
:10A900000221C4F8C860C4F8CC7009F003FE04F159
:10A91000C40E04F58072B14BC4F8ECE004214FF092
:10A92000010B04F1E00C04F5907004F5A07EC4F86E
:10A930002C2104F5B0724FF0020AC4F8F05084F8EC
:10A94000F45084F8F550C4F8105184F8145184F888
:10A95000155184F81C51C4F8305184F8345184F8EE
:10A960003551C4F8505184F85451C4F8F880C4F8F3
:10A970001881C4F8388184F8FC1084F83CB1C4F81C
:10A980000CC1C4F84C014FF0030C0620C4F8E4607D
:10A99000C4F8E870C4F80461C4F80871C4F824610C
:10A9A000C4F82871C4F84461C4F84871C4F8E030B0
:10A9B000C4F80031C4F8203184F85551C4F86CE172
:10A9C000C4F88C2104F5C07E04F5D072C4F870512F
:10A9D00084F8745184F87551C4F8905184F89451F6
:10A9E00084F89551C4F8B05184F8B45184F8B55145
:10A9F000C4F85881C4F87881C4F89881C4F8B88143
:10AA000084F85CA184F87CC184F89C01C4F8ACE1B2
:10AA1000C4F84031C4F86461C4F86871C4F86031A6
:10AA2000C4F88461C4F88871C4F88031C4F8A461A2
:10AA3000C4F8A871C4F8A03184F8BC61C4F8C4613A
:10AA4000C4F8C871C4F8CC2184F81CB204F5E07BCA
:10AA50004FF0070EFF22C4F8D881C4F8ECB104F51A
:10AA6000F07804F5007BC4F8D05184F8D45184F810
:10AA7000D551C4F8F05184F8F45184F8F55184F8B4
:10AA8000FC51C4F8105284F8145284F81552C4F8DA
:10AA9000305284F8345284F8355284F8DCE1C4F83A
:10AAA0000C82C4F82CB204F50878C4F8C031C4F89C
:10AAB000E461C4F8E871C4F8E031C4F80462C4F891
:10AAC0000872C4F80032C4F82462C4F82872C4F8CA
:10AAD0002032C4F8F891C4F8189284F85D2004F587
:10AAE000107BC4F8389284F83CA284F85CC204F568
:10AAF000187A04F5207CC4F8505284F8545284F833
:10AB00005552C4F8705284F8745284F8755284F81F
:10AB10007CE2C4F8905284F8945284F8955284F8F8
:10AB20009C02C4F8B052C4F84C82C4F84462C4F821
:10AB30004872C4F84032C4F86462C4F86872C4F859
:10AB40006032C4F88462C4F88872C4F88032C4F8F1
:10AB5000A462C4F8A872C4F85892C4F87892C4F8F1
:10AB60009892C4F86CB2C4F88CA2C4F8ACC284F851
:10AB7000B452D4F8048084F8DC1204F5287E04F57D
:10AB8000307184F8B552C4F8D05284F8D45284F8A5
:10AB9000D552C4F8A03284F8BC62C4F8C462C4F8C8
:10ABA000C872C4F8C03284F8B920C4F8B892C4F8A6
:10ABB000D8924046C4F8CCE2C4F8E01294F85E5053
:10ABC000F7F7D2FD88B30BE0B4AC010069090000CF
:10ABD0009D2C0000F0AC01007CAC0100FCAC01003D
:10ABE000D8F80820937843F030039370D8F8082001
:10ABF00042F21071D37898060CD40139FAD19170D1
:10AC000000BFD8F8083080229A7000BF012388F86E
:10AC10000C300AE06B00DBB21371D8F8082042F266
:10AC20001073D178890740F1C4806068816842F26E
:10AC30001073CA7812063ED4013BFAD18B7000BF64
:10AC4000836880229A7000BF012303736068826862
:10AC5000937803F0C7039370816842F21072CB7847
:10AC60009D061DD4266E94F8BA503046F7F77CFD49
:10AC700000283ED0B268937843F030039370B268F6
:10AC800042F21071D37898062AD40139FAD1917022
:10AC900000BFB36880229A7000BF0123337328E09D
:10ACA000013ADCD18A7000BF836880229A7000BFAD
:10ACB00001230373D6E7022394F85D50CB708268BA
:10ACC000937843F01003937083681D71826842F299
:10ACD0001073D1788F074ED4013BFAD19370AEE751
:10ACE0006B00DBB21371B26842F21073D17889073E
:10ACF0005BD5206E816842F21073CA78170625D49E
:10AD0000013BFAD18B7000BF836880229A7000BF2C
:10AD100001230373206E8268937803F0C703937056
:10AD2000816842F21072CB789B0602D42046BDE8BF
:10AD3000F88F013AF7D18A7000BF836880229A7039
:10AD400000BF012303732046BDE8F88F022394F867
:10AD5000B950CB708268937843F010039370836886
:10AD60001D71826842F21073D1788E0710D4013BB6
:10AD7000FAD19370C7E7D3780221DBB2D17013F018
:10AD8000100243D1DE072DD483680222DA705DE71A
:10AD9000D3780221DBB2D17013F010022ED1DD077F
:10ADA00014D483680222DA70B4E7013B9ED1937019
:10ADB0006EE7013B7FF435AF937021E71146022225
:10ADC000984780E511460222984750E5836801259F
:10ADD000DD7000BF836801739A7000BF83688022B2
:10ADE0009A70DEE783680125DD7000BF8368017318
:10ADF0009A7000BF836880229A70C5E7836810222A
:10AE0000DA7000BF032183680022E4E78368102220
:10AE1000DA7000BF032183680022E8E738B50446F2
:10AE20004068A64D03689B68AB4240F05083F5F73D
:10AE30005BFF23681A684FF00041FD23D162536322
:10AE4000D36A002BFCDA6068936B03689B68AB42A3
:10AE500040F03A83F5F73EFF23681A684FF000414F
:10AE60001223D1625363D36A002BFCDA6068936BC0
:10AE700003689B68AB4240F02483F5F735FF2368F5
:10AE80001A684FF00041AE23D1625363D36A002B9E
:10AE9000FCDA6068936B03689B68AB4240F00E83FA
:10AEA000F5F722FF23681A684FF00041B323D162FF
:10AEB0005363D36A002BFCDA6068936B03689B686A
:10AEC000AB4240F0F882F5F705FF23681A684FF0AF
:10AED00000419123D1625363D36A002BFCDA60688E
:10AEE000936B03689B68AB4240F0E282F5F7FCFE8F
:10AEF00023681A684FF00041CA23D1625363D36AB2
:10AF0000002BFCDA6068936B03689B68AB4240F0EF
:10AF1000CC82F5F7DFFE23681A684FF000413F232B
:10AF2000D1625363D36A002BFCDA6068936B0368C9
:10AF30009B68AB4240F0B682F5F7D6FE23681A68EC
:10AF40004FF00041A223D1625363D36A002BFCDA95
:10AF50006068936B03689B68AB4240F0A082F5F792
:10AF6000B9FE23681A684FF000410023D162536391
:10AF7000D36A002BFCDA6068936B03689B68AB4272
:10AF800040F08A82F5F7B0FE23681A684FF000415E
:10AF9000A123D1625363D36A002BFCDA6068936B00
:10AFA00003689B68AB4240F07482F5F793FE236818
:10AFB0001A684FF000410023D1625363D36A002B1B
:10AFC000FCDA6068936B03689B68AB4240F05E827A
:10AFD000F5F78AFE23681A684FF00041A023D1627A
:10AFE0005363D36A002BFCDA6068936B03689B6839
:10AFF000AB4240F04882F5F76DFE23681A684FF0C7
:10B0000000411423D1625363D36A002BFCDA6068D9
:10B01000936B03689B68AB4240F03282F5F75AFEAF
:10B0200023681A684FF000411123D1625363D36A39
:10B03000002BFCDA6068936B03689B68AB4240F0BE
:10B040001C82F5F751FE23681A684FF00041B523C2
:10B05000D1625363D36A002BFCDA6068936B036898
:10B060009B68AB4240F00682F5F734FE23681A680D
:10B070004FF000410023D1625363D36A002BFCDA06
:10B080006068936B03689B68AB4240F0F081F5F712
:10B090002BFE23681A684FF00041AB23D162536343
:10B0A000D36A002BFCDA6068936B03689B68AB4241
:10B0B00040F0DA81F5F70EFE02E000BF310C00002F
:10B0C00023681A684FF000410123D1625363D36AA9
:10B0D000002BFCDA6068936B03689B68AB4240F01E
:10B0E000C081F5F701FE23681A684FF00041B423D0
:10B0F000D1625363D36A002BFCDA6068936B0368F8
:10B100009B68AB4240F0AA81F5F7E4FD23681A681A
:10B110004FF00041A023D1625363D36A002BFCDAC5
:10B120006068936B03689B68AB4240F09481F5F7CD
:10B13000D1FD23681A684FF00041FD23D1625363AB
:10B14000D36A002BFCDA6068936B03689B68AB42A0
:10B1500040F07E81F5F7C8FD23681A684FF0004182
:10B16000C123D1625363D36A002BFCDA6068936B0E
:10B1700003689B68AB4240F06881F5F7ABFD23683C
:10B180001A684FF00041FF23D1625363D36A002B4A
:10B19000FCDA6068936B03689B68AB4240F05281B5
:10B1A000F5F7A2FD23681A684FF00041C723D1626A
:10B1B0005363D36A002BFCDA6068936B03689B6867
:10B1C000AB4240F03C81F5F785FD23681A684FF0EB
:10B1D00000410F23D1625363D36A002BFCDA60680D
:10B1E000936B03689B68AB4240F02681F5F77CFDCA
:10B1F00023681A684FF00041B923D1625363D36AC0
:10B20000002BFCDA6068936B03689B68AB4240F0EC
:10B210001081F5F769FD23681A684FF00041B123EA
:10B22000D1625363D36A002BFCDA6068936B0368C6
:10B230009B68AB4240F0FA80F5F74CFD23681A6832
:10B240004FF00041E223D1625363D36A002BFCDA52
:10B250006068936B03689B68AB4240F0E480F5F74D
:10B2600043FD23681A684FF00041D123D162536334
:10B27000D36A002BFCDA6068936B03689B68AB426F
:10B2800040F0CE80F5F726FD23681A684FF00041A4
:10B29000A223D1625363D36A002BFCDA6068936BFC
:10B2A00003689B68AB4240F0B880F5F713FD236854
:10B2B0001A684FF000412023D1625363D36A002BF8
:10B2C000FCDA6068936B03689B68AB4240F0A28035
:10B2D000F5F70AFD23681A684FF00041BB23D162DD
:10B2E0005363D36A002BFCDA6068936B03689B6836
:10B2F000AB4240F08C80F5F7EDFC23681A684FF004
:10B3000000411F23D1625363D36A002BFCDA6068CB
:10B31000936B03689B68AB4276D1F5F7E5FC236835
:10B320001A684FF00041B623D1625363D36A002BF1
:10B33000FCDA6068936B03689B68AB4261D1F5F7F8
:10B34000C9FC23681A684FF000410823D162536397
:10B35000D36A002BFCDA6068936B03689B68AB428E
:10B360004CD1F5F7C1FC23681A684FF00041BE23A9
:10B37000D1625363D36A002BFCDA6068936B036875
:10B380009B68AB4237D1F5F7A5FC23681A684FF0EC
:10B3900000410723D1625363D36A002BFCDA606853
:10B3A000936B03689B68AB4222D1F5F79DFC236841
:10B3B0001A684FF00041A923D1625363D36A002B6E
:10B3C000FCDA6068936B03689B68AB420DD1F5F7BC
:10B3D0008BFC23681A684FF00041AF23D16253639E
:10B3E000D36A002BFCDA936B38BD00219847F0E755
:10B3F00000219847DBE701219847C6E700219847DD
:10B40000B1E7012198479CE70021984787E7012190
:10B41000984772E7002198475CE70121984746E783
:10B420000121984730E7002198471AE70121984702
:10B4300004E700219847EEE600219847D8E601216D
:10B440009847C2E600219847ACE60121984796E666
:10B450000021984780E6012198476AE60121984734
:10B4600054E6002198473EE60121984728E600214E
:10B4700098470EE601219847F8E500219847E2E554
:10B4800001219847CCE501219847B6E5002198476E
:10B49000A0E5012198478AE50021984774E501213C
:10B4A00098475EE50021984748E50121984732E535
:10B4B000002198471CE50121984706E5002198479F
:10B4C000F0E400219847DAE401219847C4E4002120
:10B4D0009847AEE4F8B500F500541C3406466068A1
:10B4E0002E4F03689B68BB420D464ED1F5F7FCFB1F
:10B4F00042F21C034FF00041F3581A68C123D16295
:10B500005363D36A002BFCDA6068936B03689B6813
:10B51000BB4237D1F5F7DEFB42F21C024FF000438D
:10B52000B2581268D3625563D36A002BFCDA6068A4
:10B53000936B036815F001019B6811D1BB4227D1C1
:10B54000F5F7D2FB42F21C034FF00041F3581A68A2
:10B55000A723D1625363D36A002BFCDA936BF8BD47
:10B56000BB4217D1F5F7C0FB42F21C034FF000417C
:10B57000F3581A68A623D1625363D36A002BFCDA0E
:10B58000936BF8BD01219847C6E700219847AFE7C4
:10B590009847D7E700219847E6E700BF310C000045
:10B5A00010B4036841681A780C78417A037A0C4227
:10B5B00002EA03021BD0837A03F003030AB143F0CB
:10B5C000040343F008039A10013B82720D2B0BD841
:10B5D000DFE803F021071B070A152121150A071BC5
:10B5E0000721C368013BC3605DF8044B7047837A51
:10B5F00003F00303002AE6D043F00403E3E7C36843
:10B600005DF8044B023BC3607047C3685DF8044BB0
:10B610000233C3607047C3685DF8044B0133C360F5
:10B62000704700BF08B5034BD3F8EC00FFF7B8FF35
:10B6300008BD00BF34B0FF1F08B5034BD3F8E800C6
:10B64000FFF7AEFF08BD00BF34B0FF1F08B5034BC6
:10B65000D3F8E400FFF7A4FF08BD00BF34B0FF1F1C
:10B6600008B5034BD3F8E000FFF79AFF08BD00BF11
:10B6700034B0FF1F08B5034BD3F8DC00FFF790FF91
:10B6800008BD00BF34B0FF1F08B5034BD3F8D80086
:10B69000FFF786FF08BD00BF34B0FF1F08B5034B9E
:10B6A000D3F8D400FFF77CFF08BD00BF34B0FF1F04
:10B6B00008B5034BD3F8D000FFF772FF08BD00BFF9
:10B6C00034B0FF1F08B5034BD3F8CC00FFF768FF79
:10B6D00008BD00BF34B0FF1F08B5034BD3F8C4004A
:10B6E000FFF75EFF08BD00BF34B0FF1F08B5034B76
:10B6F000D3F8C000FFF754FF08BD00BF34B0FF1FF0
:10B7000008B5034BD3F8BC00FFF74AFF08BD00BFE4
:10B7100034B0FF1F08B5034BD3F8B800FFF740FF64
:10B7200008BD00BF34B0FF1F08B5034BD3F8B40009
:10B73000FFF736FF08BD00BF34B0FF1F08B5034B4D
:10B74000D3F8B000FFF72CFF08BD00BF34B0FF1FD7
:10B7500008B5034BD3F8AC00FFF722FF08BD00BFCC
:10B7600034B0FF1F08B5034BD3F8A800FFF718FF4C
:10B7700008BD00BF34B0FF1F08B5034BD3F8A400C9
:10B78000FFF70EFF08BD00BF34B0FF1F08B5034B25
:10B79000D3F8A000FFF704FF08BD00BF34B0FF1FBF
:10B7A00008B5034BD3F89C00FFF7FAFE08BD00BFB5
:10B7B00034B0FF1F08B5034BD3F89800FFF7F0FE35
:10B7C00008BD00BF34B0FF1F08B5034BD3F8940089
:10B7D000FFF7E6FE08BD00BF34B0FF1F08B5034BFE
:10B7E000D3F89000FFF7DCFE08BD00BF34B0FF1FA8
:10B7F00008B5034BD3F88C00FFF7D2FE08BD00BF9D
:10B8000034B0FF1F08B5034BD3F88800FFF7C8FE1C
:10B8100008BD00BF34B0FF1F08B5034BD3F8840048
:10B82000FFF7BEFE08BD00BF34B0FF1F08B5034BD5
:10B83000D3F88000FFF7B4FE08BD00BF34B0FF1F8F
:10B8400008B5024BD86FFFF7ABFE08BD34B0FF1F41
:10B8500008B5024B986FFFF7A3FE08BD34B0FF1F79
:10B8600008B5024B586FFFF79BFE08BD34B0FF1FB1
:10B8700008B5024B186FFFF793FE08BD34B0FF1FE9
:10B8800008B5024BD86EFFF78BFE08BD34B0FF1F22
:10B8900008B5024B986EFFF783FE08BD34B0FF1F5A
:10B8A00008B5024B586EFFF77BFE08BD34B0FF1F92
:10B8B00008B5024B186EFFF773FE08BD34B0FF1FCA
:10B8C00008B5024BD86DFFF76BFE08BD34B0FF1F03
:10B8D00001380B463A2800F25C82DFE810F0530290
:10B8E0004C0245023E0237023002290222021B02AC
:10B8F000AE01A701A001990192018B0184017D0194
:10B9000076016F01680161015A0153014C01450143
:10B910003E0137013001290122011B0113010B01F6
:10B920000301FB00F300EB00E300DB00D300CB00DE
:10B93000C300BB00B300AB00A3009B0093008B00CF
:10B9400083007B0073006B0063005B0053004B00BF
:10B9500043003B00BC4ABD49C2F8EC303B20042206
:10B9600008F04AB9B84ABA49C2F8E8303A20042285
:10B9700008F042B9B44AB749C2F8E4303920042289
:10B9800008F03AB9B04AB449C2F8E030382004228D
:10B9900008F032B9AC4AB149C2F8DC303720042291
:10B9A00008F02AB9A84AAE49C2F8D8303620042295
:10B9B00008F022B9A44AAB49C2F8D4303520042299
:10B9C00008F01AB9A04AA849C2F8D030342004229D
:10B9D00008F012B99C4AA549C2F8CC3033200422A1
:10B9E00008F00AB9984AA249C2F8C83032200422A5
:10B9F00008F002B9944A9F49C2F8C43031200422A9
:10BA000008F0FAB8904A9C49C2F8C03030200422AD
:10BA100008F0F2B88C4A9949C2F8BC302F200422B1
:10BA200008F0EAB8884A9649C2F8B8302E200422B5
:10BA300008F0E2B8844A9349C2F8B4302D200422B9
:10BA400008F0DAB8804A9049C2F8B0302C200422BD
:10BA500008F0D2B87C4A8D49C2F8AC302B200422C1
:10BA600008F0CAB8784A8A49C2F8A8302A200422C5
:10BA700008F0C2B8744A8749C2F8A43029200422C9
:10BA800008F0BAB8704A8449C2F8A03028200422CD
:10BA900008F0B2B86C4A8149C2F89C3027200422D1
:10BAA00008F0AAB8684A7E49C2F8983026200422D5
:10BAB00008F0A2B8644A7B49C2F8943025200422D9
:10BAC00008F09AB8604A7849C2F8903024200422DD
:10BAD00008F092B85C4A7549C2F88C3023200422E1
:10BAE00008F08AB8584A7249C2F8883022200422E5
:10BAF00008F082B8544A6F49C2F8843021200422E9
:10BB000008F07AB8504A6C49C2F8803020200422EC
:10BB100008F072B84C4A6949D3671F20042208F024
:10BB20006BB8494A664993671E20042208F064B83E
:10BB3000454A644953671D20042208F05DB8424A13
:10BB4000614913671C20042208F056B83E4A5F4939
:10BB5000D3661B20042208F04FB83B4A5C49936629
:10BB60001A20042208F048B8374A5A495366192067
:10BB7000042208F041B8344A5749136618200422B9
:10BB800008F03AB8304A5549D3651720042208F026
:10BB900033B82D4A524993651620042208F02CB878
:10BBA000294A504953651520042208F025B8264A31
:10BBB0004D4913651420042208F01EB8224A4B494F
:10BBC000D3641320042208F017B81F4A484993642D
:10BBD0001220042208F010B81B4A46495364112071
:10BBE000042208F009B8184A4349136410200422BB
:10BBF00008F002B8144A4149D3630F20042207F029
:10BC0000FBBF114A3E4993630E20042207F0F4BFA4
:10BC10000D4A3C4953630D20042207F0EDBF0A4A48
:10BC2000394913630C20042207F0E6BF064A37495E
:10BC3000D3620B20042207F0DFBF034A344993622A
:10BC40000A20042207F0D8BF34B0FF1F25B6000039
:10BC500039B600004DB6000061B6000075B60000B0
:10BC600089B600009DB60000B1B60000C5B6000060
:10BC7000D51A0000D9B60000EDB6000001B70000EB
:10BC800015B7000029B700003DB7000051B700000C
:10BC900065B7000079B700008DB70000A1B70000BC
:10BCA000B5B70000C9B70000DDB70000F1B700006C
:10BCB00005B8000019B800002DB8000041B8000018
:10BCC00051B8000061B8000071B8000081B80000F0
:10BCD00091B80000A1B80000B1B80000C1B80000E0
:10BCE000DD26000051260000C52500003925000092
:10BCF000AD2400002124000095230000092300004A
:10BD00007D220000F121000065210000D920000003
:10BD10004D2000001F4A204953620920042207F0E9
:10BD20006BBF1C4A1D4913620820042207F064BF40
:10BD3000184A1B49D3610720042207F05DBF154A4A
:10BD4000184993610620042207F056BF114A16498C
:10BD500053610520042207F04FBF0E4A13491361B7
:10BD60000422104607F048BF0A4A1149D360032055
:10BD7000042207F041BF074A0E49936002200422C3
:10BD800007F03ABF034A0C4953600120042207F030
:10BD900033BF704734B0FF1FC11F0000351F0000C4
:10BDA000A91E00001D1E0000911D0000051D0000C1
:10BDB000791C0000ED1B0000611B00002DE9F04123
:10BDC000437D012B8CB05ED0036EC26D934207D3CE
:10BDD00000231C464A1E9A420AD00CB0BDE8F081EE
:10BDE0005A1C034402661C7F4A1E23469A42F4D121
:10BDF000437D8DF80840012B00F05781036EC46D20
:10BE0000A342C0F08B8000258DF80950A34280F03A
:10BE10004A815E1C034406661D7F33468DF80A5036
:10BE2000A34280F039815C1C034404661B7F8DF8BB
:10BE30000B3004290DF1080E1FD00EEB0201002576
:10BE40000DF10B0202248027012609E00CF1010309
:10BE5000844403669CF81C3002F8013F91420CD0E8
:10BE6000437D012B60D0D0F860C0C36D9C45EDD3FD
:10BE7000002302F8013F9142F2D14368704698478F
:10BE80000CB0BDE8F08100238DF8033004699DF803
:10BE9000033042F21073E27816060AD4013BFAD15D
:10BEA000A37000BF036980229A7000BF012303754D
:10BEB0008EE7A37803F0E703A37003691A79D2B27F
:10BEC0008DF803209A7842F008029A7003690222E2
:10BED000DA70036942F21072DC78A50703D4013AE4
:10BEE000FAD19A70DDE79A7802F0C7029A70026977
:10BEF00042F21073D478A40640F1D080013BF9D10E
:10BF0000937000BF02698024947000BF012402690D
:10BF1000047502241579D4701C465BE75E1C03444B
:10BF200006661D7F33466FE78DF80750D0F8108006
:10BF30009DF8073042F2107398F803C01CF0800F90
:10BF40000AD1013BF8D188F8023000BF03699F7025
:10BF500000BF002306758CE798F8023003F0E70372
:10BF600088F80230036993F804C05FFA8CFC8DF8FE
:10BF700007C093F802C04CF0080C83F802C00369B4
:10BF8000DC70036942F2107C93F8038018F0020F12
:10BF900005D1BCF1010CF7D183F802C0D5E793F8C5
:10BFA00002C00CF0C70C83F802C0D0F8108042F237
:10BFB000107C98F803309B0611D5BCF1010CF8D128
:10BFC00088F802C000BF03699F7000BFD0F81080DE
:10BFD0000675634698F804C088F803403CE798F873
:10BFE000043088F8034037E7AB7803F0E703AB7021
:10BFF00003691C79E4B28DF806409C7844F008048B
:10C000009C7003690224DC70036942F21074DD78CD
:10C01000AE0759D4013CFAD19C7000BF036980245B
:10C020009C7000BF0123447D03750023012C8DF813
:10C03000093040F0D88000238DF8053005699DF85F
:10C04000053042F21073EC78270671D4013BFAD127
:10C05000AB7000BF036980249C7000BF0123447D46
:10C0600003750023012C8DF80A3040F0BF800023B7
:10C070008DF8043005699DF8043042F21073EC78B5
:10C0800027063BD4013BFAD1AB7000BF0369802483
:10C090009C7000BF012303750023C8E613790225B5
:10C0A0001C46D57096E60025B8E600238DF80630CC
:10C0B00005699DF8063042F21073EC78270693D498
:10C0C000013BFAD1AB70A8E79C7804F0C7049C70E0
:10C0D000046942F21073E578AD0676D5013BFAD1DA
:10C0E000A37000BF04698025A57000BF0125046905
:10C0F000057502252679E570447D97E7AB7803F056
:10C10000E703AB7003691C79E4B28DF804409C78B6
:10C1100044F008049C7003690224DC70036942F255
:10C120001074DD78AE071DD4013CFAD19C70ACE7E9
:10C13000AB7803F0E703AB7003691C79E4B28DF8C8
:10C1400005409C7844F008049C7003690224DC706C
:10C15000036942F21074DD78AE071CD4013CFAD1B9
:10C160009C7076E79C7804F0C7049C70046942F2E6
:10C170001073E578AD0632D5013BFAD1A37000BF4C
:10C1800004698025A57000BF012504690575022595
:10C190002679E5704BE69C7804F0C7049C7004692E
:10C1A00042F21073E578AD0614D5013BFAD1A370C5
:10C1B00000BF04698025A57000BF012504690575CD
:10C1C00002252679E570447D4CE702252379E57048
:10C1D000447D2BE702252379E570447D42E7022563
:10C1E0002379E57023E6036EC46D0FE6036EC46D1C
:10C1F00016E600BF08B5044B1B681BB10146184684
:10C20000FFF7DCFD08BD00BF30B0FF1F4FF47A72AE
:10C21000704B02FB01F19942F0B400F2B0806E4B1A
:10C22000994200F2B0806D4B994200F2AE806C4BA7
:10C23000994200F2AF806B4B994200F2AF806A4B9B
:10C24000994200F2B180694B994200F2AF804EF200
:10C25000E043994200F28A8047F26F23994288BFF7
:10C260004FF4807200F28380614B4FF400464FF42C
:10C270008072994280F08B8053005E4CB4FBF3F5E2
:10C28000A94280F089801344B4FBF3F5A94280F001
:10C2900087801344B4FBF3F5A94280F083801344F4
:10C2A000B4FBF3F5A94280F083801344B4FBF3F5AB
:10C2B000A9427FD21344B4FBF3F5A9427CD21344C4
:10C2C000B4FBF3F5A94279D21344B4FBF3F5A942C8
:10C2D00076D21344B4FBF3F4A14273D21344454C19
:10C2E000B4FBF3F5A9426FD21344B4FBF3F5A942B2
:10C2F0006CD21344B4FBF3F5A9423ED21344B4FB11
:10C30000F3F5A94264D21344B4FBF3F5A94229D250
:10C310001344B4FBF3F4A14228BF102423D2F02429
:10C32000354D3449354A4FF47A7707FB03F3B1FBB7
:10C33000F3F343602B6823F008032B60296821F492
:10C340007F2323F47F6343F46023334323432B6031
:10C3500013681B07FCD5284A136843F008031360D1
:10C36000F0BC70470F24013C2401D9E78022530818
:10C370001E02204BB3FBF2F37BE70D24F3E71D4BCA
:10C380000026012275E70222F1E70422EFE71346B7
:10C390000024C5E70822EAE70224E4E71022E6E7E2
:10C3A0000324E0E70424DEE72022E0E74022DEE782
:10C3B0000524D8E70624D6E70724D4E70824D2E7E3
:10C3C0000924D0E70A24CEE70B24CCE70C24CAE7E3
:10C3D0000E24C8E7DF7072006F383900379C1C00EC
:10C3E0001B4E0E000D27070086930300C2C90100F3
:10C3F0000E270700000E27072C100B4024100B40BF
:10C400002DE9F0410746884608F0C0F8194C1A4E4D
:10C41000054604E008F0BAF8401BB04226D823686D
:10C42000DB07F7D4154A164BC2F800801F6008F0EE
:10C43000ADF8144C104D064604E008F0A7F8801B38
:10C44000A84213D82268104B0E491340002BF4D099
:10C450000E4B0A681A600A601B680B481840A0F16E
:10C460000100B0FA80F04009BDE8F0810020BDE88D
:10C47000F08100BF24100B4040420F0008100B4019
:10C480000C100B4030100B4001000F0064B2FF1F76
:10C490002DE9F04F85B03F4F01900291039208F0D3
:10C4A00075F8DFF82CA13C4EBB468146DAF80080D7
:10C4B0003A4D08F06BF8044604E008F067F8001BFA
:10C4C000A84225D83368D907F7D4354A354BC2F886
:10C4D0000080536008F05AF8304C054604E008F03C
:10C4E00055F8401BA04213D83A682F4B1340002B3D
:10C4F000F5D02E4CDBF800302360CBF800302268FA
:10C50000294B1340012B03D1294A1268D2050FD4BD
:10C5100008F03CF8214BC9EB00009842C6D90198BD
:10C5200040F23312292105B0BDE8F04F07F01EB9E3
:10C53000204D21492B701A48029E204A0023236077
:10C54000039B0B6006601E4B1E4E16601E481F4A62
:10C5500088631A6008F01AF8104E074604E008F0E5
:10C5600015F8C01BB0420BD82B78002BF7D12268EE
:10C57000154B1340022B03D1012005B0BDE8F08F0D
:10C58000019840F23D12232105B0BDE8F04F07F0BD
:10C59000EDB800BF30100B4024100B4040420F009C
:10C5A00008100B4000001A0D01000F0064B2FF1FBD
:10C5B00010100B4068B2FF1F00100B4004100B401E
:10C5C0000C100B404000010002007F1111003A06E0
:10C5D0006CB2FF1F2DE9F04F93B0804607F0D6FFF5
:10C5E000A44CA54E054605E007F0D0FF401BB04225
:10C5F00000F2DC80236813F00103F5D19F49A04AC3
:10C600000B60136007F0C2FF9E4C9B4D064605E091
:10C6100007F0BCFF801BA84200F2C88022689A4B3A
:10C62000984F1340002BF3D0DFF884A23B68CAF880
:10C6300000303B60DAF80020934B1340012B40F0B0
:10C64000B5808C4EBB464FF00A0907F09FFF8A4D1C
:10C65000044604E007F09AFF001BA84225D833687F
:10C66000DA07F7D48549894B834C4FF4D5720A60B9
:10C67000834A136007F08AFF054604E007F086FF4F
:10C68000401BA04211D83A687F4B1340002BF5D0D5
:10C69000DBF80030CAF80030CBF80030DAF80020C0
:10C6A000794B1340012B00F00582B9F10109CCD17F
:10C6B00098F81120764B002A08BF4FF440130193DD
:10C6C00007F064FF6F4F6B4CDFF8B0B10090B946D4
:10C6D00007F05CFF684E054604E007F057FF401B7B
:10C6E000B04258D8236813F00103F6D1CBF80030DC
:10C6F000634B684A1A6007F049FF5F4D064604E045
:10C7000007F044FF801BA84245D83A685E4B1340AF
:10C71000002BF5D0D9F80030CAF80030C9F8003045
:10C72000DAF80020584B1340012B34D107F02EFFCC
:10C73000514E054604E007F029FF401BB0422AD8BD
:10C740002368DB07F7D4019ACBF800204C4A524B00
:10C75000136007F01BFF484D064604E007F016FF84
:10C76000801BA84217D83A68474B1340002BF5D0DE
:10C77000D9F80030CAF80030C9F80030DAF80030D3
:10C78000414D1D40012D06D107F000FF009A3A4BA4
:10C79000801A984215D9404640F29112432106F082
:10C7A000E5FF8346584613B0BDE8F08F40464FF48E
:10C7B000BF72202106F0DAFF8346584613B0BDE869
:10C7C000F08F364B1A68002A82DA354A19681160F0
:10C7D0001B68284C284E580044BF324B1D7007F090
:10C7E000D5FE054605E007F0D1FE401BB04200F241
:10C7F0006B81236813F00103F5D12048204A2A49B0
:10C800000360116007F0C2FE1E4D1B4C064605E09A
:10C8100007F0BCFE801BA04200F256812A681A4B2A
:10C8200018491340002BF3D00B68CAF800300B6096
:10C83000DAF80020144B1340012B40F0458107F03B
:10C84000A5FE0C4C0C4E054605E007F09FFE401B74
:10C85000B04200F24981236813F00103F5D1074883
:10C86000074A12490360116007F090FE054C024D23
:10C87000064625E024100B4040420F0008100B40F4
:10C880000C100B4030100B4001000F0000001A0884
:10C890000000304000001A370000022910100B4041
:10C8A0005CB2FF1F58B2FF1F0000090200001A030C
:10C8B00064B2FF1F07F06AFE801BA84200F21481D9
:10C8C0002268B24BB2491340002BF3D00B68CAF870
:10C8D00000300B60DAF80020AC4B1340012B40F025
:10C8E0000381AC4BDFF8D8921F68AB4CAB4E3F0CCA
:10C8F0003F04C9F8007007F049FE054605E007F05F
:10C9000045FE401BB04200F2F7802368D907F6D4F9
:10C91000A349A44BA44A0F601A6007F037FE9C4D50
:10C920009E4C064605E007F031FE801BA04200F257
:10C93000E3802A68954B96491340002BF3D00B688F
:10C94000CAF800300B60DAF80020904B1340012B3E
:10C9500040F0D2808F48954A0068954B95491268FF
:10C960001B68096888F83000040A060C050E88F870
:10C970002F40100C140A88F82C20120E88F824106E
:10C9800088F8283088F82D5088F82B401D0A1C0C98
:10C9900088F82A001B0E080A88F82920090C0022B2
:10C9A00088F82E6088F8275088F8264088F82530C7
:10C9B00088F8230088F8221088F83120D9F8007010
:10C9C000754E764D07F0E2FD044605E007F0DEFD0A
:10C9D000001BA84200F298803368DA07F6D4704949
:10C9E000704B754A0F601A6007F0D0FD684D6B4CB4
:10C9F000064605E007F0CAFD801BA04200F28480D5
:10CA00002A68624B624F1340002BF3D03B68CAF890
:10CA100000303B60DAF800205C4B1340012B73D1EF
:10CA20005C4862490068624B624A09681B68126888
:10CA300088F82000040A050E060C88F81F40080C30
:10CA40000C0A88F81C10090E88F8142088F8183091
:10CA500088F81D5088F81B401D0A1C0C88F81A0025
:10CA60001B0E100A88F81910120C002188F81640C5
:10CA700088F8130088F8211088F81E6088F817508D
:10CA800088F8153088F81220D9F800104B484C4C23
:10CA9000FFF7B6FC00283FD021684A48FFF7B0FCFA
:10CAA000002841D1404640F2AB12402106F05EFE24
:10CAB000834682E6374A1268B2F5D57F0CD188F8F2
:10CAC0001130414B0193FBE5404640F29912212180
:10CAD00006F04CFE834670E640464FF4C2722521B4
:10CAE00006F044FE834668E640464FF4CE722221AB
:10CAF00006F03CFE834660E6404640F2A112262145
:10CB000006F034FE834658E640464FF4D2722721A1
:10CB100006F02CFE834650E6404640F2A712242140
:10CB200006F024FE834648E602212848FFF768FC09
:10CB300083460028B6D0264A26481168164C21F0B4
:10CB400006011160116841F0020111604FF01012EE
:10CB5000026007F01BFD8DE80101D9F800800F4E3F
:10CB600007F014FD054604E007F010FD401BB0423D
:10CB70004FD82368DB07F7D4094A174BC2F8008067
:10CB8000536007F003FD054D06462CE001000F0041
:10CB900030100B4010100B4024100B4040420F008F
:10CBA00008100B400C100B400000090914100B403A
:10CBB00018100B401C100B400000090A00001B0756
:10CBC0006CB2FF1F00001A370000304000001A0648
:10CBD00028100B4044100B4000001A0D07F0D6FC43
:10CBE000801BA84215D83A68474B1340002BF5D05C
:10CBF000464B464A1B68CAF800301360DAF800302A
:10CC0000414A43491A40012A03D1424B1B68D805C7
:10CC100036D407F0BBFC009A3F4B801A98429CD94F
:10CC2000DDF8048040F233122921404606F09EFDD3
:10CC300000284ED146F2A811DFF818A1DFF81891AC
:10CC4000364F374E374D384C0022CAF80020404648
:10CC5000C9F800203A6032602A602260FFF7D6FAF5
:10CC600040F243424FF488600121CAF80020C9F81D
:10CC70000020386032602A60226088F810109CE53D
:10CC80002A4C2B4E22702B4DDDF804802A480022BE
:10CC900002AB0A6033602949294A6FF07F462E6053
:10CCA000284D0D60284D29490560116007F06EFC84
:10CCB000194D064604E007F069FC801BA8421CD809
:10CCC0002378002BF7D1DAF800101F4A0A40022A15
:10CCD00013D19DF815209307ACD502AA1C494046F4
:10CCE000FFF7D6FB0028A5D09DF8182002F00F0210
:10CCF000012A9FD14CF250319EE740F23D12232190
:10CD0000404606F033FD93E701000F0030100B4062
:10CD100064B2FF1F10100B4040420F0008D00440C7
:10CD20000CD0044010D0044014D0044068B2FF1F5F
:10CD300000100B4008100B4038100B4004100B4043
:10CD40000C100B404000010002007F1111003A0658
:10CD5000F1FFFF8000D0044004D004402DE9F04FE3
:10CD60003C4FDFF83091DFF804A13B4E85B0BB4665
:10CD7000039001910292D9F80080384D07F006FC2B
:10CD8000044604E007F002FC001BA842F3D8336815
:10CD9000D907F7D4324A334BC2F80080536007F00A
:10CDA000F5FB2E4C054604E007F0F0FB401BA042CB
:10CDB000E1D83A682C4B1340002BF5D0DBF800305B
:10CDC000CAF80030CBF80030DAF80020264B2749AB
:10CDD0001340012BCFD1264A1268D205CBD5254C62
:10CDE000254A237000230B60244B02991B781160A5
:10CDF00023BB019B5B021A48214D03602149224A53
:10CE00002248164E4FF481332B60214B086013608B
:10CE100007F0BCFB054604E007F0B8FB401BB0423E
:10CE20000ED82378002BF7D1DAF80020174B1340E7
:10CE3000022B05D1012005B0BDE8F08F019BDAE798
:10CE4000039840F2FD12322105B0BDE8F04F06F024
:10CE50008DBC00BF30100B4024100B4040420F002F
:10CE600008100B4000001A0D01000F0064B2FF1FF4
:10CE700010100B4068B2FF1F00100B4058B2FF1F8C
:10CE800004100B4038100B400C100B4002007F11B7
:10CE900001003A186CB2FF1F70B5AB4B1D6882B031
:10CEA000E5B1C378591ECAB2012A044618D9162B17
:10CEB00016D0172B00F012816378222B00D06BB9AB
:10CEC000E378E12B00F024813CD9E42B00F01881B9
:10CED000E52B00F0A880E32B00F0B68002B070BD17
:10CEE00095F88160002085F8110185F8100185F81A
:10CEF0000701C6B9162B16D0012ADDD80021D5F8B6
:10CF00008C3085F806112279DA65986C03F14C02B1
:10CF1000FFF724FF8D4A217941F2D433D058814262
:10CF200018BFD150C8E795F88200002870D0012AB8
:10CF300040F29980162B70D0172BBDD1002385F8B5
:10CF40008230D9E7032B7BD00F2BC7D1237903F095
:10CF5000F002A02AC2D195F81121002ABED003F018
:10CF60000F030C2B00F0E3800D2BB7D1784AA37987
:10CF7000516810686A4603C2D90748BF9DF800206F
:10CF80004FF0000485F8164148BF85F816219A072E
:10CF900006D595F816219DF801100A4385F816214B
:10CFA0005E0706D595F816119DF802200A4385F80C
:10CFB00016211C0706D595F816119DF803200A4383
:10CFC00085F81621D80606D595F816119DF8042087
:10CFD0000A4385F81621990606D595F816119DF88D
:10CFE00005200A4385F816215A0606D595F816112C
:10CFF0009DF806200A4385F81621DB093FF46EAF41
:10D0000095F816219DF80730134385F8163165E72A
:10D01000162B7FF471AF012A25D9012385F88230C0
:10D0200085F8813068E7222200214A4809F086F815
:10D0300049492122474802B0BDE8704009F08EB945
:10D04000012385F8063149E795F81131002B3FF4AB
:10D0500045AF1123FF22E0212846F4F791FB01237D
:10D0600085F810313AE7237995F8800098427FF6E9
:10D0700045AF16293FF642AF01A050F821F000BF9E
:10D0800029D1000023D10000FDCE0000FDCE00001C
:10D09000FDCE0000FDCE0000FDCE0000FDCE000064
:10D0A000FDCE0000FDCE0000FDCE0000FDCE000054
:10D0B000FDCE0000FDCE0000FDCE0000FDCE000044
:10D0C000FDCE0000FDCE0000FDCE0000FDCE000034
:10D0D000FDCE00001BD000003DCF000095F8811070
:10D0E000002385F8113185F8103185F807310029C2
:10D0F0003FF4E2AE95F88230002B7FF41FAFFBE6E1
:10D1000022220021134809F019F8211D212291E75C
:10D1100095F81031002B3FF4E1AE012385F8113171
:10D12000DCE6C5F88830E7E6C5F88430E4E6A279A5
:10D13000637943EA0223A5F81231E379227A43EABC
:10D140000223A5F81431C9E6C814FF1FCC14FF1F31
:10D150006CAD01008429FF1F9CBF01002DE9F04F39
:10D1600090F85E3091B083461BB1837F002B00F0B6
:10D170004A819BF979300993002B1A4621DB41F251
:10D18000D4335BF80310089108468242114600F040
:10D19000DF82C34A4BF80310104644F25043019219
:10D1A000C35C002B40F0848141F2D433089A4BF8E1
:10D1B0000320BC4B1B680D9341F2F4330D9A4BF8DE
:10D1C00003209BF97A30002B79DB41F2D4325BF8F3
:10D1D000021006918B4241F2254118BF4BF80230F4
:10D1E0001BF80120002A40F0FE80AD4A0192114652
:10D1F00044F250428A5C002A40F0E4820323DBF8C8
:10D20000FC26DBF8D009002ACABF0BF2DC624FF023
:10D210007E5111680BF59C5200289161CABF0BF535
:10D220001B624FF07E5111680BF59C52D161DBF807
:10D23000A42C002AC8BF0BF684420BF59D51CCBF2D
:10D2400012684FF07E520A60DBF8782F002ACABFBE
:10D250000BF658724FF07E5111680BF59D52012B61
:10D26000516000F05F8341F27D0041F2D43200232F
:10D270005BF802100BF8003041F2791541F2752489
:10D2800041F271308BF831338BF805378BF8D9398F
:10D290008BF8AD3C8BF8813F0BF805300BF8043070
:10D2A0000BF80030069B994201D04BF802307D4BC1
:10D2B0001B680E9341F2F4330E9A4BF803209BF84F
:10D2C0007130002B00F08C809BF86F4034B19BF8DC
:10D2D0002F301BB941F224420BF802309BF870301A
:10D2E00063B19BF830304BB90BF5A051D1ED007A0A
:10D2F000F5EEC07AF1EE10FA40F25D8441F2EC33C3
:10D300005BF80320032A00F0B7839BF86D30002BF5
:10D3100000F094819BF82D20002A40F08F814FF07F
:10D32000FF3341F2D43560485BF80540234403F1F4
:10D330001E0282FB00011144D317C3EB2113C3EB80
:10D340000313A2EB430323EAE3739C424BF805303B
:10D3500003D00BF59F520021D16141F225411BF80A
:10D36000012072B141F2E8324FF435705BF80220CF
:10D3700000FB02B200244FF0FF300BF80140C2F86E
:10D380005C04484A494C12680F920BF59F5641F2D3
:10D39000E435336041F27D0241F2791101334BF8FB
:10D3A000053000230BF8023041F275268BF831333B
:10D3B0008BF805378BF8D9398BF8AD3C8BF8813F6A
:10D3C00041F271350BF801300BF59E5241F2F43108
:10D3D0000F980BF806300BF8053094614BF80100FC
:10D3E00011B0BDE8F08F41F2E8324FF435705BF8D0
:10D3F000022000FB02B200244FF0FF300BF8014086
:10D40000C2F85C04F1E641F28D43C35C002B7FF46B
:10D41000B0AE41F2224190F8722001234354002A19
:10D4200040F0C48341F2D433C6581E2E1CBF1E22C6
:10D43000C25090F8053713B941F27D03C35C9BF8E5
:10D44000D92922B941F279121BF802201A439BF81C
:10D45000AD3C23B941F275231BF8033013439BF80D
:10D46000812F002A40F06C8441F271321BF80220B7
:10D47000002A40F06584002B40F062841E239E4207
:10D480003FF477AE41F2E4300BF59E5341F2D432D3
:10D490000649741C4BF8004099614BF8026068E63D
:10D4A000A82AFF1F80B2FF1F89888888CDCC4C3FF7
:10D4B0000BF58A61054643F250030120E85440F61B
:10D4C0004472AA4806F0ACFA42F64463E8580028D1
:10D4D00000F01A81A64AA74B0A931146A64A059264
:10D4E0001A46083B0293131F06931346A34FDFF817
:10D4F000A4A2DFF8CC92DFF8C482CDF82CB00433BC
:10D5000003930023BB4607930F460A9B07991A68AB
:10D51000099C029B02FB014202EB82025200911C19
:10D520001B68B1FBF3F1814202F1010228BF00F157
:10D53000FF318A180092924A0192009C611CB1FB53
:10D54000F3F2824206D203FB12122346002A08BFDE
:10D550000B460093039B1B6804933E68894D07F0BC
:10D5600015F8044604E007F011F8001BA842F4D8AF
:10D57000D8F80030DB07F6D4834A844B166053603A
:10D5800007F004F87F4C054604E006F0FFFF401B5F
:10D59000A042E2D8DAF800207D4B1340002BF4D0F3
:10D5A0007C4B7C4A1B68CBF800301360DBF8002012
:10D5B000774B72491340012BCFD1774A1268D005BF
:10D5C000CBD589F8003000230B60059B734A1B788C
:10D5D00001991160002B40F08380009B5B026A4838
:10D5E0006F4903606F4A674D4FF481330B606E4B98
:10D5F0006E4911606E4A1A6006F0C8FF044604E0E6
:10D6000006F0C4FF001BA8426CD899F80030002B2C
:10D61000F6D1DBF80020654B1340022B62D1009A53
:10D62000019B01320092634A03F500739342019318
:10D6300060D0029B069A1B6810687EE79BF86E20FC
:10D640003AB19BF82E2022B9002B40F070830123C1
:10D6500067E694BB9BF82F307BB341F224431BF861
:10D66000033053BB41F2284141F2264241F22743A5
:10D670000BF8014058460BF802400BF80340F6F750
:10D680003DFD41F2EC3341F2F0325BF803104BF810
:10D69000021041F2294541F22A4041F22B4141F268
:10D6A0002C4203264BF803600BF805400BF80040B2
:10D6B0000BF801400BF8024092E60BF5A052D2EDB8
:10D6C000007AF5EEC07AF1EE10FA7FF789AE92EDAE
:10D6D000037A77EEC77AC2ED007A11B0BDE8F08F19
:10D6E000009B7CE7049840F2FD12322106F03EF8E0
:10D6F000002894D1069B1868079B01339842079332
:10D700003FF603AFDDF82CB041F2D43341F27D0592
:10D7100041F2791441F2752041F271315BF8032036
:10D7200000230BF805308BF831338BF805378BF875
:10D73000D9398BF8AD3C8BF8813F0BF804300BF8EE
:10D7400000300BF80130089B93427FF42DAD30E59B
:10D75000194B01931A4644F25043D35C002B3FF41B
:10D7600028AD0BF58A611546A5E600BF0C5BFF1FCF
:10D770006CB2FF1FF058FF1F58B2FF1F64B2FF1FAB
:10D78000F85AFF1F40420F0008100B4000001A0D0E
:10D7900001000F0030100B4010100B4000100B4028
:10D7A00004100B4038100B400C100B4002007F118E
:10D7B00001003A18F86EFF1FA82AFF1F24100B4023
:10D7C00068B2FF1F0C4642F6446201F53951084623
:10D7D00003EB83030291A1580268914FDFF864A222
:10D7E000DFF88C928F4ECDF81CB05B00981CB0FB1C
:10D7F000F2F0884228BF01F1FF300133C3180093D3
:10D80000894B04931846894B1C46894B0593134654
:10D81000A0F501720392B846A346009C601CB0FBC1
:10D82000F3F2914206D903FB12022346002A08BFF5
:10D8300003460093039B1B680893DBF800707D4D43
:10D8400006F0A4FE044604E006F0A0FE001BA84279
:10D85000F3D83368D907F7D4774A784B1760536009
:10D8600006F094FE734C054604E006F08FFE401B64
:10D87000A042E2D8DAF80020714B1340002BF4D01C
:10D88000704B704A1B68C8F800301360D8F800204D
:10D890006B4B63491340012BCFD16B4A1268D20501
:10D8A000CBD589F8003000230B60059B674A1B78B5
:10D8B00004991160002B33D1009B5B025E486449E0
:10D8C0000360644A5B4D4FF481330B60624B6349E4
:10D8D0001160634A1A6006F059FE044605E006F03E
:10D8E00055FE001BA84200F28D8099F80030002BF5
:10D8F000F5D1D8F80020594B1340022B40F082801C
:10D90000009A049B01320092564A03F500739A4232
:10D91000049300F08881544A029B11681B687CE7DD
:10D92000009BCBE70026DFF84C914FF0000835460E
:10D930005C464FF4D172002104F58C6008F0FEFBC8
:10D94000D122002104F2026008F0F8FB202200211D
:10D9500004F5E16008F0F2FB04F2D463012704F55A
:10D96000DB614FF0FF324148C4F85C24C4F85454E2
:10D97000C4F8585484F80276342218609C2304F2C8
:10D98000DC60C1F800904FF07A5EC4F8EC26C4F871
:10D99000E426C4F8F036C4F8E83604F5DC6204F294
:10D9A000F463C0F800E04FF07D5106F6A4701160FA
:10D9B0005844C3F80080D12284F80477C4F8F8569C
:10D9C000C4F8FC56C4F8005784F8055784F8065785
:10D9D00084F80757002108F0B1FB06F584500021B8
:10D9E0005844202208F0AAFB0BEB060303F58351F1
:10D9F000FC36B6F57C7F04F535748D610F774D7775
:10DA000097D130E4089840F2DD12312105F0AEFEE6
:10DA100000287FF475AFDDF81CB0FFF7EFBB00BF47
:10DA200064B2FF1F24100B40F85AFF1F6CB2FF1F97
:10DA300058B2FF1F40420F0008100B4000001A0DA3
:10DA400001000F0030100B4010100B4000100B4075
:10DA500004100B4038100B400C100B4002007F11DB
:10DA600011003A11F86EFF1FEC58FF1F0000A04094
:10DA700068B2FF1FCDCC4C3E4CB99BF82F2032B181
:10DA800041F224421BF80220002A00F001819BF899
:10DA90005930A3B19BF8190088B941F22A4341F2E9
:10DAA00029441BF80310002900F0FA8041F22B41B1
:10DAB00001220BF803000BF804200BF80120BBF83F
:10DAC0004030BBF80040BBF84220BBF802009BF896
:10DAD0006D101B1B121A1BB212B219B19BF82D103C
:10DAE00001B9013B9BF86E1019B19BF82E1001B9DA
:10DAF000013303B902B31344002B40F3DB8001234D
:10DB000041F2D435D2485BF80540234403F11E02AC
:10DB100082FB00011144D317C3EB2113C3EB0313A2
:10DB2000A2EB430323EAE3739C424BF8053003D096
:10DB30000BF59F530022DA619BF857300BF5A0528A
:10DB4000002B6DD09BF81730002B69D1D2ED007AF5
:10DB5000F5EEC07AF1EE10FA71D99BF85B3043B163
:10DB60009BF81B0028B9F5EEC07AF1EE10FA40F2EE
:10DB7000A680F5EEC07AF1EE10FA7FF731AC0BF526
:10DB8000A05393ED037A77EEC77AF5EEC07AF1EE03
:10DB900010FAC2ED007A3FF623AC41F2F03241F2C6
:10DBA000EC335BF802204BF8032019E441F22D42DC
:10DBB0008354FFF7DEBA41F2D43241F2DC365BF82F
:10DBC00002208BF8313341F2E4358BF805378BF8BE
:10DBD000D9398BF8AD3C8BF8813F4BF8062041F2E8
:10DBE000244601324BF8052001220BF8062041F2B1
:10DBF0007D0541F279120BF80530964C0BF8023096
:10DC0000954841F2752641F271350BF59E520BF89D
:10DC100006300BF805309461086011B0BDE8F08F54
:10DC2000D2ED007A99E743F25003019ADDF81CB077
:10DC3000D35C002B40F001810123FFF7E0BA41F2F1
:10DC4000D43041F2DC315BF800609FED847A8BF8D0
:10DC500031338BF805378BF8D9398BF8AD3C8BF81D
:10DC6000813F41F27D054BF8016041F2791441F2A8
:10DC7000752041F271310BF80530F0EE477A0BF860
:10DC800004300BF800300BF8013082ED007A76E7B3
:10DC900041F2F0325BF802204BF80320FFF7A0BB03
:10DCA00041F22C4001220BF804100BF800200BF875
:10DCB000032004E714BF4FF0FF33002320E741F2B5
:10DCC00025411BF801306BB141F2E8334FF4357454
:10DCD0005BF803300BF8010004FB03B34FF0FF3196
:10DCE000C3F85C1441F2D4360BF59F535BF8066021
:10DCF0001E6041F27D0541F2791441F2752041F236
:10DD0000713100230BF80530DFED547A8BF8313395
:10DD10008BF805378BF8D9398BF8AD3C8BF8813F00
:10DD20000BF804300BF800300BF8013027E79BF8B4
:10DD30002D30002B14BF01234FF0FF33FFF7F1BA52
:10DD4000474C44F250430BF58A61E35C002B3FF4EF
:10DD500095AB43F250030125E55440F64472414827
:10DD600005F05EFE42F64463E158002944D03E4B84
:10DD7000181D1A1F039004F5395002900027904691
:10DD80009946D9F80030029ADFF8E0A0126803FB48
:10DD900007F31E3303EB83035B009C1CB4FBF2F41C
:10DDA0008C4203F1010328BF01F1FF341C441046EB
:10DDB0000AF5A05505E0AA4519D0029BD8F8001035
:10DDC000186804F1010EBEFBF0F38B4252460AF5CF
:10DDD000007A04D200FB13E3002B08BF7446039BB8
:10DDE00021461868FEF7BAFF01340028E3D1D8F8BD
:10DDF00000100137B942C4D841F27D0541F27914CF
:10DE000041F2752041F2713141F2D43200230BF816
:10DE100005308BF831338BF805378BF8D9398BF80F
:10DE2000AD3C8BF8813F0BF804300BF800300BF859
:10DE300001305BF80230FFF722BB40F6447209491B
:10DE40000BF58A6005F0ECFD0023FFF7D8B900BFA1
:10DE500089888888CDCC4C3FCDCC4C3ECDCC4C3E37
:10DE6000A82AFF1F0C5BFF1FF058FF1FF85AFF1F67
:10DE7000F8B590F87B200446002A51D0FE2A00F025
:10DE80007781531E03F0FE03FE2B00F07B81D12B24
:10DE900000F37A81A92B00F37981872B00F3788135
:10DEA000692B00F37D81512B00F37C813D2B00F326
:10DEB0007B812B2B00F37A811F2B00F37981152BAB
:10DEC00000F378810D2B00F37781092B00F3768125
:10DED000052B00F38381032B00F38281012BD4BF38
:10DEE00000230123D20700F1C280D94381EAE17205
:10DEF000A2EBE172531E002A00F04181B04A52F8B1
:10DF00002330002943F0010240F33381DBB243F0B8
:10DF10000103D2B241F2884041F28441225463505D
:10DF200041F28942A15C002963D194F85C30184623
:10DF3000002B5DD094F85900002859D041F28A4551
:10DF400001206155A0549F4D53B994F859303BB905
:10DF500094F85B3023B994F85730002B00F0FF8021
:10DF6000B4F842206088B4F84030218894F85560B5
:10DF7000101A591A00B209B2002E00F0BA80637D5F
:10DF8000002B40F0B68004F5A4528F4B1678013672
:10DF900083FB0673A3EBE67303EB4303A6EB430398
:10DFA000137094F871302F78002B40F0B18004F595
:10DFB000A4521378012B03F1010305D813701378D1
:10DFC000012B03F10103F9D911B9002800F0B58044
:10DFD0000144002940F3AC80012604F5A4531B78CA
:10DFE000052B00F2AA80DFE803F07E736C655C44C9
:10DFF000F8BD41F28A43E35C1BB394F8593023BB6C
:10E00000627E12B36F4D714E95E8070041F2894769
:10E0100041F28A4E0023E35504F80E3086E80700EB
:10E02000DFF8B4E142F64C6219465EF80200A6F150
:10E030001402FEF793FEE05D0028D9D094F85C301E
:10E0400082E794F85C305F4D7EE794F85B2012B96C
:10E05000E27E002AD6D194F8572012B9E27D002A38
:10E06000D0D194F85C20002A69D0564D78E7591C2D
:10E0700044E741F28443E058F8F7EEFD801965D09B
:10E080000F28C8BF102640F3B280FF23002E40F3B4
:10E09000A98041F2844141F288426350A354012097
:10E0A000F8BD012E2B7975D1052B5DD900232B717D
:10E0B0000120F8BDAB78334403F00303AB700120BB
:10E0C000F8BD6B78334403F001036B700120F8BD99
:10E0D000EB781E44122EDABF26EAE676F3B213235B
:10E0E000EB700120F8BDF31903F003032B7001203E
:10E0F000F8BD94F85630002B3FF453AFA37D002BAE
:10E100003FF441AF94F871302F78002B3FF44FAFBC
:10E11000022F3FF459AF04F5A45202261378012BC5
:10E120007FF452AF16701378012B7FF44DAFF9E7EF
:10E1300014BF4FF0FF3600264FE70120F8BD227FC5
:10E14000002A7FF45FAF1F4D01E7064686EAE673BB
:10E15000A3EBE6735A1E002B4FD1012396E741F241
:10E160008A430122E254FBE6194A12F823309EE763
:10E17000FF220132FE2A46DCD2B21346CAE602234F
:10E180001A46C7E60F23ADE60E23ABE60D23A9E63C
:10E190000C23A7E6052B89D80E4A12F8233086E710
:10E1A0000B239FE60A239DE609239BE6082399E6B5
:10E1B000072397E6062395E6052393E6042391E6D5
:10E1C000C4B30100BC14FF1FABAAAA2A0C59FF1F3D
:10E1D000C4AD01009CB80100A82AFF1F032381E6FB
:10E1E00002237FE60133FE2BA8BFFE2351E710F187
:10E1F0000F0FAADA6FF00F0647E7044B53F82230EF
:10E2000043F0010342E7FE231A4683E6C4B301004C
:10E2100041F22D4290F8753000212DE9F047044677
:10E22000815423B990F87430002B00F00D8241F234
:10E230001C4341F28C42E35C0021A154002B40F0CE
:10E24000408241F21D46A35D002B40F01082012167
:10E2500041F29343E25C002A7ED041F21F4294F8DF
:10E2600055300121A154002B40F0268294F85630FD
:10E27000002B40F0218294F85730002B40F01C8294
:10E2800094F85930002B40F0178294F85B30002B43
:10E2900040F0128294F85C30002B40F00D8294F82C
:10E2A0005D30002B40F0088294F85E30002B40F087
:10E2B000038294F85F30002B40F0FE8194F86130C7
:10E2C000002B40F0F98194F86230002B40F0F4818B
:10E2D00094F86330002B40F0EF8194F86430002B09
:10E2E00040F0EA8194F86530002B40F0E58194F825
:10E2F0006630002B40F0E08194F86730002B40F04E
:10E30000DB8194F86830002B40F0D68194F86F30B0
:10E31000002B40F0D18194F85830002B40F07485E8
:10E32000226C23689A4240F0C781B4F84620E38803
:10E330009A4240F0C181A26CA3689A4240F0BC812D
:10E34000B4F84C20A3899A4240F0B68141F293433D
:10E350000022E254BDE8F08741F28C42A05C002824
:10E3600000F0DC8194F85530002B40F0258294F8C1
:10E370005630002B40F0208294F85730002B40F0AC
:10E380001B8294F85930002B40F0168294F85B30D1
:10E39000002B40F0118294F85C30002B40F00C828E
:10E3A00094F85D30002B40F0078294F85E30002B2B
:10E3B00040F0028294F85F30002B40F0FD8194F829
:10E3C0006130002B40F0F88194F86230002B40F06F
:10E3D000F38194F86330002B40F0EE8194F86430C0
:10E3E000002B40F0E98194F86530002B40F0E48187
:10E3F00094F86630002B40F0DF8194F86730002BF2
:10E4000040F0DA8194F86830002B40F0D58194F820
:10E410006F30002B40F0D08194F85830002B40F042
:10E42000CB8141F2EC33E358002B00F0CF81012B7C
:10E4300000F0E081022B00F02082032B00F0278403
:10E4400041F28F43E35C5BBB94F869307BB194F895
:10E45000293063B904F59E5241F264451078AE4EFE
:10E4600004F5A35180F0010010700E60635194F820
:10E470006530ABB994F8252092B194F86120002A58
:10E4800040F0658494F8293053B9D4F800375B42E2
:10E49000002B08BF01230122C4F8003784F80527A8
:10E4A00041F29043E35C63BB94F86A3083B194F823
:10E4B0002A306BB941F2C13141F26440625C964E40
:10E4C00004F5A35382F00102012562541E60255019
:10E4D00094F86630ABB994F8262092B194F8622093
:10E4E000002A40F0E78394F82A3053B9D4F8D4399D
:10E4F0005B42002B08BF01230122C4F8D43984F801
:10E50000D92941F29143E35C63BB94F86B3083B14A
:10E5100094F82B306BB941F2C23141F26440625C35
:10E520007D4E04F5A35382F00102022562541E6061
:10E53000255094F86730ABB994F8272092B194F83D
:10E540006320002A40F0E98394F82B3053B9D4F8C3
:10E55000A83C5B42002B08BF01230122C4F8A83C61
:10E5600084F8AD2C41F29243E35CC3B994F86C306B
:10E5700083B194F82C306BB941F2C33141F264405D
:10E58000625C654E04F5A35382F0010203256254D8
:10E590001E60255094F86830002B00F0868194F8B6
:10E5A0005C301BB1237F002B00F038822046FEF741
:10E5B000D5FD41F2EC33E258012A1ED041F225414B
:10E5C00041F22647605C41F2284641F2274500238C
:10E5D000E355A355635558B141F2E8304FF4357512
:10E5E0002058635405FB00434FF0FF31C3F85C141F
:10E5F000022A02D02046F5F727FE94F855301BB1C9
:10E60000637D002B00F04D8194F8052712B941F28B
:10E610007D03E25C94F8D9391BB941F27913E35CCC
:10E62000134394F8AD2C1AB941F27522A25C1A4337
:10E6300094F8813F1BB941F27133E35C134341F21B
:10E640001F42A354BDE8F08741F21C42825CAABB82
:10E6500041F21D43C35C2BB941F28943C15C0029DF
:10E660003FF4F6AD41F28C430022E254E9E504F5B3
:10E67000A05520460435FEF771FDD5ED007A41F234
:10E68000104141F21C43F5EEC07A4FF0FF300022FA
:10E69000F1EE10FA6050E25440F34F8104F5A053BC
:10E6A00093ED037A77EEC77AF5EEC07AF1EE10FAC1
:10E6B000C5ED007A40F22681BDE8F08741F28C4238
:10E6C000835404F5A05520460435FEF747FDD5EDEB
:10E6D000007A41F2104141F21D43F5EEC07A4FF04D
:10E6E000FF300022F1EE10FA6050E25430DD04F504
:10E6F000A05393ED037A77EEC77AF5EEC07AF1EE88
:10E7000010FAC5ED007AD7D841F21C4141F21E4300
:10E710006254E254BDE8F087CDCCCC3E00297FF4B2
:10E7200080AE94F85F1000293FF47BAEE17F0029B2
:10E730007FF477AE41F28E41615C00297FF471AEC7
:10E7400041F21F4001212154A154E154BDE8F0875A
:10E7500041F21E4394F85510E254002900F0D8808D
:10E7600094F85930002B40F01181637E002B00F0AB
:10E770000D8141F2144341F21842E358A2584FF47C
:10E78000357141F21E4001FB03430226265401FB72
:10E79000024403F2D46004F2D4620168116003F50C
:10E7A000DB6304F5DB6219681160012384F8053727
:10E7B000984B2B60BDE8F08741F28C4141F29343C6
:10E7C000002001226054E254BDE8F0872046FFF7A4
:10E7D0004FFB002800F00D8294F97930002B04DA09
:10E7E00094F97A30002BFFF667AF2046FEF7B6FCAF
:10E7F000BDE8F08794F858300BB1237ECBB194F884
:10E800005D300BB1637FA3B194F85A300BB1A37E96
:10E810007BB194F8603013B194F820304BB194F888
:10E820005C30002B7ED1237F002B7BD0637F002BBD
:10E8300078D141F22643E35C002B70D141F22843AA
:10E84000E35C002B6BD141F22E43E35C002B66D1DD
:10E8500041F22F43E35C002B61D141F23243E35C90
:10E86000002B5CD141F22E43E35C33B941F22F43DC
:10E87000E35C13B92046F5F7E1FD204641F22E4551
:10E88000F6F72EF82046F6F751F9635D43BB41F2E7
:10E890002F46A35D002B00F004822046F6F794FC7F
:10E8A00026E041F22242A354AEE694F82820002A42
:10E8B0003FF475AE94F86420002A40F0148294F876
:10E8C0002C30002B7FF46BAED4F87C3F5B42002BE6
:10E8D00008BF01230122C4F87C3F84F8812F5EE643
:10E8E0002046F6F751FA41F22F43E35C002BD4D1D6
:10E8F0002046F6F78DFF2046F7F77AFA2046F8F71C
:10E900003FF89DE541F21E43A255E254BDE8F08771
:10E91000627D002A3FF424AF0122E25448E72046FA
:10E92000F5F792FC41F22643E35C002BA5D141F2BE
:10E930002843E35C002BA0D194E741F21E4394F8F6
:10E940005510E25411B9627D002AE5D194F859308E
:10E95000002B40F0CB80637E002B00F0C78041F29B
:10E9600018434FF43572E3582A482B4F02FB0343F8
:10E9700041F21E420221A15403F2D46603F5DB6189
:10E9800001223760086083F8052711E794F85730B3
:10E99000002B40F0FD80E37D002B00F0F98041F278
:10E9A000184841F2144354F80860E1584FF43572A6
:10E9B00002FB06F041F21E4704EB000E042302FBAB
:10E9C0000141E3550EF254400EF2D46C01F2544171
:10E9D0000EF5DB6E8842DCF800A0DEF8009004D073
:10E9E00005F01EF854F80860E35D4FF4357202FB41
:10E9F000064404F2D46004F5DB610122C0F800A0F3
:10EA0000C1F8009084F80527002B7FF4D1AEBDE853
:10EA1000F08700BFCDCC4C3E0000A04094F86130A0
:10EA2000ABB141F2780341F22141E2580123002ABF
:10EA300063540CDD41F27C0141F27D05625C63555B
:10EA400004F5A053CF4882F001026254986094F814
:10EA50006230ABB141F2741341F22141E25801231B
:10EA6000002A63540CDD41F2781141F27915625CA1
:10EA7000635504F5A053C34882F0010262549860C4
:10EA800094F86330ABB141F2702341F22141E25876
:10EA90000123002A63540CDD41F2742141F27525F3
:10EAA000625C635504F5A053B64882F001026254DB
:10EAB000986094F86430002B3FF478AD41F26C33E9
:10EAC00041F22141E2580123002A63547FF76EADE1
:10EAD00041F2703141F27135625C635504F5A05327
:10EAE000A84882F00102625498605FE594F85730BC
:10EAF0001BB9E37D002B40F0478194F85B301BB9D4
:10EB0000E37E002B40F0678194F85660002E7FF47E
:10EB1000D3ADA37D002B3FF4CFAD41F2184741F2B6
:10EB20001E42E3594FF4357101FB03401021A154FB
:10EB300000F25440F5F73AF9E359C3EB831304EBC1
:10EB4000830000F6A470F5F7C3FAE359C3EB83130F
:10EB500004EB830341F27D0001271F5441F226425A
:10EB600041F2274341F2284120466654A654E65418
:10EB7000F5F76AFB41F2EC3241F2F033A750E7506F
:10EB800041F21E43E35C002B7FF412AEBDE8F08738
:10EB900094F85B30A3BBE37E93B341F2184641F295
:10EBA000144354F806E0E3584FEA8E12C3EB831384
:10EBB000CEEB020004EB830104EB800041F21E4720
:10EBC00000F6A47001F6A47108238842E35507D02B
:10EBD000FC2204F025FF54F806E0E35D4FEA8E12B4
:10EBE000CEEB020204EB820441F27D020121A1542A
:10EBF0000AE72046F5F774FE2046F5F797FF1FE475
:10EC000094F85630002B7FF457ADA37D002B3FF4D2
:10EC100053AD41F2184841F2144754F80860E359E3
:10EC20004FF4357202FB064002FB034141F21E4ED7
:10EC300000F2544001F254414FF0100C884204F8A5
:10EC40000EC004D004F0ECFE54F80860E359B201A1
:10EC5000C3EB8313901B04EB830104EB800001F6EC
:10EC6000A47100F6A470884206D0FC2204F0D8FEFD
:10EC700041F21843E658B201931B04EB830341F2BF
:10EC80007D020121995441F21E43E35CBCE620461B
:10EC9000F5F726FE41F210434FF0FF32E250FFF746
:10ECA000CFBB2046F6F79EFB635D002B7FF418AECA
:10ECB000A35D1BE641F210424FF0FF31A15041F23B
:10ECC000144741F2184641F21D4541F21C4004F53B
:10ECD000A1510122E251A2516255235420460A70EB
:10ECE000F5F7B2FA0DE441F2104241F214414FF04F
:10ECF000FF30A05041F21847032041F21C4641F278
:10ED00001D4504F5A15260500121E051A355204654
:10ED100061551170F5F798FA41E441F2104241F261
:10ED200014414FF0FF30A05041F21847022041F249
:10ED30001C4641F21D4504F5A15260500121E051ED
:10ED4000A355204661551170F5F77EFA0AE441F2A9
:10ED500010424FF0FF31A15041F2144741F21846E2
:10ED600041F21C4541F21D4004F5A1520121E3513D
:10ED7000A3516355215420461170F5F765FAFFF74A
:10ED80008FBB00BFCDCC4C3E41F218474FF43576D7
:10ED9000E35941F21E4106FB03F3E21804206054DC
:10EDA00002F2D46302F2544002F5DB62D3F8009021
:10EDB000D2F80080F4F7FAFFE35906FB034303F2AD
:10EDC000D46003F5DB610122C0F80090C1F8008037
:10EDD00083F80527D4E641F2184641F21E42A359B2
:10EDE000C3EB831304EB83000823A35400F6A47041
:10EDF000F5F76EF9A359C3EB831304EB830341F2D8
:10EE00007D0201219954BBE6BDE8F0872DE9F04F62
:10EE100086460D46BEE80F00CA4CDFF844B39FEDAE
:10EE2000CA7ADBF8006004F140070FC7BEE80F00A4
:10EE30000FC797B041F2F838BEE80F001096109E49
:10EE400054F808C00B9644F80860CCEB060607EEB1
:10EE5000906A0FC7F8EE677ADFF808C367EE877A23
:10EE6000F7EE006ACCED047A9EE80F009CED007A84
:10EE700037EE877A87E80F00B4EEE67AF1EE10FA03
:10EE800005DBFDEEC76AF8EEE66A37EE667AAF4B51
:10EE90008CED007ADFEDAE6A93ED007AB4EEE67A9F
:10EEA000F1EE10FA0ADD37EE677AB4EEE67AF1EEAB
:10EEB00010FA48BFB0EE667A83ED007AA54BDFED1D
:10EEC000A46A93ED007AB4EEE67AF1EE10FA0ADD68
:10EED00037EE677AB4EEE67AF1EE10FA48BFB0EE9C
:10EEE000667A83ED007A9C4B93ED007AB5EEC07A9A
:10EEF000F1EE10FAC4BF77EE677AC3ED007A974B54
:10EF00001A79013AD2B2042A06D841F232438D4925
:10EF1000E35C002B00F0CD8441F26843B4F8442058
:10EF2000E3580C92D31A002BB8BF5B4241F249223E
:10EF30009342D4BF002301230A9394F855200192F1
:10EF4000134694F8159094F85620009294F85710B0
:10EF500094F81680029183EA0909009B94F85900FD
:10EF600094F817C0039083EA0808029B94F85B703A
:10EF700094F819E0049783EA0C0C039B94F85C2046
:10EF8000E77E059283EA0E0E049B94F86110207FC1
:10EF900006915F40059B94F8626094F821100796F3
:10EFA00049EA080848EA0C085840069B94F8636050
:10EFB00094F822200D9648EA0E0894F823C094F89D
:10EFC00024E094F8689048EA0708594094F864707F
:10EFD000079B08975A4048EA000094F86570089B20
:10EFE0000997014386EA0C0C114383EA0E0E94F84C
:10EFF0002570099B94F8662094F8260094F86760C1
:10F000000E9241EA0C0141EA0E0E5F4094F827C0CF
:10F010000A9B0F9650404EEA0707384386EA0C01D8
:10F02000014341F2EC3094F8282054F800A089EA1A
:10F0300002020A43BAF1030F43EA0203414A0BD129
:10F0400092F86D7092F82D1092F86E0092F82E20C2
:10F050007940424011430B4394F86F2094F82FC03D
:10F0600094F8351094F875E094F876800A9210467A
:10F0700094F836208EEA010E80EA0C004EEA000C6D
:10F0800088EA0207B4F8400021886288B4F8468014
:10F090004CEA0707B4F842C088420CBFBE4647F0AE
:10F0A000010EE78894450CBF70464EF00100B4F89D
:10F0B00008E0B4F848C0B8450CBF014640F0010173
:10F0C000B4F84A706089F4450CBF0A4641F0010269
:10F0D000B4F84CE0A189874218BF42F001028E4586
:10F0E00018BF42F00102002A40F0AD82002B40F030
:10F0F000AA8241F22343134EE35C002B40F0E582E9
:10F100003046FFF785F841F2EC3396F8552056F873
:10F1100003A096F8563001920093114629B994F84D
:10F120005E30084A002B00F0C083009929B994F89A
:10F130005F30044A002B00F0B48394F86530014A34
:10F14000BBB911E0CC14FF1F6F12833AD428FF1F04
:10F15000000000002C29FF1F0029FF1FBC14FF1F07
:10F1600080B2FF1FC828FF1F92F86930002B00F003
:10F17000948394F86630C44A23B992F86A30002B1D
:10F1800000F0878394F86730BF4A23B992F86B3058
:10F19000002B00F07A8394F86830BB4A23B992F8C8
:10F1A0006C30002B00F06D83B74C04F140070FCF9B
:10F1B00026460FC60FCF0FC60FCF0FC697E80F001A
:10F1C00041F2DC3EFF2786E80F00AF75EF7554F87B
:10F1D0000E30002B04DB4FF0FF32AB7544F80E20ED
:10F1E000AA4B1A68002A03DB4FF0FF31EA75196059
:10F1F00041F2E8330AF1FF300128E358A24A40F215
:10F200008F8300232B7092F861102B72994214BFE8
:10F21000022119466B70297192F862106B72994243
:10F2200014BF02211946AB70697192F86310AB727A
:10F23000994214BF02211946EB70A97192F864201B
:10F24000EB729A4218BF0223EB7141F22D4394F8FE
:10F250007820E35CEA7613B182F00103EB7641F2A9
:10F26000884341F28C41E65C2E76615C0026E654D0
:10F27000854B29B141F2B841595CB1FA81F1490994
:10F280000023BAF1010F85F821102B772B736B73D4
:10F2900000F0318341F22E41AB73615C39B1DBF890
:10F2A00000301593159BDBB2802B40F2B581BAF18B
:10F2B000010F00F0B781002641F23043EE73E65CA7
:10F2C000714B2EB141F23147DB5D002B40F0A28241
:10F2D000002301282B746B74AB7440F2AD826C4B2D
:10F2E00093ED007A93EDB56AF2EE047A03F5B5601A
:10F2F000D0ED006A03F67C03B4EEE77AF1EE10FA83
:10F3000093ED007AB4EEE76A4CBF01230023F1EEDF
:10F3100010FAF4EEE76A4CBF4FF0010E4FF0000E0A
:10F3200041F22B47F1EE10FAB4EEE77A6B7741F237
:10F330002C404CBF01230023F1EE10FA85F81EE0AB
:10F34000EB7748BF4FF0010EE35D58BF4FF0000E62
:10F3500085F820E014F800E06B76002385F81AE0C9
:10F36000E3552354EB742B7594F8733085F82260C1
:10F3700053B1DBF800301393139BC3F30803B3F5C9
:10F38000807F94BF0023012342486B75D0ED007A43
:10F39000F5EEC07AF1EE10FA0DDDB2EE0E7A67EE00
:10F3A000877AFDEEE77A17EE903A13F0010F14BF5B
:10F3B000002302236B75384BD3ED007AF5EEC07A4B
:10F3C000F1EE10FA0DDDB2EE0E7A67EE877AFDEE01
:10F3D000E77A17EE903A13F0010F14BF00230323CE
:10F3E0006B7341F22F4314F803E0BEF1000F09D014
:10F3F000DBF800301293129BDBB2802B8CBF03230F
:10F4000000236B7394F872701F4BC7B993F80567AC
:10F41000002E00F0DC8194F8D9091B4B002800F085
:10F42000CB8194F8AD3C184E002B00F0BA8194F8D3
:10F43000810F154E002800F0AA8101232B73DBF801
:10F4400000301193119894F80537DFF83CC0C0F3F1
:10F4500008061BB941F27D031CF8033094F8D90962
:10F46000DFF824C020B941F279101CF800001843DD
:10F4700094F8AD3CDFF810C083B941F275231CF855
:10F48000033003430AE000BFCC14FF1FAC28FF1F6A
:10F49000A01BFF1FCC28FF1FD428FF1F94F8810F4B
:10F4A000DFF844C3002840F0C58041F271301CF8F9
:10F4B00000000343002F00F0A581002A00F0C08067
:10F4C000002B40F00A8301202873BEF1000F04D105
:10F4D00019B941F23243E35C1BB100232B746B7406
:10F4E000AB74C04BC04AD3ED007AF5EEC07AF1EEB2
:10F4F00010FA0BDD93ED0D7A77EEC77AF5EEC07A50
:10F50000F1EE10FAC3ED007A40F2E18241F270426E
:10F51000B54BA15C00297CD041F2D431002558586C
:10F520009D541E281CBF1E225A5041F22543AE4A4C
:10F53000E15C61B141F2E8314FF43570515800FBA4
:10F54000012100254FF0FF30D554C1F85C0444F28E
:10F550005043A64AD35C002B40F017820321D4F815
:10F56000FC36D4F8D029002BC4BFA14B1868A14B9E
:10F57000D8BF4FF07E50002A1860C8BFA3F6E8132A
:10F58000D4F8A42CC8BF18689B4BD8BF4FF07E504E
:10F59000002A1860C8BFA3F5E363D4F8782FC8BF6A
:10F5A0001868964BD8BF4FF07E50002A1860CABF2B
:10F5B000A3F589634FF07E521A68914B01291A60B6
:10F5C00000F0E08241F27D0041F2D4320023235466
:10F5D00041F2791641F2752541F27130A158824FFE
:10F5E00084F8313384F8053784F8D93984F8AD3C90
:10F5F00084F8813FA3556355235401B1BB5041F2B8
:10F60000E43141F268434FF0FF30B4F844206050D9
:10F61000E25017B0BDE8F08F0023BAF1010FAB73D1
:10F620007FF449AE41F22643E35C002B0CBF002679
:10F63000022641E6002F00F0E680002A40F04D82CD
:10F6400000232B7341E741F27C4241F271430B9856
:10F65000A050E15C0C9E644A41F2684026500029AB
:10F660003FF447AD92F865100020D054002940F0D7
:10F670003B820B4694F866205B4922B191F8262024
:10F68000002A08BF012394F86720574922B191F856
:10F690002720002A3FF42DAD94F86820524922B16A
:10F6A00091F82820002A3FF424AD002B7FF421ADEF
:10F6B0004D4E06F140070FCF0FC60FCF0FC60FCF2D
:10F6C0000FC697E80F0086E80F009DE80C00134373
:10F6D000029A94F85F1094F86A0094F86B6094F8BA
:10F6E0005A8094F860C094F85DE094F869701A4309
:10F6F0001346039A03911A431346049A94F86E1022
:10F7000004901A431346059A94F86D0005961A431F
:10F710001346069A94F86C601A431346079A1A43E4
:10F7200013460D9A1A431346089A1A431346099A28
:10F730001A4313460E9A1A4313460F9A1A4349EA7C
:10F74000020394F85E20029294F8702006920A9ABE
:10F7500094F858901A431346029A1343039A13439A
:10F7600043EA090343EA080343EA0C03049A43EA21
:10F770000E033B431343059A13431E433043069A3B
:10F78000014341F223430A43E2540199C6E441F2A2
:10F790007130305C00287FF450AE002B3FF44FAE48
:10F7A0004BE641F27523F35C0F4E034394F8810F4F
:10F7B00000287FF442AEEAE741F27910185C94F831
:10F7C000AD3C3043084E002B7FF431AEE9E741F207
:10F7D0007D001E5C94F8D909034B00287FF421AE0C
:10F7E000EAE700BFA428FF1FCC14FF1FA82AFF1FB1
:10F7F000A81BFF1F6428FF1F6828FF1F6C28FF1F1E
:10F800007028FF1F23B1B6F5807F94BF0027012722
:10F810002F735AE6DBF800301493149BDBB2802B75
:10F820003FF656AD0023EB7301284FF000032B7415
:10F830006B74AB743FF653AD41F2E8334FF435705F
:10F84000E358B84F00FB0343D3F80007012800F04A
:10F850005B81022800F00A82032800F01E8241F238
:10F860002840385C002800F05081D3F8FC36012B8A
:10F8700000F00382022B00F01B82032B08BF2B74C5
:10F8800043E141F2924153548EE441F29141535489
:10F8900081E441F29041535474E441F28F41535456
:10F8A00067E441F28E43D15447E441F28D43D15491
:10F8B0003BE441F271400B5C0A93002B7FF42CABCC
:10F8C00041F27C47DFF8B4E2CF590B9E5EF822E0AC
:10F8D000B1F844300C93F21B724541F26842CCBF40
:10F8E000012700270F548B507FF727AB41F26C4262
:10F8F0008E50FFF722BB41F228418A4E615C0029FD
:10F900007FF4C8AC41F22643F35C002B40F0AB819E
:10F9100041F22F43F35C002B14BF00230223B9E410
:10F9200000212970002B00F0F78092F861202972E5
:10F930008A420CBF0A460222012B69702A7100F02C
:10F94000DC8094F86220002A0CBF002102210022F2
:10F95000022B69716A72AA7000F0CB8094F8632060
:10F96000002A0CBF002102210022032BA971AA72D8
:10F97000EA7000F0C78094F86430002B0CBF0022BE
:10F9800002220023EA71EB725FE4674A42F64463A5
:10F99000D15802F539534FF497721B68B2FBF3F25A
:10F9A0008A4280F0668102F22D1200925F4ADFF8EF
:10F9B0009C81DFF8CCB1DFF898A15D4F01920394F0
:10F9C000009C601CB0FBF3F28A4206D203FB1202D9
:10F9D0002346002A08BF03460093564BDFF8889160
:10F9E0001B680293544B554D1E6804F0CFFD04462E
:10F9F00004E004F0CBFD001BA842F3D83B68D90714
:10FA0000F7D44F4A4F4B1660C9F8003004F0BEFDE2
:10FA10004A4C054604E004F0B9FD401BA042E1D881
:10FA2000D8F80020484B1340002BF4D0474B474AEE
:10FA30001B68CAF800301360DAF80020424B4449D2
:10FA40001340012BCED1434A1268D205CAD58BF898
:10FA50000030414A00230B60019B13603F4B1B7831
:10FA6000002B40F00D81009B5B0235483C49036050
:10FA70003C4A324D4FF481330B603B4B3B491160A4
:10FA80003B4A1A6004F082FD044605E004F07EFD66
:10FA9000001BA84200F2F6809BF80030002BF5D145
:10FAA000DAF80020314B1340022B40F0EB80009A33
:10FAB000019B013200922F4A03F500739342019398
:10FAC00000F0EE802C4A52F8043C116878E741F2CD
:10FAD000E4334FF0FF31D15018E5B6F5807F8CBF8D
:10FAE000002001202873F0E492F8253083F0010310
:10FAF000C0E5AB71AA72EA703DE702226972A97093
:10FB00006A712BE702223CE7A874BAF1020F04BF26
:10FB100003236B73FFF7E3BB02222B726B702A7116
:10FB20000FE700BFCC14FF1FA82AFF1FF85AFF1FC2
:10FB300024100B40F458FF1F6CB2FF1F40420F000F
:10FB400008100B4000001A0D01000F0030100B4090
:10FB500064B2FF1F10100B4000100B4058B2FF1F83
:10FB600004100B4038100B400C100B4002007F11AA
:10FB700011003A11F86EFF1FEC58FF1F8CAF010007
:10FB800068B2FF1F0027504DDFF850A14FF0000969
:10FB90003E464FF4D172002105F58C6006F0CEFA96
:10FBA000D122002105F2026006F0C8FA20220021CD
:10FBB00005F5E16006F0C2FA4FF0FF31C5F85C14BC
:10FBC00005F2D46305F5DB614FF001083F4AC5F843
:10FBD0005464C5F8586485F802861A60C1F800A01C
:10FBE00034229C2305F2DC61C5F8EC26C5F8E42636
:10FBF000C5F8F036C5F8E8364FF07A5E05F2F463E2
:10FC000005F5DC62C1F800E007F6A4704FF07D5105
:10FC100011602044C3F80090D122002185F80487A8
:10FC2000C5F8F866C5F8FC66C5F8006785F805678D
:10FC300085F8066785F8076706F080FA07F58450AF
:10FC400000212044202206F079FAE31903F58351BC
:10FC5000FC37B7F57C7F05F535758E6181F81C8022
:10FC60004E7796D1AEE40B46FFF714BB01236B74BD
:10FC70004BE701F59672009298E60323AB7444E7D4
:10FC8000009BF2E6029840F2DD12312103F06EFD96
:10FC900000287FF40CAF039C60E401232B7434E74D
:10FCA00043F250030A4A039CD35C23B9012156E472
:10FCB00003236B7429E70749074840F6447203F0B1
:10FCC000AFFE00214BE400BFCC14FF1F0000A0409A
:10FCD000A82AFF1F0C5BFF1F1C19FF1FCDCC4C3E39
:10FCE0002DE9F0439BB00646402200210AA806F009
:10FCF00025FAFF2506F5005701A8232200218DF8DB
:10FD000061508DF862503C4606F018FA06F5195815
:10FD100001238DF81A508DF81B508E4D8DF85D30F3
:10FD200008F10C083837283406F10A0901A90AA895
:10FD3000FFF76CF801A94046F9F7E8FE9DF8251099
:10FD4000C1B139780029F1D1606803689B68AB4282
:10FD500040F0E780F0F7C8FF23681A684FF00041D1
:10FD6000AE23D1625363D36A002BFCDA0123926B7A
:10FD70003B70DBE73B78002B40F0D5804FF48042AE
:10FD80000021754806F0DAF974497548F8F7B8FDAE
:10FD90007449484601F5804E51F8043F4FEA134C30
:10FDA0001A0A0CF4706C22F47F624CEA020203F02F
:10FDB000F00313438E4520F8023FEDD160680368DD
:10FDC0009B68AB4240F0AA80F0F78EFF23681A6868
:10FDD0004FF000411523D1625363D36A002BFCDA44
:10FDE0006068936B03689B68AB4240F09480F0F7C7
:10FDF00071FF23681A684FF000411C23D1625363DE
:10FE0000D36A002BFCDA6068936B03689B68AB4293
:10FE10007ED1F0F75FFF23681A684FF000415B2343
:10FE2000D1625363D36A002BFCDA6068936B03687A
:10FE30009B68AB4269D1F0F757FF23681A684FF00F
:10FE400000417523D1625363D36A002BFCDA6068EA
:10FE5000936B03689B68AB4254D1F0F73BFF236878
:10FE60001A684FF000410023D1625363D36A002B1C
:10FE7000FCDA6068936B03689B68AB423FD1F0F794
:10FE800029FF23681A684FF000413F23D162536372
:10FE9000D36A002BFCDA6068936B03689B68AB4203
:10FEA0002AD1F0F721FF23681A684FF000415C2344
:10FEB000D1625363D36A002BFCDA6068936B0368EA
:10FEC000E6689B68AB4214D1F0F704FF236806F59F
:10FED000FF501A68711E1F304FF0004611F8013FA5
:10FEE000D6625363D36A002BFCDA8842936BF5D158
:10FEF0001CE701219847E9E700219847D3E7012152
:10FF00009847BEE701219847A9E70021984794E761
:10FF1000012198477FE7012198476AE70021984728
:10FF200054E7984718E7606803689B68AB420FD1B5
:10FF3000F0F7DAFE23681B684FF00041AF22D96268
:10FF40005A63DA6A002AFCDA00229B6B3A7015E7E2
:10FF50009847EFE7310C00003070FF1FCC14FF1FF3
:10FF6000D407FF1F2C70FF1F2DE9F0439DB00646FC
:10FF7000402200210CA806F0E1F8FF2423220021F2
:10FF800003A88DF869408DF86A4006F0D7F842F66C
:10FF900058630DF10409002106F500578DF8224041
:10FFA00048468DF82340029101913C46F358914A0E
:10FFB000914D082106F5195806F00EF908F10C08C4
:10FFC000CDF86C903837283406F10A0903A90CA83B
:10FFD000FEF71CFF03A94046F9F798FD9DF82D1088
:10FFE000C1B139780029F1D1606803689B68AB42E0
:10FFF00040F0E780F0F778FE23681A684FF0004180
:020000021000EC
:10000000AE23D1625363D36A002BFCDA0123926BD7
:100010003B70DBE73B78002B40F0D5804FF480420B
:100020000021764806F08AF875497648F8F768FCAA
:100030007549484601F5804E51F8043F4FEA134C8C
:100040001A0A0CF4706C22F47F624CEA020203F08C
:10005000F00313438E4520F8023FEDD1606803683A
:100060009B68AB4240F0AA80F0F73EFE23681A6816
:100070004FF000411523D1625363D36A002BFCDAA1
:100080006068936B03689B68AB4240F09480F0F724
:1000900021FE23681A684FF000411C23D16253638C
:1000A000D36A002BFCDA6068936B03689B68AB42F1
:1000B0007ED1F0F70FFE23681A684FF000415B23F2
:1000C000D1625363D36A002BFCDA6068936B0368D8
:1000D0009B68AB4269D1F0F707FE23681A684FF0BE
:1000E00000417523D1625363D36A002BFCDA606848
:1000F000936B03689B68AB4254D1F0F7EBFD236828
:100100001A684FF000410023D1625363D36A002B79
:10011000FCDA6068936B03689B68AB423FD1F0F7F1
:10012000D9FD23681A684FF000413F23D162536321
:10013000D36A002BFCDA6068936B03689B68AB4260
:100140002AD1F0F7D1FD23681A684FF000415C23F3
:10015000D1625363D36A002BFCDA6068936B036847
:10016000E6689B68AB4214D1F0F7B4FD236806F54E
:10017000FF501A68711E1F304FF0004611F8013F02
:10018000D6625363D36A002BFCDA8842936BF5D1B5
:100190001CE701219847E9E700219847D3E70121AF
:1001A0009847BEE701219847A9E70021984794E7BF
:1001B000012198477FE7012198476AE70021984786
:1001C00054E7984718E7606803689B68AB420FD113
:1001D000F0F78AFD23681B684FF00041AF22D96217
:1001E0005A63DA6A002AFCDA00229B6B3A7015E740
:1001F0009847EFE798B20100310C00003070FF1F04
:10020000CC14FF1FD407FF1F2C70FF1F2DE9F04FE8
:10021000ADB005460590402200211CA805F08EFFD8
:1002200005F53853FF2438332322002113A81E4636
:1002300001938DF8A9408DF8AA4005F07FFF05F5E0
:100240001953194606F50B7205F500530A920A4632
:1002500018460C320992024601233832DFF870B199
:100260008DF862408DF8634006928DF8A7304FF00C
:1002700000040021012341F2EC328DF834408DF866
:1002800035408DF837408DF838400A984D4CADF820
:1002900039108DF83B108DF836300F9405F04EFF75
:1002A000494B019A1B784FF0000182F81812032B7A
:1002B00024D8DFE803F04A793B02019E002206F1D0
:1002C00018040021B2627069ADF8391022468DF829
:1002D0003B10FCF743FDFF23224673620021706947
:1002E0000DADFCF73BFD95E8070033462C3383E862
:1002F0000700224600217069FCF730FD002713A992
:100300001CA8FEF783FD13A90998F9F7FFFB9DF8D8
:100310006D10069B00295DD01978002900F05581E9
:10032000032FA4D038462DB0BDE8F08F2749019B9C
:100330000A681B690892934200F2638100220A60F6
:10034000214A032313700327D9E74FF00003019ECE
:100350008DF840308DF841308DF843308DF84430C1
:10036000184B1293012500214FF000034FF4007247
:1003700006F118003768ADF845108DF847308DF854
:100380004250766805F0DAFE0F4B10AC1D7094E811
:100390000700019D2B4640F282242C33AF61EE61B1
:1003A0002C6283E80700CEE7019B084AD9681368EE
:1003B000994200F2FD8100211160034A022313706B
:1003C000C1E700BF06CBAF428014FF1F7C14FF1FA4
:1003D00024100B401B78002B40F0DA80059BAB4DBE
:1003E00003F5005428344FF480420021A84805F05A
:1003F000A5FEA849A848F8F783FAA849059B01F586
:10040000804603F10A0051F8043F4FEA134E1A0ADE
:100410000EF4706E22F47F624EEA020203F0F003E3
:100420001343B14220F8023FEDD1606803689B6836
:10043000AB4240F0AA80F0F757FC23681A684FF0EF
:1004400000411523D1625363D36A002BFCDA606844
:10045000936B03689B68AB4240F09480F0F73AFCE2
:1004600023681A684FF000411C23D1625363D36A9A
:10047000002BFCDA6068936B03689B68AB427ED10B
:10048000F0F728FC23681A684FF000415B23D16223
:100490005363D36A002BFCDA6068936B03689B6834
:1004A000AB4269D1F0F720FC23681A684FF0004195
:1004B0007523D1625363D36A002BFCDA6068936BB7
:1004C00003689B68AB4254D1F0F704FC23681A68B8
:1004D0004FF00043D36200235363D36A002BFCDA4E
:1004E0006068936B03689B68AB423FD1F0F7F2FB07
:1004F00023681A684FF000413F23D1625363D36AE7
:10050000002BFCDA6068936B03689B68AB422AD1CE
:10051000F0F7EAFB23681A684FF000415C23D162D0
:100520005363D36A002BFCDA6068936B0368E66858
:100530009B68AB4214D1F0F7CDFB236806F5FF5161
:100540001A681F31013E4FF0004016F8013FD0629B
:100550005363D36A002BFCDAB142936BF5D1DFE62B
:1005600001219847E9E700219847D3E701219847FF
:10057000BEE701219847A9E70021984794E70121A8
:1005800098477FE7012198476AE70021984754E799
:10059000059B3E4D03F500542834606803689B6852
:1005A000AB4240F01581F0F79FFB23681B684FF0CA
:1005B0000041AF22D9625A63DA6A002AFCDA9B6BE7
:1005C000069B4FF000021A700DE7059B2F4D03F5B7
:1005D00000542834606803689B68AB4240F0FA809E
:1005E000F0F782FB23681B684FF00041AE22D9620E
:1005F0005A63DA6A002AFCDA9B6B069B01221A70A6
:100600008EE6019C1046E26801300860002A3FF443
:100610009AAE0599224FDFF890A0DFF89080DFF8BE
:10062000909001F588415031049104F506710B91C9
:1006300000210791089803FB010101EB8101019B57
:100640004900881C9B68B0FBF3F0904228BF02F180
:10065000FF300131411810460B9A00910292009C24
:10066000611CB1FBF3F2824206D203FB1212234655
:10067000002A08BF0B460093019B5B690393DAF8DD
:100680000060084D03F082FF044618E0310C0000C2
:100690003070FF1FCC14FF1FD407FF1F2C70FF1FEB
:1006A00030100B4040420F006CB2FF1F68B2FF1FBA
:1006B00064B2FF1F03F06AFF001BA842DFD8DBF81B
:1006C0000030D907F6D4444A444B1660536003F017
:1006D0005DFF434C054604E003F058FF401BA04279
:1006E000CDD83A683F4B1340002BF5D03E4B3E4AE5
:1006F0001B68C9F800301360D9F80020394B3B491A
:100700001340012BBBD13A4A1268D205B7D588F8FD
:100710000030384A00230B60029B1360364B1B7875
:10072000002B2FD1009B5B022B4834490360344AD5
:100730002B4D4FF481330B60324B33491160334AF8
:100740001A6003F023FF044604E003F01FFF001BC0
:10075000A84219D898F80030002BF6D1D9F800201B
:10076000294B1340022B0FD1009A029B01320092B9
:10077000049A03F50073934202930DD0019A936893
:10078000D0686CE7009BCFE7039840F2FD1232215E
:1007900002F0ECFF0028E7D1019BDA68079B0133E8
:1007A0009A4207937FF6CFAD019B07991B6941E7FA
:1007B000019CA168606901FB03F10133136004F13E
:1007C0001802FCF7CBFA00287FF4BDAD012796E5AF
:1007D0009847EAE6984705E708100B4000001A0D15
:1007E00040420F0001000F0030100B4064B2FF1FA9
:1007F00010100B4000100B4058B2FF1F04100B40AC
:1008000038100B400C100B4002007F1101003A1809
:100810002DE9F041DFF84C839AB0044640220AA843
:10082000002105F08BFCD8F80030FF2613F00107FB
:100830008DF861608DF8626000F0D284C64D04F5D9
:10084000245634363046F9F797FE96F874C28DF880
:1008500049C096F894C28DF84AC004F5285E96F80F
:10086000B4C28DF84BC0774696F8D4C28DF84CC010
:1008700004F529539EF829C08DF846C004F52A5086
:1008800097F849C09EF828808DF847C093F849C072
:100890008DF83D808DF840C097F8488090F828C0CA
:1008A0008DF841C007461430194604F52752407DA3
:1008B0008DF8420091F828C091F8290092F84C1068
:1008C0008DF83E80383204F52B5E93F84880527DD7
:1008D0008DF8480073468DF844108DF845208DF84A
:1008E0003F808DF843C096F8F4C196F814228DF835
:1008F0004E2096F8F5218DF8512034331A7D9EF85C
:10090000280097F8481096F834E296F854728DF85B
:100910004FE08DF8507096F815E296F835725B7DD1
:1009200096F855628DF84DC08DF852E08DF85370F1
:100930008DF854608DF855008DF856108DF85720BD
:100940008DF8583072B604F530531833DA6862B651
:10095000824F196A38680290029E586A9208711A8A
:10096000101A18BF1E625A6201299A6AB8BF012183
:100970000E46810291FBF6F132B1002904D040F31A
:100980006684002A40F3668402EB4202521848BF94
:10099000033293F8301092109A62002900F013820B
:1009A000002AB8BF52426E4E911E86FB0162A2EB36
:1009B000E1720132D96A02FB0012DA62ADF8282036
:1009C00072B604F531500C30C26862B639680391D2
:1009D000DDF80CE0016A466A9208C1EB0E01961B35
:1009E00018BFC0F820E042620129826AB8BF012125
:1009F0008E46B10291FBFEF132B1002904D040F3E2
:100A00002E84002A40F32E8402EB4202521848BF83
:100A1000033290F8301092108262002940F08283F5
:100A200082EAE271A1EBE2710239012940F31C84F0
:100A30008910A1F10B02A1F1040E22EAE272BEF1CB
:100A4000000FA8BF724401310A44C16A95F81DE045
:100A500002FB0612C262ADF82A2072B604F53252C9
:100A6000D26862B639680491049ED3F88810D3F82E
:100A70008C009208711A101A18BFC3F88860C3F866
:100A80008C200129D3F89020B8BF01210E468102A5
:100A900091FBF6F132B1002904D040F31F84002A03
:100AA00040F31F8402EB4202521848BF033293F80E
:100AB00098109210C3F89020002940F03F8382EAFA
:100AC000E271A1EBE2710239012940F30D84891032
:100AD0000A1FA1F10B0622EAE272002EA8BF9219AA
:100AE00001310A44BEF1000F03D0012A01D0013ABE
:100AF0005200D3F89410AE7F00FB0212C3F894208A
:100B0000ADF82E2072B604F532523432D26862B695
:100B100039680491DDF810E0D3F8BC10D3F8C000B8
:100B20009208C1EB0E01101A18BFC3F8BCE0C3F85D
:100B3000C0200129D3F8C420B8BF01218E4681020C
:100B400091FBFEF182B100290ED040F3CF83002A41
:100B500040F3CF8308E000BF8814FF1F80B2FF1F5F
:100B6000ABAAAA2A8414FF1F02EB4202521848BF04
:100B7000033293F8CC109210C3F8C420002940F03F
:100B8000198382EAE271A1EBE2710239012940F393
:100B9000B38389100A1FA1F10B0E22EAE272BEF1A3
:100BA000000FA8BF724401310A441EB1012A01D0CE
:100BB000013A5200D3F8C810EE7F00FB0212C3F8CE
:100BC000C820ADF8302072B604F533522832D2680E
:100BD00062B639680491DDF810E0D3F8F010D3F86C
:100BE000F4009208C1EB0E01101A18BFC3F8F0E030
:100BF000C3F8F4200129D3F8F820B8BF01218E46AC
:100C0000810291FBFEF132B1002904D040F35E83F2
:100C1000002A40F35E8302EB4202521848BF0332BF
:100C200093F800119210C3F8F820002940F0CD820B
:100C300082EAE271A1EBE2710239012940F34C83AF
:100C400089100A1FA1F10B0E22EAE272BEF1000F19
:100C5000A8BF724401310A441EB1012A01D0013AF1
:100C60005200D3F8FC1095F8206000FB0212C3F884
:100C7000FC20ADF8322072B604F534521C32D26832
:100C800062B639680491DDF810E0D3F82411D3F886
:100C900028019208C1EB0E01101A18BFC3F824E115
:100CA000C3F828210129D3F82C21B8BF01218E4691
:100CB000810291FBFEF132B1002904D040F31E8382
:100CC000002A40F31E8302EB4202521848BF03324F
:100CD00093F834119210C3F82C21002900F04C82B3
:100CE000002AB8BF52429A4E911E86FB0162A2EBC7
:100CF000E1720132D3F830619FED967A9FED966AEA
:100D000004F5025102FB0062C3F83021888D0B6BA1
:100D1000ADF8342003EB00134A6B03EBD3735B1085
:100D2000D01A0028B8BF4042B0F5807FC8BF1A462D
:100D300007EE902AF8EEE77A0B6377EEC77A01F1B7
:100D40001C0187EE867AC8BF8B61F7EE006AB4EEAD
:100D5000E67AF1EE10FA00F1FC814FF6FF7304F52C
:100D600088465436ADF82C3096F80531002B6AD001
:100D700096F8042102F0FF01002A64D096F80831A9
:100D8000032B00F05B83022B00F02283DFF8DC8171
:100D9000D8F80030DB0740F1D482DFF8D4813B681B
:100DA00098F800200793079B092A00F25D83DFE88B
:100DB00012F04A0392037A036C035E03B803AA039A
:100DC0009B0350031E0082EAE271A1EBE27102393B
:100DD000012940F341828910A1F10B020E1F22EA82
:100DE000E272002EA8BF921901310A44E2E5D6F85A
:100DF0008C3093F85C701D2F12D84FF000084346DA
:100E00003A46012186F806813046F0F7B9FCD6F85B
:100E10008C304146DF6503F14C02986CFBF79EFF76
:100E20004E4B41F2D43299588F4241F2E43118BF0F
:100E30009F504B4A01375F504A49116096F805317F
:100E4000002286F8042104F58942543251684F1C6F
:100E500004D04FF0FF308DF8621050609168481C4C
:100E600004D04FF0FF308DF861109060507896F804
:100E7000111197788DF85A0096F817218DF83B10CC
:100E80000020B6F812118DF83C2086F817014FF6B5
:100E9000FF72B6F81401ADF8361096F816118DF8F9
:100EA0006070A6F81221A6F81421ADF838008DF86C
:100EB0003A1053B196F8042196F806318DF85C206B
:100EC00001228DF859208DF85B3027490AA8FDF7DB
:100ED0009DFF44F2D6422B7FE97EA15463B196F880
:100EE0000731012786F8067133B9FF220321304606
:100EF000F0F746FC86F8077195F917701A4A002F2B
:100F0000C0F295811D2F40F37E8104F519501649DA
:100F10000C30F8F7FBFD95F8211042F2380349B385
:100F2000E15C002900F0B6812D7E6DB104F10C006A
:100F300004F538542946FAF7CDFA04F15002E56574
:100F4000E06C0021FBF70AFF1AB0BDE8F08100BF9A
:100F5000ABAAAA2A0000FA4300F47B47CC14FF1F77
:100F6000A428FF1FCDCC4C3F8814FF1FAC14FF1FDB
:100F7000B814FF1FE35CBE4F04F500562836002B63
:100F800040F0C4814FF480420021BA4805F0D6F801
:100F9000B948BA49F7F7B4FCB94804F10A0E00F5AC
:100FA000804C50F8043F190C1A0A01F4706122F4C5
:100FB0007F620A4303F0F003134384452EF8023F97
:100FC000EFD1706803689B68BB4240F0DD81EFF7AA
:100FD0008BFE42F228034FF00041E3581A681523B4
:100FE000D1625363D36A002BFCDA7068936B036899
:100FF0009B68BB4240F0C581EFF76CFE42F22803CC
:101000004FF00041E3581A681C23D1625363D36A3E
:10101000002BFCDA7068936B03689B68BB4240F05E
:10102000AD81EFF757FE42F228034FF00041E3583D
:101030001A685B23D1625363D36A002BFCDA7068B1
:10104000936B03689B68BB4240F09581EFF74CFEC1
:1010500042F228034FF00041E3581A687523D16229
:101060005363D36A002BFCDA7068936B03689B6848
:10107000BB4240F07D81EFF72DFE42F228034FF096
:101080000041E3581A680023D1625363D36A002BEE
:10109000FCDA7068936B03689B68BB4240F0658123
:1010A000EFF718FE42F228034FF00041E3581A68A8
:1010B0003F23D1625363D36A002BFCDA7068936BD1
:1010C00003689B68BB4240F04D81EFF70DFE42F292
:1010D00028034FF00041E3581A685C23D162536340
:1010E000D36A002BFCDA7068936B0368F6689B6820
:1010F000BB4240F04C81EFF7EDFD42F2280306F5CC
:10110000FF50E3581A68711E1F304FF0004611F867
:10111000013FD6625363D36A002BFCDA8142936BA2
:10112000F5D101E7002AB8BF5242DFF858E1911E1D
:101130008EFB01E2A2EBE172013286E4002AB8BF25
:1011400052425049023A81FB0261A1EBE2714A1C12
:10115000CFE4DFED4D7AB4EEE77AF1EE10FA40F32A
:10116000EE80DFED4A6AE7EE267AFCEEE77ACDED17
:10117000017ABDF80430F2E582EAE271A1EBE27196
:101180000239012940F3C0808910A1F10B02A1F1BD
:10119000040E22EAE272BEF1000FA8BF72440131D0
:1011A0000A44002E3FF4A6AD012A1CBF02F1FF3213
:1011B00052009FE5002AB8BF52423249023A81FBF1
:1011C0000261A1EBE2714A1CF4E4002AB8BF52426A
:1011D0002C49023A81FB0261A1EBE2714A1C40E515
:1011E000404602F0FDFC2A4D00283FF428AB39466A
:1011F0002846232204F0A2FF4046AE75EE7502F0A9
:10120000F5FCFFF71CBB4FF0000886F8068143464B
:10121000FAB201213046F0F7B3FAD6F88C304146E5
:10122000DF6503F14C02986CFBF798FD6DE692F9CF
:101230001670002FC0F2B0801D2F3FF766AE4FF042
:10124000000886F806814346FAB20221E2E7002A46
:101250007FF79AAB002199620122FFF7ABBB002A0E
:101260007FF7D2AB002181620122FFF7EEBB00BF06
:10127000310C00003070FF1FD407FF1FCC14FF1F7C
:101280002C70FF1FABAAAA2A0000000000FF7F47B6
:101290008814FF1F04F50053B94AD86A03689B6895
:1012A000934277D1EFF720FD42F228034FF000413F
:1012B000E3581B68AE22D9625A63DA6A002AFCDA64
:1012C00042F2380201219B6BA1542DE6002A7FF7E0
:1012D000A2AC0021C3F8F8100122C2E4002A7FF773
:1012E000E1AB0021C3F89010012202E4002A7FF74D
:1012F0003BAC0021C3F8C41001225BE4002A7FF755
:10130000E2AC0021C3F82C110122F3E470680368F9
:101310009B68BB4224D1EFF7E7FC42F228034FF071
:101320000041E3581B68AF22D9625A63DA6A002A87
:10133000FCDA42F2380200219B6BA15422E6002322
:101340000DE5404602F04CFC00283FF426AD3B681A
:1013500008938C4B089A1A60404602F047FC1CE543
:101360009847DAE700219847B1E60121984799E6C6
:101370000121984781E60021984769E601219847B5
:1013800051E60121984739E60021984721E60121DD
:101390009847B2E6984787E7537E002B40F0D88005
:1013A000917E002940F0CE8092F82270002F00F04C
:1013B000D68096F81031002B7FF4A7AD1123FF22C1
:1013C000E0213046F0F7DCF9012386F810319CE586
:1013D000D6F80C21D6F88C30106893F85C7003F0C6
:1013E000F7F8FF22142100233046F0F7C9F9D6F8A8
:1013F0000C31986803F0ECF80023FF2216213046E8
:10140000F0F7BEF9D6F80C31D86803F0E1F81D2FDB
:1014100040F2C2805C4B41F2D43241F2E430995840
:101420008F4218BF9F50594A5949116001371F50C8
:10143000002386F8043196F8053104E500220B46B6
:1014400086F80421FFE4012388F8003096F805317E
:10145000F9E44C49D6F80C210968D2685B1A93422A
:1014600084BF092388F8003096F80531EBE4454A3B
:10147000D6F80C11126889689B1A8B42F4D905239F
:1014800088F8003096F80531DDE43E4AD6F80C11B4
:10149000126849689B1A8B42E6D9022388F800300B
:1014A00096F80531CFE40023FF221A213046F0F7E9
:1014B00067F9384A39681368099101333E2B31497D
:1014C0001360099808608CBF0423032388F8003058
:1014D00096F80531B7E42B4AD6F80C111268096862
:1014E0009B1A8B42C0D9D8E70023FF221621304631
:1014F000F0F746F93B680593224B059A1A600823DA
:1015000088F80030B0E71F4AD6F80C1112688968D5
:101510009B1A8B42A8D9072388F8003096F805312A
:1015200091E40023FF2214213046F0F729F93B68AB
:101530000693144B069A1A60062388F8003096F832
:10154000053180E43046FF221721F0F719F9DCE479
:1015500030460023FF221621F0F712F9D5E496F861
:101560001131002B3FF4D1AC1123FF22E32130468F
:10157000F0F706F986F8107186F81171C5E400BF1E
:10158000310C0000B014FF1FCC14FF1FA428FF1F54
:10159000CDCC4C3FB414FF1F4FF0000843463A46F1
:1015A00086F8068101213046F0F7EAF8D6F88C304B
:1015B0004146DF6503F14C02986CFBF7CFFB29E74E
:1015C0002DE9F04F2DED028B4FF48D721F4B0280F1
:1015D000436002218BB08346102002F09BFF102055
:1015E00002F08AFF1A4B1B4A1B4E002814BF1846F4
:1015F000104600F5A0710368426806EBC30308308B
:101600005B6881421A60F6D1144A1548136F04686A
:10161000D2F86C80134ADFF850C0126801920BF5C3
:101620000051234301240C7442F20C0444F20101E2
:101630000BF10C070360DCF800204BF8048007F581
:10164000005EC8F8001000241BE000BF9CB201003F
:101650005CB70100B8AF010010BD010028BA01005D
:101660003C80044018BA010000BB01005CF8310066
:10167000821A93420246C1F0BD833F2901F0C6841D
:101680000C46C04BC04D611C9B1A0CEBC10A002BD1
:10169000ECD10CEBC4046368019ABC48DFF80CC3BE
:1016A00042F0625545F400152B43C8F80C3042F265
:1016B0001803C8F800C00BF50051C0F804E0B448A6
:1016C0004BF803001D20C8610C460A4642F2200177
:1016D00042F22803AE4D4BF801501A2151622834D2
:1016E0004BF803E007F5005207F500530C321433B2
:1016F000E7606260A360012102F00CFFA068A54AC8
:1017000003681B6807F50057934207F11C0741F077
:1017100079840079012102F0FDFE322002F058FFA9
:10172000A0689D4D03689B68AB4241F06784EFF76A
:10173000D1FA0A2002F04CFFA06803689B68AB4214
:1017400041F05884EFF7D0FA0A2002F041FFA06878
:1017500003689B68AB4241F04984EFF7BBFA322043
:1017600002F036FF3846F9F759FB42F238038B4A4C
:1017700000210BF8031002F580704FF0FF310023B9
:10178000D15003F58073B3F5804FF9D10432824212
:10179000F5D183490BF10A0001F5804751F8043F68
:1017A0004FEA134E1A0A0EF4706E22F47F624EEA6C
:1017B000020203F0F00313438F4220F8023FEDD101
:1017C000606803689B68AB4241F00C84EFF78CFAC9
:1017D00042F228034FF000415BF803301A681523EA
:1017E000D1625363D36A002BFCDA6068936B0368A1
:1017F0009B68AB4241F0F283EFF76CFA42F22803A8
:101800004FF000415BF803301A681C23D162536328
:10181000D36A002BFCDA6068936B03689B68AB4269
:1018200041F0D883EFF756FA42F228034FF0004117
:101830005BF803301A685B23D1625363D36A002BD1
:10184000FCDA6068936B03689B68AB4241F0BE832F
:10185000EFF74AFA42F228034FF000415BF80330F9
:101860001A687523D1625363D36A002BFCDA60686F
:10187000936B03689B68AB4241F0A483EFF72AFAAD
:1018800042F228034FF000415BF803301A6800234E
:10189000D1625363D36A002BFCDA6068936B0368F0
:1018A0009B68AB4241F08A83EFF714FA42F22803B7
:1018B0004FF000415BF803301A683F23D162536355
:1018C000D36A002BFCDA6068936B03689B68AB42B9
:1018D00041F07083EFF708FA42F228034FF000411D
:1018E0005BF803301A685C23D1625363D36A002B20
:1018F000FCDA6068936B0368E4689B68AB4241F074
:101900005583EFF7E7F942F2280304F5FF505BF83F
:1019100003301A68611E1F304FF0004411F8013F78
:10192000D4625363D36A002BFCDA8842936BF5D1FF
:101930001C4B1C495C68086822689B68DFF870C013
:10194000DFF870E00BF500510D463C352F460BF5E6
:101950000151049542F23C0543EA02080022124B71
:101960004BF805303A713A737A733A610A654A6501
:10197000C4F80080B8600270BB685A70BB689A7087
:10198000BB6819E080F0FA0200BB010078B2FF1FCB
:101990007CAC0100550C0000310C00003070FF1FC2
:1019A0002C70FF1F50B9010070AC010000003F8097
:1019B000008793039F860100FF21D970BB685A718D
:1019C000BB6850219971BB68DA71B9688B7803F0F4
:1019D0007F038B70BB6890461222DA70C246C14604
:1019E0004FF0FF350123164903FA08F0002207E003
:1019F000BD4202D93D469146C2460132402A18D026
:101A000031F8023F00FB03F3BCFBF3F3C3F5C3372C
:101A1000A3F5C334734507F1A007A4F1A004E7D9E7
:101A2000A542EAD9C246914664B10132402A254610
:101A3000E6D1B8F1020F05D008F10108D2E700BFE6
:101A400096B9010042F2440209F03F035BF802201C
:101A5000049F43EA8A13DBB25370BA68537943F0A8
:101A600020035371BA68537943F080035371BA6805
:101A7000937843F0800393703B79BC4A03EB4303B4
:101A800002EBC3030121DB685A09920002F16042B4
:101A900002F5614203F01F030BF5025499401C3418
:101AA000116042F29C0EB24900230F604FF00E0805
:101AB0004BF80E30A01C4FF01F0E4FF0430A04F1FC
:101AC000040CA21D422104F108054FF00F096360C8
:101AD000A360E36023826361A36104F11003C4F88F
:101AE0003CE0C4F81C90A062C4F82CA0C4F830C03C
:101AF0006163A26324624FF02309C4F82480242781
:101B00002364C4F844A0A5662065C4F858C004F155
:101B10000A004FF0220C2266C4F8883004EB080259
:101B20002123272504F10C0AE367E166C4F884E069
:101B30002067C4F874C0C4F8802002211020A46477
:101B4000C4F86480C4F84C906765E565C4F878A073
:101B500002F0E0FC102002F0CFFC00280CBF0123B3
:101B6000002384F88C3041F03F8104F144094FF0A8
:101B70000908804BC4F890800BF50452154693E891
:101B8000030042F2301734354FF0040E4FF0010CD1
:101B900042F234140BF807E082F831C005EB0E076F
:101BA000754A4BF8042003F1080E87E803009EE80D
:101BB00003000BF5055282E8030000212975C5F8E2
:101BC0008412C5F888126D486D496E4AAA610D608D
:101BD000016841F000610160916821F00C019160A1
:101BE000916841F004019160516A41F00401516231
:101BF000516A21F003015162516A41EA0C015162BC
:101C0000D16841F00801D160916841F00301916011
